:100000000C948B210C94BC210C94BC210C94BC212D
:100010000C94BC210C94BC210C94BC210C94BC21EC
:100020000C94BC210C94BC210C94BC210C94BC21DC
:100030000C94BC210C94198C0C94BC210C94BC2104
:100040000C94BC210C94C7750C94BC210C94BC215D
:100050000C94BC210C94BC210C946DCB0C94CF8BD4
:100060000C94BC210C947E3F0C94743F0C94BC21E6
:100070000C94BC210C94BC210C94BC210C94BC218C
:100080000C94BC210C94BC210C94BC210C94BC217C
:100090000C94BC210C94BC210C94BC210C94BC216C
:1000A0000C94BC210C94BC210C94BC210C94BC215C
:1000B0000C94BC210C94BC210C94BC210C94BC214C
:1000C0000C94BC210C94BC210C94BC210C94BC213C
:1000D0000C94BC210C94BC210C94BC210C94BC212C
:1000E0000C94BC21234B9249CB495F4BCB49CB4964
:1000F000CB49CB49CB49CB49CB49CB49CB49CB4960
:10010000CB49CB49CB49CB49CB49CB49CB49CB494F
:10011000CB49CB49CB49CB49CB49CB49CB49CB493F
:10012000594BCB49CB49CB49CB49CB49CB49CB499F
:10013000CB49324BCB49CB49CB49CB49CB49CB49B6
:10014000CB49CB49CB49CB49764BC849AD63966384
:10015000BC6399639363BF639C63A8639F63BA6343
:10016000A263A56346F649F638F63CF642F680F6F9
:100170004DF651F657F65BF65FF665F669F66DF6E5
:1001800080F673F677F67BF6A1F9A6F9ABF9B5F927
:10019000BFF938FAC9F9D1F9D9F9E3F9EDF9F7F965
:1001A00006FA10FA38FA1AFA24FA2EFA084AD73B55
:1001B0003BCE016E84BCBFFDC12F3D6C74319ABD36
:1001C00056833DDA3D00C77F11BED9E4BB4C3E915A
:1001D0006BAAAABE000000803F05A84CCDB2D44E49
:1001E000B93836A9020C50B9918688083CA6AAAA4B
:1001F0002ABE000000803F000D9496140C94B26259
:100200000C9487D60C94A1F90C9413490C94C980D2
:100210000C9438FA0D948A390C94B5D60C94A863D2
:100220000C94F7F90D947B110C942E600C9488FFBC
:100230000D9457110C942DFD0C94A2630C94226024
:100240000C949D8E0C94764B0C9469C30C949C6317
:100250000C948ADC0D94750F0C94C8490C94018D94
:100260000C94594B0C941AFA0C94468D0C94ABD800
:100270000C94BA630D9416000D948E140C946DF6C4
:100280000C94368D0D94E80F0C94F85B0C9449F6A1
:100290000C9447440C943F6A0C94D1DD0C945F4B52
:1002A0000D946F110C94A48E0C9446F60C94CACC49
:1002B0000C943CF60C94D5DD0C94B7900C94CB497F
:1002C0000C94EDF90C9483FF0C945D510C9465F63D
:1002D0000D941A100D94F0100C94BD5C0C94DFFC7E
:1002E0000C947EFF0C94BAD80C9428FD0C9498477B
:1002F0000C9487D70C9451F60C94B4FF0C9496DCB4
:100300000D9439100C94248D0D9458100C940749B9
:100310000C940A490C94A5630C9448600C94BF6338
:100320000D94FF100D9475110C94015C0C9432FD2A
:100330000C9410FA0D94A5140C941C660C945B5D3F
:100340000C9475CC0C94E3F90C9423FD0C94A192BD
:100350000C94DFCC0C94AD630C94A28B0D94E11043
:100360000C94C53F0C9448670C946F660C94FB6525
:100370000C9406FA0C9487510C94095C0C94CCD81C
:100380000C9434600C9491410C94AEFF0C941EFDBF
:100390000C94A2FF0C946ED70C9483D80C9424FA7E
:1003A0000D94BC010D948E0F0C943C600D94631160
:1003B0000C944DF60C9496630C94488D0C94D9F9DA
:1003C0000C94C0D80C943E4D0C9444600C94BFF92E
:1003D0000C9499630C94D9DD0C94E3CC0C9486D8DE
:1003E0000D9469110C94C73F0C94C6CC0C94C93F72
:1003F0000C9469F60C9493630D9481110D94A90FDC
:100400000C94A8FF0C944A8D0C948CD80C94BC636B
:100410000D9492140C94CD3F0C945C510D940E00ED
:100420000C94D95B0C94DBCC0D946C390C9457F67E
:100430000C94C9F90D943F110C94CB3F0C94DDDD65
:100440000C94B5F90D945D110C949F630C94C263E8
:100450000C943ADA0D94DB100C94ABF90C942766EB
:100460000C94C6D80C945BF60C94D0630C9480F674
:100470000C9498D80C94C45B0C94CC8B0C94605165
:100480000C94B1650C94F45D0C947BF60C945FF6BF
:100490000C9430670C944C600C94548E0C946C6FDC
:1004A0000D94BA100C94234B0C9489D80D94EF0042
:1004B0000C9440600C942EFA0C94D1F90D94BC0F5E
:1004C0000C949B650C9477F60C9438600C94A6F908
:1004D0000C9415940C9473F60C9492490C9442F677
:1004E0000C94E9510D9401100C9422490C94419400
:1004F0000D9490140C942D8D0C94D75B0D94481191
:100500000D94CF0F0D9494140C94BAFF0C94A0D7B3
:100510000C94CD5E0C945BD70C94E4650D9497120B
:100520000C94324B0C9438F64E414E494E49545976
:10053000494E46CDCCCC3D0AD7233C17B7D13877AE
:10054000CC2B329595E6241FB14F0A0000204100C4
:1005500000C84200401C4620BCBE4CCA1B0E5AAE0E
:10056000C59D7400407A10F35A00A0724E1809001D
:1005700010A5D4E80000E87648170000E40B540208
:100580000000CA9A3B000000E1F505000080969843
:1005900000000040420F000000A086010000001093
:1005A0002700000000E803000000006400000000D5
:1005B000000A00000000000100000000002C76D8B6
:1005C00088DC674F0823DFC1DFAE59E1B1B796E59C
:1005D000E3E453C63AE651997696E8E6C28426EB00
:1005E000898C9B62ED407C6FFCEFBC9C9F40F2BA13
:1005F000A56FA5F490055A2AF75C936B6CF9676DAB
:10060000C11BFCE0E40D47FEF520E6B500D0ED90FF
:100610002E0300943577050080841E080000204ECC
:100620000A000000C80C333333330F986E12831165
:1006300041EF8D2114893BE65516CFFEE6DB18D13C
:10064000844B381BF77C1D901DA4BBE4242032840E
:10065000725E228100C9F124ECA1E53D27434F4D94
:100660004D554E49434154494F4E004452595255FD
:100670004E004552524F525300494E464F0045439B
:10068000484F0047322F4733206261642070617207
:10069000616D65746572730A005265706F732E2EFA
:1006A0002E004D65736820706F696E74206F7574CD
:1006B000206F662072616E67650A00417474656E12
:1006C0007465207574696C69732E00496D70726968
:1006D0006D616E746520696E636F727265637465B7
:1006E000004D6F746575727320626C6F7175C3A96C
:1006F0007300456E642066696C65206C6973740ACA
:1007000000426567696E2066696C65206C69737468
:100710000A00286E6F2066696C6529004375727245
:10072000656E742066696C653A20005344207072CF
:10073000696E74696E67206279746520004E6F740B
:10074000205344207072696E74696E670A0050729B
:10075000696E742074696D653A2000496E76616C2B
:1007600069642050696E204D6F64650A000A5374F5
:100770006174733A2046696C616D656E742075739F
:1007800065643A20002C204C6F6E67657374206A94
:100790006F623A2000546F74616C2074696D653A21
:1007A00020002C204661696C65643A20002C2046AC
:1007B000696E69736865643A20005072696E74737B
:1007C0003A200053746174733A2000526566726F68
:1007D0006964697373656D656E7400452025530007
:1007E0006F66660044454255473A004D313132202C
:1007F00053687574646F776E004D31313320530048
:10080000526566726F69642E206475206C69742E5F
:100810002E2E004C697420656E20636861756666D3
:10082000652E2E2E00534F564F4C205356303120FC
:100830004F46462E002F2F20004D31343520533C9B
:10084000696E6465783E206F7574206F66207261F2
:100850006E67652028302D31290A00416363656C7D
:1008600065726174696F6E3A2050003F4A206F755F
:1008700074206F662072616E67652028302E3031DB
:1008800020746F20302E33290A0046523A00204649
:100890006C6F773A200050726F74656374656420E2
:1008A00050696E0A004D424C2041646A7573742091
:1008B0005A0020643A0020693A0020703A006469C6
:1008C000730043290A0061626C656420286D696EBB
:1008D0002074656D702000436F6C642065787472BD
:1008E0007564657320617265200046696C616D6591
:1008F0006E742072756E6F7574200044C3A96361B5
:100900006C61676573206170706C697175C3A973E0
:10091000004572723A20546F6F2066617221005454
:100920006F6F206661722066726F6D2072656665FA
:1009300072656E636520706F696E740A004545507C
:10094000524F4D204F4B0A00506F7765722D6C6FE0
:100950007373207265636F766572792000446F6EE1
:1009600065207072696E74696E672066696C650ACD
:10097000004D3737004D3331007E06790672066B25
:10098000065D064572726F722077726974696E67D0
:1009900020746F20454550524F4D210A004D34318F
:1009A00030004D313132004D3130380053544F500A
:1009B00050C389005072696E7465722073746F70D1
:1009C0007065642064756520746F206572726F7243
:1009D000732E2046697820746865206572726F7284
:1009E00020616E6420757365204D39393920746F2C
:1009F00020726573746172742E202854656D706561
:100A00007261747572652069732072657365742EE6
:100A10002053657420697420616674657220726564
:100A20007374617274696E67290A004E6F2043689F
:100A300065636B73756D2077697468206C696E658A
:100A4000206E756D6265722C204C617374204C6948
:100A50006E653A2000636865636B73756D206D6920
:100A6000736D617463682C204C617374204C696EE3
:100A7000653A20004C696E65204E756D6265722086
:100A80006973206E6F74204C617374204C696E65BD
:100A9000204E756D6265722B312C204C6173742071
:100AA0004C696E653A20004D31313000534420725C
:100AB000656164206572726F720A002121204B49C2
:100AC0004C4C20636175736564206279204B494CFE
:100AD0004C20627574746F6E2F70696E0A0021214C
:100AE000204B494C4C20636175736564206279200A
:100AF000746F6F206D75636820696E6163746976C9
:100B0000652074696D65202D2063757272656E7441
:100B100020636F6D6D616E643A2000627573793A7F
:100B20002070617573656420666F7220696E7075E0
:100B3000740A00627573793A207061757365642078
:100B4000666F7220757365720A00627573793A2058
:100B500070726F63657373696E670A004DC3A96431
:100B60006961207265746972C3A9004DC3A9646983
:100B70006120696E73C3A972C3A9004D3130303052
:100B80002053004D36303000363726033C3D380EBA
:100B90002E303E121A1C180AFF43080908440001AF
:100BA00043686172676572206D6D00526574726191
:100BB0006974206D6D004469616DC3A8747265200D
:100BC00066696C2E004520656E206D6DC2B30020F5
:100BD000082046616374657572002008204D6178B5
:100BE000002008204D696E0054656D702E204175FF
:100BF000746F2E00566D696E20636F757273650099
:100C0000566D696E00566D6178204500566D6178AD
:100C1000205A00566D6178205900566D6178205831
:100C200000416D6178204500416D6178205A004196
:100C30006D6178205900416D6178205800416363EF
:100C40002E636F75727365004163632E72C3A9745E
:100C500072616374696F6E0043616973736F6E00D4
:100C600025697920256964202569682025696D201A
:100C70002569730023646566696E652044454641B5
:100C8000554C545F004B6420004B6920004B702092
:100C900000504944204175746F74756E6520666913
:100CA0006E697368656421205075742074686520CE
:100CB0006C617374204B702C204B6920616E642032
:100CC0004B6420636F6E7374616E74732066726F11
:100CD0006D2062656C6F7720696E746F20436F6E54
:100CE00066696775726174696F6E2E680A00504993
:100CF00044204175746F74756E65206661696C651A
:100D000064212074696D656F75740A000A20436C54
:100D1000617373696320504944200A00204B643A90
:100D20002000204B693A2000204B703A20002054CC
:100D3000753A2000204B753A2000206D61783A20EA
:100D400000206D696E3A200020643A20002062691C
:100D500061733A2000504944204175746F74756E78
:100D6000652073746172740A00504944204175749F
:100D70006F74756E65206661696C656421205465C9
:100D80006D706572617475726520746F6F2068692B
:100D900067680A00504944204175746F74756E6528
:100DA00000504944204175746F74756E652066610A
:100DB000696C656421204261642065787472756491
:100DC0006572206E756D6265720A004572723A2016
:100DD0007574663820666F6E74206E6F7420696E4D
:100DE000697469616C697A65642E00000C0F00FEFD
:100DF00007022603BC01FFFE0AFE08FE05080806DE
:100E0000000040F0C888889878100508080600009F
:100E1000C0F88888888888F8050505060001203014
:100E2000F830200508080600002070F82020202057
:100E3000E00509090600FF2070A8A8B8888870207E
:100E4000050606060001E08CEA8C8A0A05090906F7
:100E500000FFF8A88888888888A8F8050A0A06008C
:100E6000FE205050505088A8A88870030303060045
:100E70000340A040FFFFFFFFFFFFFFFFFFFFFFFF5B
:100E8000FFFFFFFFFFFFFFFFFFFF0000000605FF62
:100E90000107070602008080808080008003030332
:100EA000060105A0A0A005060606000050F8505057
:100EB000F8500509090600FF2070A8A07028A87046
:100EC00020050707060000C8C810204098980507AD
:100ED0000706000040A0A040A89068010303060296
:100EE000058080800309090601FF20404080808042
:100EF0004040200309090601FF8040402020204097
:100F0000408005070706000020A8702070A8200573
:100F100005050600012020F820200203030601FF3A
:100F2000C04080050101060003F80202020601002C
:100F3000C0C00507070600000810102040408005CB
:100F40000707060000708898A8C88870030707067E
:100F5000010040C040404040E00507070600007027
:100F60008808102040F8050707060000F808103030
:100F700008887005070706000010305090F8101020
:100F8000050707060000F880F008088870050707C5
:100F9000060000304080F0888870050707060000D2
:100FA000F808101020202005070706000070888828
:100FB0007088887005070706000070888878081018
:100FC00060020505060100C0C000C0C0020606069A
:100FD00001FFC0C000C0408003050506010120409C
:100FE000804020050303060002F800F8030505060B
:100FF000010180402040800507070600007088102E
:10100000202000200507070600007088B8A8B880D7
:1010100070050707060000708888F888888805072B
:1010200007060000F04848704848F005070706002A
:101030000070888080808870050707060000F048EF
:1010400048484848F0050707060000F88080F0800F
:1010500080F8050707060000F88080F08080800592
:1010600007070600007088808098887005070706CB
:101070000000888888F8888888030707060100E050
:101080004040404040E005070706000038101010BF
:101090001090600507070600008890A0C0A0908807
:1010A000050707060000808080808080F80507071C
:1010B00006000088D8A888888888050707060000E9
:1010C0008888C8A89888880507070600007088885F
:1010D00088888870050707060000F08888F08080FF
:1010E0008005070706000070888888A890680507B3
:1010F00007060000F08888F0A09088050707060022
:101100000070888070088870050707060000F820C6
:10111000202020202005070706000088888888886E
:1011200088700507070600008888888850502005C9
:10113000070706000088888888A8A85005070706C2
:10114000000088885020508888050707060000881E
:10115000885020202020050707060000F8081020EE
:101160004080F80309090601FFE0808080808080CC
:1011700080E00507070600008040402010100803AB
:1011800009090601FFE020202020202020E005039F
:10119000030600052050880501010600FEF8030340
:1011A000030601058040200505050600007008784B
:1011B00088780507070600008080F0888888F00599
:1011C000050506000070808088700507070600008E
:1011D000080878888888780505050600007088F07A
:1011E0008070050707060000304840E04040400599
:1011F00007070600FE7088888878087005070706CC
:1012000000008080F0888888880307070601004076
:1012100000C0404040E00409090601FE1000301003
:10122000101010906005070706000080808890E08D
:101230009088030707060100C04040404040E00599
:101240000505060000D0A8A8A8A805050506000009
:10125000B0C88888880505050600007088888870F1
:101260000507070600FEF0888888F08080050707DC
:101270000600FE78888888780808050505060000BD
:10128000B0C880808005050506000078807008F0F1
:101290000507070600002020F82020201805050576
:1012A000060000888888986805050506000088887B
:1012B0008850200505050600008888A8A850050567
:1012C0000506000088502050880507070600FE88A4
:1012D000888850204080050505060000F810204051
:1012E000F80309090601FF204040408040404020AB
:1012F0000109090602FF8080808080808080800351
:1013000009090601FF80404040204040408005031D
:101310000306000248A890FFFFFFFFFFFFFFFFFF4B
:10132000FFFFFFFFFFFFFFFFFFFFFFFFFFFFFFFFCD
:10133000FFFFFFFFFFFFFFFF0000000605FF0107A3
:101340000706020080008080808080050707060075
:10135000FF2070A8A0A870200507070600003048ED
:1013600040E04048B0050505060000A8508850A898
:101370000507070600008850F820F820200107071D
:10138000060200808080008080800408080601003A
:1013900070806090906010E0030101060107A006D4
:1013A00007070600007884B4A4B484780305050612
:1013B000010460A06000E00505050600002850A0BB
:1013C0005028050303060001F8080803010106017F
:1013D00003E00607070600007884B4A4A484780517
:1013E0000101060007F804040406010560909060FE
:1013F0000507070600002020F8202000F803050557
:1014000006010440A02040E0030505060104C020B9
:101410004020C0030303060105204080050707069E
:1014200000FE88888898E880800508080600007813
:10143000E8E8E868282828020202060203C0C00380
:1014400002020601FE20C003050506010440C0405B
:1014500040E003050506010540A04000E005050544
:10146000060000A0502850A0050A0A06000040C04F
:1014700048506050B0507810050A0A06000040C07D
:1014800048506050A8081038050A0A060000C0201D
:101490004830E050B05078100507070600002000E3
:1014A0002020408870050A0A06000040200070884D
:1014B00088F8888888050A0A0600001020007088CD
:1014C00088F8888888050A0A06000020500070887D
:1014D00088F8888888050A0A06000068B0007088C5
:1014E00088F88888880509090600005000708888F7
:1014F000F8888888050A0A0600002050207088882D
:10150000F888888805070706000078A0A0F0A0A04A
:10151000B80509090600FE70888080808870106018
:10152000050A0A060000402000F88080F08080F85C
:10153000050A0A060000102000F88080F08080F87C
:10154000050A0A060000205000F88080F08080F82C
:101550000509090600005000F88080F08080F8033B
:101560000A0A060100804000E04040404040E0039D
:101570000A0A060100204000E04040404040E003ED
:101580000A0A06010040A000E04040404040E0035D
:101590000909060100A000E04040404040E0050786
:1015A00007060000704848E8484870050A0A060027
:1015B0000068B0008888C8A8988888050A0A0600CC
:1015C0000040200070888888888870050A0A060014
:1015D0000010200070888888888870050A0A060034
:1015E0000020500070888888888870050A0A0600E4
:1015F0000068B0007088888888887005090906002E
:1016000000500070888888888870050505060001EC
:1016100088502050880509090600FF087098A8A87E
:10162000A8C87080050A0A06000040200088888843
:1016300088888870050A0A060000102000888888BB
:1016400088888870050A0A0600002050008888886B
:1016500088888870050909060000500088888888F5
:10166000888870050A0A060000102000888850202B
:1016700020202004070706010080E0909090E08081
:10168000050707060000708890A09088B00508083C
:1016900006000040200070087888780508080600D9
:1016A00000102000700878887805080806000020DF
:1016B0005000700878887805080806000068B000B7
:1016C00070087888780507070600005000700878D1
:1016D000887805080806000020502070087888786F
:1016E000050505060000702870A0780507070600AC
:1016F000FE70888088701060050808060000402091
:10170000007088F080700508080600001020007046
:1017100088F080700508080600002050007088F0EE
:10172000807005070706000050007088F080700385
:101730000808060100804000C0404040E00308085F
:10174000060100204000C0404040E00308080601B8
:101750000040A000C0404040E0030707060100A091
:1017600000C0404040E00509090600005020500834
:10177000788888887005080806000068B000B0C83E
:10178000888888050808060000402000708888883E
:101790007005080806000010200070888888700511
:1017A0000808060000205000708888887005080826
:1017B00006000068B000708888887005070706007A
:1017C000005000708888887005050506000120001B
:1017D000F800200505050600007898A8C8F005085F
:1017E00008060000402000888888887005080806E0
:1017F000000010200088888888700508080600000E
:10180000205000888888887005070706000050006F
:101810008888888870050A0A0600FE1020008888DB
:1018200088502040800509090600FE8080F08888E5
:1018300088F080800509090600FE500088888850DD
:10184000204080534F564F4C20535630310052C3E6
:10185000A96375702E20636F75702E00436F6E66DE
:10186000696775726174696F6E0052657072656E3A
:1018700064726520696D70722E00256C642E256976
:101880006D00546F74616C2066696C616D656E7477
:1018900000496D70722E206C61202B206C6F6E677A
:1018A0007565003E200054707320696D70722E20A3
:1018B000746F74616C005465726D696EC3A9657351
:1018C000004E62726520696D7072657373696F6E28
:1018D0007300313235004245443A4550434F53205E
:1018E0003130304B0050726F74656374696F6E20D5
:1018F0006163746976650054656D70204D61780090
:101900003237350054656D70204D696E0045313AAF
:10191000204550434F53203130304B00416C696DAE
:101920002E004D45414E2057454C4C0050726F746F
:101930006F636F6C6500312E300042617564730017
:101940003131353230300052414D505320312E3339
:10195000004E697665617520706172206772696CEE
:101960006C65004578747275646575727300323009
:1019700032302D30382D32380053746174732E207C
:10198000696D7072696D616E746500546865726D21
:10199000697374616E63657300496E666F7320636B
:1019A0006172746500496E666F7320696D7072694B
:1019B0006D616E7465004D3130303000417272C31C
:1019C000AA74657220696D70722E0053746F700076
:1019D00041637475616C69736572206DC3A9646934
:1019E00061004D323100506173206465206DC3A9E0
:1019F0006469610052C3A9676C65720050617573B8
:101A00006520696D7072657373696F6E00537572CE
:101A10007665696C6C6572005072657373657220CF
:101A20006C6520626F75746F6E00706F75722063E5
:101A3000686175666665722E2E2E0000496E73C34E
:101A4000A97265722066696C616D656E740065745B
:101A5000206170702E20626F75746F6E00706F75EC
:101A60007220636F6E74696E7565722E2E2E004142
:101A70007474656E7465006368617267656D656E28
:101A8000742066696C616D656E74000050726573D8
:101A900073657220626F75746F6E00706F7572205F
:101AA00072657072656E6472650000417474656E73
:101AB0007465207265707269736500696D70726516
:101AC0007373696F6E0000417474656E74650050C5
:101AD000757267652066696C616D656E7400004D96
:101AE00069736520C3A0206E6976656175204F4BD0
:101AF0002100506F696E742073756976616E740091
:101B00002569202F202575004732392053310043A5
:101B10006C696320706F757220636F6D6D656E63A5
:101B20006572004F726967696E652058595A2E2E8A
:101B30002E004E69766561752064657320636F6958
:101B40006E730048617574657572206C697373C338
:101B5000A965004E6976656175206475206C6974AD
:101B600000562E72C3A9742E207265707269736557
:101B70000052C3A9742E72657072697365206D6D11
:101B80000053617574205A206D6D005669742E20C3
:101B900072C3A97472616374C2B00052C3A9747233
:101BA0006163746174696F6E206D6D0052C3A974B6
:101BB00072616374696F6E206175746F001FE0203D
:101BC000102010201010201020201020103030087D
:101BD00040048003001FE03FF03FF03FF01FE01F94
:101BE000E03FF03FF03FF00FC0078003003FFFF001
:101BF00038007030FC3020FC102078102030102C81
:101C000000D02E31D02F7BD02F7BD02E31D02C0086
:101C1000D020301020781020FC1030FC30380070BC
:101C20003FFFF03FFFF038007031863023871027E8
:101C300087902F87D02F03D0203010207810207865
:101C4000102030102F03D02F87D0278790238710A4
:101C50003186303800703FFFF01FFFF81FFFF80497
:101C60001040020820020820041040082080104183
:101C7000001041000820800410400000001FFFF801
:101C80001FFFF81EF79C043F633E0C6363633C60D8
:101C900063630C6063630C3C63630C1E36630C036C
:101CA00036630C0336630C631C630C7E1C3E3F3CA6
:101CB000081C3F2568753A2530326875002530329A
:101CC00068753A25303268750020202020202020B9
:101CD0000020520020204D363033200020204D348B
:101CE000313220530046696C616D656E74207275E7
:101CF0006E6F75742073656E736F723A00205500B5
:101D000046696C616D656E74206C6F61642F756ED1
:101D10006C6F6164206C656E677468733A00202094
:101D20004D3230392053004175746F2D52657472F5
:101D30006163743A20533D3020746F20646973618D
:101D4000626C652C203120746F20696E746572702E
:101D500072657420452D6F6E6C79206D6F7665739A
:101D600020617320726574726163742F7265636F92
:101D70007665720020204D32303820530052656362
:101D80006F7665723A20533C6C656E6774683E20CE
:101D9000463C756E6974732F6D3E002057002020FD
:101DA0004D323037205300526574726163743A20AB
:101DB000533C6C656E6774683E20463C756E697472
:101DC000732F6D3E205A3C6C6966743E0020204D96
:101DD000343133205300506F7765722D4C6F73731D
:101DE000205265636F766572793A0020204D33305A
:101DF000312050005049442073657474696E6773D4
:101E00003A0020460020480020204D313435205330
:101E1000004D6174657269616C20686561747570EC
:101E200020706172616D65746572733A002020479D
:101E30003239205334205A0020204732392053337E
:101E400020490020204D3432302053004D65736806
:101E500020426564204C6576656C696E673A0020A7
:101E6000204D323036205800486F6D65206F666611
:101E70007365743A00204A0020204D3230352042EC
:101E800000416476616E6365643A20423C6D696E20
:101E90005F7365676D656E745F74696D655F75739B
:101EA0003E20533C6D696E5F666565647261746562
:101EB0003E20543C6D696E5F74726176656C5F663E
:101EC000656564726174653E204A3C6A756E635F45
:101ED0006465763E0020540020204D32303420507E
:101EE00000416363656C65726174696F6E2028756B
:101EF0006E6974732F7332293A20503C7072696E88
:101F0000745F616363656C3E20523C7265747261FC
:101F100063745F616363656C3E20543C74726176E8
:101F2000656C5F616363656C3E0020204D3230312B
:101F30002058004D6178696D756D20416363656C53
:101F400065726174696F6E2028756E6974732F7382
:101F500032293A0020204D3230332058004D61782C
:101F6000696D756D2066656564726174657320289E
:101F7000756E6974732F73293A00537465707320FA
:101F800070657220756E69743A0020440020204DFF
:101F90003230302053002044697361626C65640AFA
:101FA0000046696C616D656E742073657474696E4A
:101FB00067733A0020204D3134392043203B2055AF
:101FC0006E69747320696E2043656C736975730A5A
:101FD0000020286D6D29002020473231202020204C
:101FE0003B20556E69747320696E206D6D0024F47A
:101FF000D43050C38E20C2A24017828B7011127A47
:10200000910D816CD90AA861E108C7586607615132
:1020100043061E4B5D05C145A7041A411104093D45
:102020009803713931034036DB0265339102D430B5
:102030005402802E1D02632CEE01752AC501B028C2
:10204000A001102781018F2564012B244B01E02280
:102050003401AC211F018D200D01801FFC00841E66
:10206000ED00971DDF00B81CD200E61BC600201B48
:10207000BC00641AB200B219A8000A19A0006A18BC
:102080009900D117910040178B00B51684003116C6
:102090007E00B31579003A157300C7146F00581409
:1020A0006A00EE1366008813630025135E00C712F2
:1020B0005B006C12570015125400C11151007011D1
:1020C0004F0021114B00D61049008D1047004610DB
:1020D000440002104200C00F4000800F3E00420F3B
:1020E0003C00060F3B00CB0E3800930E37005C0E11
:1020F0003500270E3400F30D3200C10D3100900D74
:102100003000600D2E00320D2D00050D2C00D90C75
:102110002B00AE0C2900850C29005C0C2700350C27
:1021200027000E0C2600E80B2400C40B2400A00B93
:1021300023007D0B23005A0B2100390B2100180BC3
:102140002000F80A1F00D90A1E00BB0A1E009D0AC3
:102150001D00800A1D00630A1C00470A1B002C0A90
:102160001B00110A1A00F7091A00DD091900C40939
:102170001900AB091900920917007B0918006309BF
:1021800017004C09160036091600200916000A0926
:102190001500F5081500E0081400CC081400B80874
:1021A0001400A4081400900813007D0812006B08A6
:1021B00013005808120046081200340811002308C2
:1021C00011001208110001081100F0071000E007CB
:1021D0001000D0071000C0071000B0070F00A107C3
:1021E000100091070E0083070F0074070F006507AA
:1021F0000E0057070E0049070E003B070D002E0783
:102200000E0020070D0013070D0006070D00F9064C
:102210000C00ED060D00E0060C00D4060C00C8060C
:102220000C00BC060C00B0060C00A4060B009906BE
:102230000C008D060B0082060B0077060B006C0667
:102240000B0061060A0057060B004C060A00420606
:102250000A0038060A002E060A0024060A001A069A
:102260000A001006090007060A00FD050900F4052A
:102270000900EB050900E2050900D9050900D005B0
:102280000900C7050900BE050900B5050800AD0530
:102290000800A50509009C050800940508008C05A8
:1022A0000800840508007C050800740508006C051A
:1022B0000700650508005D050700560508004E0586
:1022C00007004705070040050800380507003105ED
:1022D00007002A050700230507001C050600160550
:1022E00007000F0507000805060002050700FB04AC
:1022F0000600F5040700EE040600E8040600E20408
:102300000700DB040600D5040600CF040600C9045C
:102310000600C3040600BD040600B7040600B104AD
:102320000500AC040600A6040600A00405009B04FA
:10233000060095040500900406008A040500850443
:102340000500800406007A04050075040500700489
:1023500005006B04050066040500610405005C04CB
:10236000050057040500520405004D04050048040B
:102370000500430405003E0404003A04050035044A
:102380000500300404002C04050027040400230485
:1023900005001E0404001A040400160405001104BC
:1023A00004000D04040009040500040404000004F2
:1023B0000400FC030400F8030400F4030400F00329
:1023C0000400EC030400E8030400E4030400E00359
:1023D0000400DC030400D8030400D4030400D00389
:1023E0000400CC030400C8030300C503030024F465
:1023F00004D9201BC40C5C0E9804C4095F02650755
:102400007101F405F900FB04B30048048700C1031F
:1024100069005803550003034500BE023A008402D8
:10242000310053022A002902250004022000E401A1
:102430001C00C8011900AF011700980114008401A5
:102440001300710110006101100051010E004301E1
:102450000D0036010B002B010B0020010B001501B4
:1024600009000C01090003010800FB000800F3004B
:102470000800EB000700E4000600DE000600D800BC
:102480000600D2000600CC000500C7000500C2000F
:102490000500BD000400B9000400B5000400B1004F
:1024A0000400AD000400A9000400A5000300A20080
:1024B00003009F0004009B000300980003009500A8
:1024C000020093000300900003008D0002008B00C7
:1024D00003008800020086000200840003008100DF
:1024E00002007F0002007D0002007B0002007900F4
:1024F0000200770001007600020074000200720002
:102500000100710002006F0002006D0001006C000C
:1025100002006A0001006900020067000100660015
:10252000010065000100640002006200010061001A
:102530000100600001005F0002005D0001005C001E
:1025400001005B0001005A00010059000100580021
:102550000100570001005600010055000100540021
:10256000010053000000530001005200010051001F
:102570000100500001004F0001004E0000004E001D
:1025800001004D0001004C0001004B0000004B0019
:1025900001004A0001004900010048000000480015
:1025A0000100470001004600000046000100450010
:1025B000000045000100440001004300000043000A
:1025C0000100420000004200010041000000410003
:1025D0000100400001003F0000003F0001003E00FC
:1025E00000003E0001003D0000003D0001003C00F5
:1025F00000003C0000003C0001003B0000003B00EC
:1026000001003A0000003A000100390000003900E2
:1026100001003800000038000000380001003700D9
:1026200000003700010036000000360000003600D0
:1026300001003500000035000000350001003400C5
:1026400000003400000034000100330000003300BB
:1026500000003300010032000000320000003200B0
:1026600001003100000031000000310001003000A5
:10267000000030000000300001002F0000002F009B
:1026800000002F0000002F0001002E0000002E008F
:1026900000002E0001002D0000002D0000002D0084
:1026A00000002D0001002C0000002C0000002C0078
:1026B00000002C0001002B0000002B0000002B006C
:1026C00000002B0001002A0000002A0000002A0060
:1026D00000002A0001002900000029000000290054
:1026E0000000290000002900010028000000280047
:1026F000000028000000280000002800010027003A
:10270000000027000000270000002700000027002D
:102710000100260000002600000026000000260020
:102720000000260001002500000025000000250013
:102730000000250000002500000025000100240005
:1027400000002400000024000000240000002400F9
:1027500001002300000023000000230000002300EC
:1027600000002300000023000000230001002200DD
:1027700000002200000022000000220000002200D1
:1027800000002200010021000000210000002100C3
:1027900000002100000021000000210000002100B5
:1027A00001002000000020000000200000002000A8
:1027B0000000200000002000000020000000200099
:1027C00001001F0000001F0000001F0000001F008C
:1027D00000001F0000001F0000001F0001001E007D
:1027E00000001E0000001E0000001E000000043754
:1027F00000001E290000511B0000581000001009A5
:102800000000CC04000078020000410100006F705D
:10281000656E00545249474745524544007A5F6D02
:10282000696E00795F6D696E00785F6D696E005248
:1028300065706F7274696E6720656E6473746F7013
:10284000207374617475730A004563686563206F53
:10285000726967696E65005761726E696E673A20CA
:10286000486F6D696E672042756D702044697669A6
:10287000736F72203C20310A00000048420000487B
:1028800042000080400202040000A0400000A0407E
:1028900000000040FFFFFF020000000000000000F9
:1028A0000000000000000000000000000000000028
:1028B0000000000000000000000000000000000018
:1028C0000000000000000000000000000000000008
:1028D00000000000000000000000000000000000F8
:1028E00000000000000000000000000000000000E8
:1028F00000000000000000000000000000000000D8
:1029000000000000000000000000000000000000C7
:1029100000000000000000000000000000000000B7
:1029200000000000000000000000000000000000A7
:10293000000000000000000001FFFE001E7807E01C
:10294000003E00F3C003C00007FFFE00FE7F07E06B
:10295000003E07F3F803C0000FFFFE01FE7F03F007
:10296000007E0FF3FC03C0001FFFFE03FE7F83F019
:10297000007E1FF3FE03C0001FFFFE07FE7FC1F8AD
:1029800000FC3FF3FF03C0003F80000FE007E1F8C9
:1029900000FC7F003F83C0003F00000FE007E0FC29
:1029A00001F87F003F83C0003F00000FC003E0FC40
:1029B00001F87E001F83C0003F00000FC003E07CD1
:1029C00001F07E001F83C0003F80001F8001F07E69
:1029D00003F0FC000FC3C0003FE0001F8001F07E49
:1029E00003F0FC000FC3C0001FFFF81F8001F03E82
:1029F00003E0FC000FC3C00007FFFE1F8001F01FB3
:102A000007C0FC000FC3C00003FFFF1F8001F01FC1
:102A10008FC0FC000FC3C00000007F9F8001F01F2B
:102A20008FC0FC000FC3C00000003F9F8001F00F6B
:102A30008F80FC000FC3C00000001F9FC003F00F79
:102A4000DF80FE001FC3C00000001F8FC003E0072F
:102A5000DF007E001F83C00000001F8FE007E0073B
:102A6000FF007F003F83E00000003F8FE007E003AE
:102A7000FE007F003F83E0001FFFFF07FE7FC003D3
:102A8000FE003FF3FF03FFFC1FFFFF03FE7F8003F9
:102A9000FE001FF3FE03FFFC1FFFFE01FE7F00018F
:102AA000FC000FF3FC01FFFC1FFFFC00FE7F000198
:102AB000FC0007F3F800FFFC1FFFF0001E78000089
:102AC000F80000F3C0003FFC000000000000000020
:102AD00000000000000000000000000000000000F6
:102AE00000000000000000000000000000000000E6
:102AF000000000000000000000000000101000A313
:102B000040010800000000000000000010100084D8
:102B100000010800000000000000000018300084E0
:102B200000010800000000000000000014538FA7FF
:102B3000471F0F910000000000000000145450A433
:102B400048A108510000000000000000129450A4A9
:102B50004FA108510000000000000000111450A413
:102B6000482108510000000000000000111450A48A
:102B700048A1084A000000000000000010138FA4C4
:102B8000471F0F840000000000000000000000004C
:102B9000000000080000000000000000000000002D
:102BA0000000001000000000000000000000000015
:102BB0000000000000000000000000000000000015
:102BC000000000000000000000000210000003E010
:102BD00000000000000000000000022000000410BF
:102BE000000000100000000000000240000004008F
:102BF000000000100000000000000381CB8F840360
:102C00009EE7C859CE700000000002822C50840458
:102C1000511428522888000000000243E850840420
:102C200051142853E8600000000002220850840478
:102C30005114285208100000000002122851841478
:102C4000511428D22888000000000209C84E83E3EE
:102C50009117C749C8700000000000000000800004
:102C6000000400000000000000000000001F000041
:102C70000004000000000000000000000000000050
:102C80000000000000000000000000000000000044
:102C9000000000000000000001FFFFFFFFFFFFFF3A
:102CA000FFFFFFFFFFFF0FFFFFFFFFFFFFFFFFFF24
:102CB000FFFFFFFF1E0000000000000000000007F3
:102CC000FFFF380000000000000000000003FFFFCD
:102CD000700000000000000000000001FFFF600025
:102CE00000000000000000000000FFFF6000000086
:102CF00000000000000000007FFFC0000000000096
:102D00000000007800003FFFC00FC0FC0000000082
:102D1000007818001FFFC03FE1FF000000000078AE
:102D20003C000FFFC07FF3FF8000000000783C00F4
:102D300007FFC0FFFFFFC000000000783C0003FF5A
:102D4000C1F87F87E00000000078000001FFC1F0BB
:102D50003F03E00000000078000000FFC1E01E011A
:102D6000E01F0003E0783C03F07FC1E01E01E07F3C
:102D7000C00FF8783C07FC3FC1E01E01E1FFE01FF7
:102D8000FC783C0FFE1FC1E01E01E3FFF03FFE7820
:102D90003C1FFE0FC1E01E01E3F3F83F3E783C3FCD
:102DA0003F07C1E01E01E7E0FC7C1F783C3E1F07A7
:102DB000C1E01E01E7C07C7C0F783C3C0F03C1E002
:102DC0001E01E7807C780F783C3C0F03C1E01E01B8
:102DD000E7803C7800783C3C0F03C1E01E01E780AF
:102DE0003C7800783C3C0F03C1E01E01E7803C7852
:102DF00000783C3C0F03C1E01E01E7C03C7800783E
:102E00003C3C0F03C1E01E01E3E03C78007C3C3C0D
:102E10000F03C1E01E01E3FF3FF8007FBC3C0F033E
:102E2000C1E01E01E1FF3FF8003FBFFC0F03C1E01E
:102E30001E01E0FF3FF8001FBFFC0F03C1E01E01B1
:102E4000E07F3FF8000FBFFC0F03600000000000B0
:102E5000000000000000000760000000000000000B
:102E600000000000000670000000000000000000EC
:102E70000000000E3800000000000000000000000C
:102E8000001C1E0000000000000000000000007890
:102E90000FFFFFFFFFFFFFFFFFFFFFFFFFF001FF3F
:102EA000FFFFFFFFFFFFFFFFFFFFFF8070012C010F
:102EB00090012701B0012201C0011D01F00118019C
:102EC0001002130130020E01600209019002040198
:102ED000C002FF000003FA004003F5008003F00089
:102EE000D003EB002004E6007004E100E004DC0005
:102EF0004005D700C005D2004006CD00D006C8006E
:102F00008007C3003008BE00F008B900C009B40053
:102F1000B00AAF00B00BAA00D00CA500000EA000B4
:102F2000500F9B00C01096005012910000148C00AE
:102F3000C0158700B0178200B0197D00D01B780043
:102F4000001E730040206E0090226900F02464008F
:102F500040275F0090295A00E02B5500102E5000AA
:102F600020304B0010324600E033410090353C00E9
:102F70001037370070383200A0392D00B03A2800E1
:102F8000A03B2300603C1E00103D1900903D140042
:102F9000103E0F00703E0A00C03E0500003F0000DA
:102FA000403FFBFF803FF6FFC03FF1FF6874747045
:102FB000733A2F2F6D61726C696E66772E6F726730
:102FC00000322E302E362E31002020506C616E6E75
:102FD000657242756666657242797465733A20005F
:102FE0002046726565204D656D6F72793A20004309
:102FF0006F6D70696C65643A2053657020323520BE
:10300000323032300A00204C617374205570646194
:103010007465643A20323032302D30382D32382009
:103020007C20417574686F723A20284B656E67206A
:10303000436F6D7075746572732C20574B290A00AD
:10304000322E302E362E310A004D61726C696E00C0
:1030500020536F6674776172652052657365740AD8
:1030600000205761746368646F67205265736574EC
:103070000A002042726F776E206F7574205265735C
:1030800065740A002045787465726E616C20526523
:103090007365740A00506F77657255700A00617528
:1030A000746F25632E67004732385859004D313010
:1030B0003031006572726F722077726974696E6761
:1030C00020746F2066696C650A00446F6E6520731A
:1030D0006176696E672066696C652E0A004D32392B
:1030E00000427574C3A9657300255320256320250C
:1030F0006320256320256300656E6473746F7073AD
:10310000206869743A200054656D70C3A9726174B7
:10311000757265005669742E202076656E74696C30
:103120002E20200042757365004C6974205A004DB2
:10313000656E75207072696E636970616C005072A3
:10314000C3A963682E20242062757365005072C382
:10315000A963682E2024206C697400526566726F22
:1031600069646972004261627973746570205A0003
:10317000466C7578005669746573736500205369F1
:103180007A653A200043616E6E6F74206F70656ED1
:10319000207375626469722000534420496E69741B
:1031A000204661696C0053442063617264206F6B38
:1031B0000A006F70656E526F6F74206661696C658E
:1031C000640A00766F6C756D652E696E6974206691
:1031D00061696C65640A004E6F205344206361721C
:1031E000640A004D3234004D3233202573004669A5
:1031F0006C652073656C65637465640A0046696C70
:1032000065206F70656E65643A2000454E4420531A
:103210005542524F5554494E450A002220706F7353
:10322000002220706172656E743A2200535542523A
:103230004F5554494E452043414C4C2074617267B0
:1032400065743A220053756263616C6C204F766539
:1032500072666C6F77004578636565646564206DA0
:10326000617820535542524F5554494E452064656C
:103270007074683A310A0044656C6574696F6E2039
:103280006661696C65642C2046696C653A2000466D
:10329000696C652064656C657465643A0057726991
:1032A00074696E6720746F2066696C653A200066E9
:1032B0007265736800646F696E67004E6F772000F7
:1032C0004275736520656E20636861756666652E5C
:1032D0002E2E004732363A20436861756666616774
:1032E00065206475206C69740057616974696E6744
:1032F00020666F72206865617475702E0A00416DDA
:103300006F726365206C6F6E677565757220666994
:10331000786500416D6F726365207465726D696ECA
:10332000C3A96500416D6F726365206D616E75653F
:103330006C6C652E2E2E00536F72746965204732B7
:1033400036003F53706563696669656420582C597F
:1033500020636F6F7264696E617465206F7574208D
:103360006F6620626F756E64732E0A003F285229C3
:1033700065706561742076616C7565206E6F742070
:10338000706C61757369626C653B206D7573742038
:103390006265206174206C6561737420312E0A00AF
:1033A0003F537065636966696564206E6F7A7A6CF5
:1033B000652074656D7065726174757265206E6FDD
:1033C0007420706C61757369626C652E0A003F53DE
:1033D00070656369666965642066696C616D656EB8
:1033E000742073697A65206E6F7420706C617573D8
:1033F00069626C652E0A003F537065636966696592
:1034000064207072696D65206C656E677468206EEB
:103410006F7420706C61757369626C652E0A003F71
:10342000537065636966696564206E6F7A7A6C654E
:103430002073697A65206E6F7420706C6175736992
:10344000626C652E0A003F52657472616374696F25
:103450006E204D756C7469706C696572206D757342
:1034600074206265207370656369666965642E0AFD
:10347000003F5370656369666965642052657472C4
:10348000616374696F6E204D756C7469706C6965E9
:1034900072206E6F7420706C61757369626C652E3A
:1034A0000A003F537065636966696564206C6179E1
:1034B000657220686569676874206E6F7420706C2F
:1034C00061757369626C652E0A0043292E0A003FFC
:1034D000537065636966696564206265642074651C
:1034E0006D7065726174757265206E6F7420706C9A
:1034F00061757369626C65202834302D004732365F
:10350000207374617274696E672E2E2E0A00207407
:103510006F6F206C6F6E6720657874727573696F5A
:103520006E2070726576656E7465640A0020636F44
:103530006C6420657874727573696F6E2070726543
:1035400076656E7465640A00DB0FC93F45BCDA3FDF
:103550008FB30240FCF0274056946140FE4B9B40E5
:1035600084A5D840E0231841346A5641E859974170
:1035700064DBD5416E271742B4B75542CE1A974245
:10358000C8AED542B5885A43D40684BFA65FA7BF4C
:103590007443E0BF10B11AC01C2C58C0E8F697C0A5
:1035A000B849D6C04E4E17C124D355C1802497C107
:1035B000A0B5D5C1121A17C244AE55C2781797C22A
:1035C0006CACD5C267885AC37C3C3E5E2B3D3F2F16
:1035D0005B5D3B2C2A225C00496E76616C6964203D
:1035E00065787472756465720A004572722054457C
:1035F0004D502E204D4158004D415854454D5020BE
:10360000747269676765726564004572722054451B
:103610004D502E204D494E004D494E54454D5020A1
:1036200074726967676572656400202F00204240EC
:103630003A0020403A0020573A003F00496E697432
:1036400069616C6973657220454550524F4D004960
:103650006D70722E20616E6E756CC3A965004D325F
:1036600035004D69736520656E2070617573652E38
:103670002E2E00454550524F4D2056657273696F8E
:103680006E204572726F7200454550524F4D204971
:103690006E646578204572726F7200454550524FD6
:1036A0004D20435243204572726F720049676E6F1E
:1036B0007265720052657365740043686172676574
:1036C0007220636F6E6669672E00456E726567696A
:1036D000737472657220636F6E6669672E00436F44
:1036E0006E6669672E206176616E63C3A9650041CD
:1036F0007272C3AA74004D617263686500444543E9
:103700004841524745522046494C004348414E47A4
:1037100045522046494C414D454E54005265737404
:1037200061757265722064C3A96661757473005215
:10373000C3A9676C6572207072C3A963682E2024C8
:1037400000436170746575722066696C2E0052C307
:10375000A974726163746174696F6E004D373032A1
:1037600020542564004D36303020423020542564EA
:10377000004D373032203B2564004D373031205426
:103780002564004D373032004D373031004D363032
:10379000302042300050757267657220656E636F2D
:1037A0007265004F5054494F4E5320524550524974
:1037B00053453A00494D50522E2050415553450033
:1037C0002020427573653A20005061726B696E6704
:1037D0002E2E2E000000417474656E74652066699B
:1037E0006C616D656E7400706F75722064C3A96D35
:1037F00061727265720000417474656E7465007266
:103800006574726169742064752066696C616D65A8
:103810006E7400004275736520656E206368617583
:103820006666650050617469656E746572205356F2
:10383000502E2E2E0000486F74656E6420746F6FDA
:1038400020636F6C640A004D3630303A2054726F3A
:10385000702066726F6964005072657373206275C0
:1038600074746F6E20746F2068656174206E6F7A57
:103870007A6C650A004D32342053256C642054253F
:103880006C64004739322E392045257300473120BA
:10389000462564004739322E39205A2573004731B6
:1038A000205A3020463230300047312058257320CE
:1038B000592573204633303030004D343230205398
:1038C0002569205A2573004D313036205025692056
:1038D000532569004D31303920532569004D313968
:1038E0003020532569004D32303020442573004785
:1038F000323852305859004739322E39204530205D
:103900005A300A47315A2573004D34323020533033
:10391000205A300020496E76616C696420657874A5
:103920007275646572200000000000000000000055
:103930000000000000914300007A4300009B4343D5
:103940006F6E6669672E20656E7265676973747243
:10395000C3A9650053657474696E67732053746FEF
:10396000726564202800526564C3A96D6172726536
:10397000722053565000494D50522E2053544F50F0
:1039800050C389450025533A202553004B494C4CE0
:103990004544005072696E7465722068616C74658C
:1039A000642E206B696C6C28292063616C6C6564E3
:1039B000210A006563686F3A004572726F723A00BF
:1039C0000A4D6561737572656420706F696E7473FA
:1039D0003A0A00337833206D6573682E205A206FC1
:1039E00066667365743A200047323620616E6E75E4
:1039F0006CC3A90044C3A9706C61636572205A004E
:103A000041425300504C410044C3A9706C6163654E
:103A1000722025736D6D0044C3A9706C616365727B
:103A200020302E316D6D0044C3A9706C61636572E6
:103A300020316D6D0044C3A9706C616365722031E3
:103A4000306D6D0044C3A9706C6163657220756E42
:103A50002061786500427573652074726F7020660E
:103A6000726F69646500457874727564657572007B
:103A700044C3A9706C6163657220590044C3A97086
:103A80006C616365722058004368616E67657220DF
:103A900066696C616D656E740052657472616974FB
:103AA0002066696C616D656E74004368617267655C
:103AB000722066696C616D656E74005072C3A96393
:103AC000686175662E20706572736F005072C3A9AD
:103AD0006368617566666167652024005265746F6E
:103AE00075720000002100240027002A002D0030FC
:103AF00000330001010000040107010A0100002257
:103B000000250028002B002E0031003400020100A7
:103B100000050108010B01000020002300260029F8
:103B2000002C002F003200000100000301060109F3
:103B30000105050505070508080808020202020A32
:103B40000A08080404040401010101010101010340
:103B500003030303030303040707070C0C0C0C0CFB
:103B60000C0C0C0202020206060606060606060BEE
:103B70000B0B0B0B0B0B0B01021020200808102065
:103B800040102040800201020108040201010204E9
:103B900008102040808040201008040201800402A8
:103BA00001804020100804020108040201010204FF
:103BB0000810204080010204081020408000000A04
:103BC0000B02090C0D0E08070304010000000000A1
:103BD00000000000000000000000000000000000E5
:103BE00000000000000000000012111000000000A2
:103BF00000000000000000000000000000000000C5
:103C0000000000043A003A416E6E756C6572004D1A
:103C10006F7576656D656E74004D38340052C3A9BA
:103C2000676C6572204E69762E206C69740044C3FF
:103C3000A96D617272657220696D707265737369C6
:103C40006F6E00496D7072696D65720043616E6ED2
:103C50006F7420656E746572207375626469723A60
:103C60002000022E2E00417272C3AA746572206D6C
:103C70006F7465757273004F726967696E65206154
:103C800075746F0047323800496D707265737369DF
:103C90006F6E20534400496D70722E20656E207047
:103CA00061757365004F726967696E6520257325BC
:103CB000732573205072656D69657200496E736576
:103CC00072742066696C616D656E7420616E64202B
:103CD000707265737320627574746F6E0A00534F4F
:103CE000564F4C2053563031207072C3AA74652E43
:103CF00000496D7072657373696F6E00220A00551A
:103D00006E6B6E6F776E20636F6D6D616E643A20BF
:103D100022006F70656E206661696C65642C2046B8
:103D2000696C653A200020453A00205A3A00205933
:103D30003A0045207061732F6D6D005A20706173D9
:103D40002F6D6D0059207061732F6D6D00582070BC
:103D500061732F6D6D00496E69742E004D343238D9
:103D60000046696C616D656E74005061732F6D6DF6
:103D70000044C3A9766961742E206A6F6E63742E45
:103D800000416363C3A96CC3A9726174696F6E005B
:103D900056C3A96C6F636974C3A90052C3A9676C49
:103DA0002E2064C3A963616C206F726967696E65B8
:103DB00000436F696E2073756976616E7400546597
:103DC000726D696EC3A90053756976616E740020C7
:103DD00062797465733B2063726320004E6F2045E7
:103DE0004550524F4D2E0A00454550524F4D2064CC
:103DF00061746173697A65206572726F722E0A0050
:103E00002073746F7265642073657474696E677370
:103E100020726574726965766564202800202863C5
:103E2000616C63756C6174656429210A0020213D11
:103E30002000454550524F4D20435243206D697339
:103E40006D61746368202D202873746F7265642916
:103E50002000496E6465783A2000204D61726C69DB
:103E60006E3D563831290A00454550524F4D207657
:103E7000657273696F6E206D69736D61746368201C
:103E800028454550524F4D3D0048617264636F6450
:103E900065642044656661756C742053657474694B
:103EA0006E6773204C6F616465640A003B200000FC
:103EB00000FA430000FA430000A0400000C841009F
:103EC00000A0420000A0420000C8430080CF43F49D
:103ED000010000F401000064000000E8030000435A
:103EE00061703A004348414D4245525F54454D5040
:103EF0004552415455524500424142595354455050
:103F000050494E470041524353004D4F54494F4E84
:103F10005F4D4F44455300544845524D414C5F500E
:103F2000524F54454354494F4E004C4F4E475F4605
:103F3000494C454E414D45004155544F5245504F17
:103F400052545F53445F53544154555300534443B8
:103F50004152440050524F4D50545F535550504FB2
:103F6000525400454D455247454E43595F504152CA
:103F700053455200434153455F4C494748545F42C3
:103F800052494748544E45535300544F47474C45B8
:103F90005F4C494748545300534F4654574152458C
:103FA0005F504F574552004255494C445F5045526F
:103FB00043454E54004C4556454C494E475F44419D
:103FC0005441005A5F50524F42450052554E4F5592
:103FD00054004155544F4C4556454C005052494EA3
:103FE000545F4A4F420050524F475245535300418D
:103FF00055544F5245504F52545F54454D50005602
:104000004F4C554D45545249430042494E41525937
:104010005F46494C455F5452414E5346455200530A
:10402000455249414C5F584F4E5F584F46460046F7
:1040300049524D574152455F4E414D453A4D61728F
:104040006C696E20322E302E362E3120285365704A
:1040500020323520323032302031353A35383A345A
:10406000392920534F555243455F434F44455F55CF
:10407000524C3A68747470733A2F2F67697468757C
:10408000622E636F6D2F4D61726C696E4669726D41
:10409000776172652F4D61726C696E2050524F547A
:1040A0004F434F4C5F56455253494F4E3A312E3095
:1040B000204D414348494E455F545950453A534F6E
:1040C000564F4C2053563031204558545255444594
:1040D000525F434F554E543A3120555549443A6347
:1040E000656465326132662D343161322D34373486
:1040F000382D396231322D633535633632663336C9
:104100003766660A00656E7175657565696E67204C
:1041100022006F6B00526573656E643A20004F4653
:10412000460A004661646520486569676874200036
:104130004661696C656420746F20656E61626C65B0
:1041400020426564204C6576656C696E670A004D97
:1041500065736820426564204C6576656C206461F7
:1041600074613A0A00496E76616C6964206D65730A
:10417000682E0A00206E6F7420656E746572656427
:104180002E0A00206F6620004D424C204732392015
:10419000706F696E7420004A206F7574206F6620FE
:1041A00072616E67652028302D0049206F7574207C
:1041B0006F662072616E67652028302D004D657333
:1041C000682070726F62696E6720646F6E652E0A78
:1041D000005374617274206D6573682070726F6231
:1041E000696E67207769746820224732392053311D
:1041F000222066697273742E0A004732380A4732E9
:104200003920533200686173206E6F2064617461DD
:104210002E0A004D65736820426564204C65766502
:104220006C696E67200053206F7574206F66207272
:10423000616E67652028302D35292E0A004D3432F5
:104240003120696E636F7272656374207061726190
:104250006D657465722075736167650A00204D395C
:104260003220580020204D61783A200020204D69EE
:104270006E3A2000536F667420656E6473746F70BD
:10428000733A20004C69740020436F756E74205897
:104290003A00453100626564002C207379737465BF
:1042A0006D2073746F70706564212048656174655A
:1042B000725F49443A200045727220646520636849
:1042C00061756666650048656174696E6720666140
:1042D000696C656400202D20496E76616C696420EC
:1042E0006578747275646572206E756D6265722092
:1042F000210A0045727220544845524D4951554596
:1043000000546865726D616C2052756E61776179D9
:1043100000000A01140211241FBECFEFD1E2DEBF5C
:10432000CDBF00E00CBF12E0A0E0B2E0E4EAF5E9A6
:1043300002E00BBF02C007900D92AC3EB107D9F767
:1043400026E1ACEEB2E001C01D92A731B207E1F761
:1043500011E2CAE8D1E200E006C021970109802FEE
:10436000FE010F941147C938D10780E00807A9F76B
:104370000F9445320D94C04A0C9400002F923F9246
:104380004F925F926F927F928F929F92AF92BF9265
:10439000CF92DF92EF92FF920F931F93CF93DF9311
:1043A000CDB7DEB7AD970FB6F894DEBF0FBECDBF69
:1043B0008DA72091E80D2CA781E08093E80D8091D6
:1043C00027158D3409F4BEC2843511F40C943D32A6
:1043D000873411F00C944F32809125159091261559
:1043E0008531910511F40C945132B4F48430910567
:1043F0003CF4823091050CF05CC097FF31C09EC246
:104400008A30910509F429C18B30910509F42AC13C
:10441000049709F093C2E2C08D31910509F451C1AE
:104420006CF48B31910509F422C10CF03AC14A9722
:1044300009F084C20E94619D0C9451328A35910525
:1044400009F443C124F48A9709F4F9C177C28B3582
:10445000910509F43EC18C35910509F43FC16EC246
:104460008091A106813011F00C9451320E94FDDD43
:1044700080910D04882311F40C948C3285E40E9401
:1044800072F0882311F40C948C3288E50E9472F04B
:1044900081110C948C3289E50E9472F081110C9488
:1044A0008C328AE50E9472F081110C948C320C944B
:1044B0005A322091A106213011F00C94513211E0B2
:1044C000029709F010E00E94FDDD19821A821B821A
:1044D0001C821D821E821F82188682E50E94BBF00C
:1044E000882309F44BC00E943BF06B017C0120E063
:1044F00030E0A9010F941640882309F455C080913B
:10450000511190915211A0915311B091541188A35F
:1045100099A3AAA3BBA38091551190915611A09184
:104520005711B09158118CA39DA3AEA3BFA3809047
:10453000D60D9090D70DA090D80DB090D90D409089
:10454000DA0D5090DB0D6090DC0D7090DD0DA50153
:10455000940168A179A18AA19BA10F9416408111B1
:104560000C94B732A30192016CA17DA18EA19FA1F1
:104570000F9416408823C1F00C94B73289E40E944E
:10458000BBF0882331F00E943BF069837A838B83F0
:104590009C838AE40E94BBF0882331F00E943BF0A8
:1045A0006D837E838F83988720E030E0A901698145
:1045B0007A818B819C810F94164081110C946B330E
:1045C00020E030E0A9016D817E818F8198850F9474
:1045D000164081110C946B330C947E3380E50E945D
:1045E000BBF0882329F00F94D1246B017C0103C018
:1045F000C12CD12C760183E50E94BBF0882361F0A9
:104600000E943BF020E030E04AE754E40F947C4005
:104610000F949F486B017C010E94B0EC8091E20CEA
:10462000811105C060E089E996E00E944ED60E94A3
:104630007BFAC60ED71EE81EF91E0E947BFADC012B
:10464000CB018C199D09AE09BF09B7FD02C00C94BE
:10465000513280E00E945339F0CF81E00E948AF10C
:104660000C94513280E00E948AF10C9451320F94E4
:10467000790781110C9451328CE0E3E7F2E0DE011E
:10468000119601900D928A95E1F760E070E080E567
:104690000E94B2E5BE016F5F7F4F0E94A0D10C94D3
:1046A00051328091AE048770873011F00C948533BD
:1046B00060E08FE40E94D7F081110C9451320C9489
:1046C00085330F94C4250C94513210923C0E0C94F7
:1046D00051328FE080933C0E0C945132809124151E
:1046E000882349F1893009F0A6C00FE7A02E02E027
:1046F000B02E81E5E82E81E1F82ED12C00E010E00B
:10470000D5018D915D010E94BBF0882369F00E9464
:104710003BF0F7016083718382839383133011F43C
:1047200001E002C0DD24D3941F5FF4E0EF0EF11C22
:10473000143031F775C0AFE72A2EA2E03A2EB2E569
:10474000EB2EBEE0FB2E21E531E139A328A311E6D3
:10475000C12E11E1D12E00E010E0D1018D911D019B
:104760000E94BBF0882309F44BC00E943BF02B0150
:104770003C01133049F0F60120813181428153819F
:104780000F942B472B013C01A8A1B9A12D913D917C
:104790004D915C91C301B2010F942B474B015C0119
:1047A0002DEB37E346E855EB0F948C4987FD0AC0A3
:1047B0002DEB37E346E855E3C501B4010F941640ED
:1047C0001816F4F4133051F440925D1150925E11BA
:1047D00060925F117092601101E012C0A501940116
:1047E000F70160817181828193810F942C47D701F9
:1047F0006D937D938D939C931397812F0E94678572
:104800001F5FB4E0EB0EF11CE8A1F9A13496F9A307
:10481000E8A3F4E0CF0ED11C143009F09ECF05C000
:10482000DD2019F00E94868A06C0002321F08DE564
:1048300091E10E94C1EC0E94888A0C9451328091CF
:10484000A106813011F00C94513289E40E94BBF032
:10485000F82E882321F00E9437F0182F01C010E0B5
:104860008AE40E94BBF0082F882319F00E9437F0D9
:1048700001C080E0FF2011F0133020F4002341F04C
:10488000833030F082EA96E00E942CF40C9451328E
:1048900090E1E1E5F1E1A6EDBDE001900D929A9580
:1048A000E1F7FF2091F024E01202F0011124EB5D0A
:1048B000FD4E40815181628173814093D60D5093AA
:1048C000D70D6093D80D7093D90D002391F034E08B
:1048D0008302F0011124E75EFD4E80819181A28167
:1048E000B3818093DA0D9093DB0DA093DC0DB09330
:1048F000DD0D40E050E0BA0186E40E94FF556B01F7
:104900007C0120E030E0A9010F948C4918164CF48A
:1049100020E030E040E752E4C701B6010F9426489A
:1049200003C060E070E0CB0169837A838B839C8352
:10493000CE0101960E94F8880C9451320F94BD0567
:104940000C94513280912515909126158737910549
:1049500009F455C70CF0F3C08C34910509F40EC46A
:104960000CF069C08931910509F4EAC254F582312D
:10497000910509F44FC65CF48031910509F43AC2FF
:104980000CF04DC2029708F4FDC10C943A32863106
:10499000910509F479C264F48431910509F453C294
:1049A000459711F00C943A320E94D6970C945132EC
:1049B0008731910509F472C2489709F486C20C94B4
:1049C0003A328F31910509F48DC3BCF48C319105D5
:1049D00009F440C34CF48A31910509F4C5C24B97E0
:1049E00009F4D0C20C943A328D31910509F43AC3DE
:1049F0004E9709F43EC30C943A328A32910509F479
:104A000091C364F48032910509F443C3819711F096
:104A10000C943A320E94E65A0C9451328934910532
:104A200009F499C38B34910511F00C943A320E9429
:104A300047EA0C9451328A36910509F49EC4ACF5CC
:104A40008335910509F4DFC5BCF48E34910509F472
:104A50009DC30CF497C38135910509F4C0C5823517
:104A6000910511F00C943A3280913C0E8F7D80615B
:104A700080933C0E0C9451328C35910509F4F0C5AD
:104A800054F48435910509F4C5C58535910509F4BB
:104A9000C4C50C943A328836910509F409C48936A4
:104AA000910509F456C40C943A328037910509F403
:104AB00002C5F4F48D36910509F421C47CF48B36DB
:104AC000910509F497C48C36910511F00C943A3293
:104AD0001092E70D109223020C9451328E369105FC
:104AE00009F492C48F36910509F4A1C40C943A32AA
:104AF0008337910509F43EC68CF48137910509F49A
:104B0000E7C48237910511F00C943A320F94AC0A45
:104B100089EA91E10F94012E0C9451328537910569
:104B200009F42BC68637910511F00C943A320091A6
:104B3000B9031091BA0394E0F12C40E044C68E32E0
:104B4000A1E09A0711F40C94D52F0CF076C08D3C9F
:104B5000910509F49AC774F58B39910509F419C5C3
:104B600084F48937910509F455C60CF44BC68C388A
:104B7000910509F4CFC48139910509F452C60C940A
:104B80003A32893C910509F407C754F48E3B9105EC
:104B900009F4DFC4883C910509F4B7C60C943A3295
:104BA0008B3C910509F41EC78C3C910509F439C76B
:104BB0000C943A328C3D910511F40C94122EECF4C5
:104BC000803D910509F4D7C754F48E3C910509F452
:104BD0006FC78F3C910509F48AC70C943A32813D26
:104BE000910511F40C94052E833D910511F00C9460
:104BF0003A320F9447230C9451328232E1E09E07FF
:104C000011F40C94DB2E64F48D3D910511F40C9499
:104C1000392E823E910511F40C948F2E0C943A3269
:104C20008C3221E0920711F40C94412F8D32914087
:104C300011F40C94562F0C943A32863FA1E09A0757
:104C400011F40C948F300CF048C08D39E1E09E07D0
:104C500011F40C94FF31E4F4803921E0920711F44F
:104C60000C9419304CF48F32914011F00C943A327C
:104C70000E9416560C9451328A39B1E09B0709F410
:104C800023C48C39914011F40C941C300C943A32AA
:104C90008C3AF1E09F0711F40C942F307CF4843AA5
:104CA00031E0930711F40C942C30853A914011F0C7
:104CB0000C943A320F94E1240C945132843FB1E0C9
:104CC0009B0711F40C948C30853F914011F00C94AB
:104CD0003A320F94511B0C9451328D3BF2E09F07F6
:104CE00011F40C9430310CF58C3032E0930711F450
:104CF0000C94AC306CF4873FB1E09B0711F40C943A
:104D00009230883F914011F40C949B300C943A32CD
:104D10008835F2E09F0711F40C94B4308B35924043
:104D200011F40C94B7300C943A32873E33E0930779
:104D300011F40C94F131CCF48E3BB2E09B0711F4EA
:104D40000C943331803A934011F00C943A32209114
:104D5000B9033091BA0390913C12926090933C1247
:104D6000C9010E94E1990C945132883EF3E09F07FB
:104D700011F40C941632893E934011F40C941932BC
:104D80000C943A3280E50E94BBF0882329F00F94FE
:104D9000D1246B017C0103C0C12CD12C760183E5A9
:104DA0000E94BBF0882361F00E943BF020E030E0DD
:104DB0004AE754E40F947C400F949F486B017C01B8
:104DC0000E94B0EC8091B9039091BA03009721F052
:104DD00061E00E94E2D605C060E08BEB96E00E94A5
:104DE0004ED640E0C701B6010E94363F0F94CB0576
:104DF0000C94513263E478E18091B9039091BA0345
:104E00000F94543F892B11F40C94513240E060E030
:104E100070E08BEC96E00E94A1F50C9451328091E9
:104E2000201584FF02C00C9425348091221587FF41
:104E300002C00C94253480912315837011F00C94DA
:104E400025340C94413481E097E00E942CF489E5EC
:104E500092E10E94F3C48BE1E9E5F2E1DE011196F3
:104E600001900D928A95E1F760E070E0CE01019625
:104E70000E94119BCE0101960E940EF182EF96E0F6
:104E80000E942CF40C9451320E94179780913C128E
:104E9000877F806280933C120C945132E091B90379
:104EA000F091BA038081882329F0803209F41082BE
:104EB0003196F8CF60E08091B9039091BA030E94D7
:104EC0002F9A1092C1030C94513283E50E94BBF0DB
:104ED000882321F00E9403F00E94B65B84E50E94C3
:104EE000BBF08823A9F00E9403F06B017C010E94B3
:104EF000728BC0927C0DD0927D0DE0927E0DF0926F
:104F00007F0DCD28CE28CF2819F081E08093380E70
:104F10000E946F37882381F00E9428970E9447EAF9
:104F200081EB9EE00E94CD961092281510922915D3
:104F300010922A1510922B150F94CB050C94513218
:104F400080913C1282FF03C08B7F80933C12809142
:104F50002E04882319F081E00F94BE040E948D8BEB
:104F60000F94CB050C94513280913C1283FD02C00A
:104F70000C94513283E50E94BBF081110C944F34A4
:104F80000C94513283E40E9472F08823C1F18CE1C9
:104F900097E00E942CF48091A013882339F1BE0180
:104FA0006F5F7F4F8DE993E10E943BC28E010F5FDF
:104FB0001F4FD8018D918D01882319F00E94273849
:104FC000F8CFCE0101960E94B3998091F60D882307
:104FD00089F080E20E94273806EF1DE0F8018191F8
:104FE0008F01882339F00E942738F8CF82E197E0BB
:104FF0000E942CF48AE00E9427380C945132809150
:105000003C1282FF21C08BE297E00E942CF4609159
:1050100038127091391280913A1290913B124AE005
:105020000E942E388FE20E942738609134127091CE
:10503000351280913612909137124AE00E942E3834
:105040000E942C390C9451328DE397E00E942CF48D
:105050000C9451328091B9039091BA030E94E19966
:105060000C94513280913C128E7F80933C120C94B0
:10507000513280913C1283FD02C00C9451320F9446
:10508000A6058091B9039091BA030E943F990C94B0
:10509000513280913C1282FD0E94B0EC80913C1212
:1050A00083FD02C00C94513260E080E50E94D7F08D
:1050B000182F682F8091B9039091BA030E942F9AFC
:1050C00083E50E94BBF0882321F00E9403F00E9438
:1050D000B65B0E94289711110C9451320E9447EA46
:1050E0000C9451320E943E8B6C8F7D8F8E8F9F8FE0
:1050F000BE016F5F7F4FCE014C960E94075A60E061
:10510000CE0101960E94E2D60E9434F5BE016F5F87
:105110007F4F8EE497E00E941DF58AE00E942738B9
:105120000C9451326DE070E080E50E94C8F08C0173
:1051300097FF02C00C945132E82E60E089E40E948F
:10514000D7F081110C945434802F0F947C3081114E
:1051500003C60C94543480E50E9472F0882311F445
:105160000C9451320E9413F090E08536910510F0B6
:1051700084E690E08093C1030C9451320E948D8BA1
:105180000C9451320E94A3EA0C94513260E070E01A
:1051900083E50E94C8F08E34910531F40E9414EB2F
:1051A0000F94CB050C94513283EC97E00E942CF4C1
:1051B0006091C7047091C8048AEB97E00E94F2F4F2
:1051C0006091C9047091CA048DEA97E00E94F2F4DC
:1051D0006091C7047091C8048091C9049091CA0479
:1051E000681B790B8091380E815021E030E08230CD
:1051F00010F020E030E0621B730B82EA97E00E941F
:10520000F2F48AE00E94273883EC97E00E942CF4A5
:105210008091CB049091CC04A091CD04B091CE04A8
:105220008C8F9D8FAE8FBF8FBE016F5F7F4FCE0182
:105230004C960E94075ABE016F5F7F4F85E997E049
:105240000E941DF58091CF049091D004A091D104CB
:10525000B091D2048C8F9D8FAE8FBF8FBE016F5FD8
:105260007F4FCE014C960E94075ABE016F5F7F4F61
:1052700085E897E00E941DF520E030E04AE754E41D
:105280006091D3047091D4048091D5049091D60498
:105290000F942648AB01BC018DE697E00E94FFF415
:1052A0008DE60E9427388AE00E9427380C945132FC
:1052B0008091740C83FF02C00C9451320E940DDF68
:1052C00087FF02C00C94513289E40E94BBF088230E
:1052D00011F40C948B340E9413F090E01816190608
:1052E00014F481E090E026E0289FF001299FF00D62
:1052F0001124E15DFB4F808191810C949534809164
:10530000740C83FF02C00C9451320E940DDFF82E02
:1053100087FF02C00C94513289E40E94BBF0082F31
:10532000882311F40C949E340E9413F090E0181618
:10533000190614F481E090E026E0289FF001299FEF
:10534000F00D1124E15DFB4F8081918110E00C9400
:10535000AE340E940DDF182F87FD0AC082E191E470
:105360000E942CF4812F0E943CC68AE00E942738BC
:105370002CA52093E80D0C94733680E50F94D0078C
:1053800081110C94513281E40E9472F0882329F03B
:1053900060917007062F10E002C00FEF10E089E463
:1053A0000E94BBF0882399F00E9413F090E0181639
:1053B000190614F481E090E026E0289FF001299F6F
:1053C000F00D1124E15DFB4F0481158108C083E5D8
:1053D0000E94BBF0882319F00E9403F08B01B801F2
:1053E0000F3F110519F010F06FEF70E06093700738
:1053F0000C94513280E50F94D00781110C945132F6
:10540000109270070C9451328EE40E94BBF08823F6
:1054100011F40C9451320E9403F06093B015709314
:10542000B1158093B2159093B3150C94513283E566
:105430000E9472F0882329F083E50F94D0078093AF
:10544000740C0E9434F584EE97E00E942CF4809155
:10545000740C882369F1F9E7EF2EF9E0FF2E00E0E4
:1054600010E020E08091740C90E0A0E0B0E0002E0D
:1054700004C0B695A795979587950A94D2F780FFB3
:105480000EC0DD24D394D20E222319F08CE20E94A8
:105490002738F701859194910E942CF42D2D0F5FF0
:1054A0001F4F32E0E30EF11C05301105D9F6A2CDF5
:1054B00080EE97E09DCD41E060E070E08BEE97E0FC
:1054C0000E94A1F50C9451320E94B9360C945132CD
:1054D00083E50E94BBF0882371F00E9413F0282F0F
:1054E00030E02D3331051CF480930002DAC78CE3E1
:1054F00080930002D6C70E9434F54091000250E02C
:1055000060E070E089EF97E00E94E1F48AE00E9499
:105510002738C7C78091740C83FDC3C789E40E94F4
:10552000BBF0882311F40C94F8340E9413F090E03F
:105530001816190614F481E090E026E0289FF00187
:10554000299FF00D1124E15DFB4F828193810C9422
:1055500003358091740C83FDA4C789E40E94BBF0DD
:10556000882311F40C940A350E9413F090E0181669
:10557000190614F481E090E026E0289FF001299FAD
:10558000F00D1124E15DFB4F8281938110E00C94BA
:105590001B3583E50E94BBF0882309F482C70E9473
:1055A00013F0182F90E0CD970CF01CE31093F1024C
:1055B0000E947BFA6B017C01212F30E0A8EEB3E062
:1055C0000F94C046C60ED71EE81EF91EC092ED020B
:1055D000D092EE02E092EF02F092F00262C70E94D7
:1055E000A5CB0E94A3EA0E942AEE0E94933768EEA0
:1055F00073E080E090E00E9408F460E085E298E0CB
:105600000E944ED64EC780913C0E8F7E8062809362
:105610003C0E47C70F94362444C783E50E9472F0BE
:10562000882309F43EC70E947BFA6093D80C7093DC
:10563000D90C8093DA0C9093DB0C0E943BF020E0B5
:1056400030E04AE754E40F947C400F949F48609305
:10565000F2027093F3028093F4029093F50221C753
:105660000E940DDF87FD1DC79091201594FD04C099
:105670009091221597FF0AC07FE7C72E72E0D72EC0
:10568000E5E7EE2EECE0FE2E10E009C09091231528
:10569000937091F7682F81E00F94962402C7D6018A
:1056A0008D916D010E94BBF0882309F459C013301D
:1056B00009F04FC00E943BF04B015C0120E030E05C
:1056C00040EA51E40F94164087FF3AC0A5019401C7
:1056D0006091950C7091960C8091970C9091980C1C
:1056E0000F9426482B013C019B01AC016091A50C55
:1056F0007091A60C8091A70C9091A80C0F947C40FF
:105700006093A50C7093A60C8093A70C9093A80CA3
:1057100060916407709165078091660790916707B3
:105720000F941B40A30192010F947C400F949F485B
:10573000609364077093650780936607909367078B
:105740008092950C9092960CA092970CB092980C27
:1057500007C00E943BF0F701648B758B868B978B9B
:105760001F5FF4E0EF0EF11C143009F098CF0E9497
:10577000C5EB97C60F94002294C68091B90390910F
:10578000BA03009709F4D8CBDC012C91222309F449
:10579000D3CB60E00E94E2D684C6F8018081282F36
:1057A0002B7F213499F08035E9F4818180538A3050
:1057B000C8F498012E5F3F4F89012F5F3F4FF801DA
:1057C00080818032C9F3915041F70CC0218121338F
:1057D00049F4813421F0853461F741E0EACFFF24B8
:1057E000F394E7CF41110E9434F5FF2021F085E3C7
:1057F00098E00E942CF4C8010E94323952C60E94DF
:105800000F8B4FC681E08093D8048093D7040E9409
:10581000338B47C61092D8041092D7040E94338B62
:1058200040C660E070E083E50E94C8F0823038F046
:105830000E9430F589E398E00E942CF432C68C0176
:10584000112788E40E94BBF08823E1F00E9437F022
:105850008A3A910544F00E9437F08530914034F443
:105860000E9437F005C08AEA90E002C084E091E02F
:1058700026E0209FF001219FF00D1124E15DFB4FF8
:105880009183808382E40E94BBF08823D9F00E9438
:1058900037F0059744F00E9437F08437910534F4CF
:1058A0000E9437F005C085E090E002C083E790E0F9
:1058B00026E0209FF001219FF00D1124E15DFB4FB8
:1058C0009383828386E40E94BBF0882309F4E9C5B0
:1058D0000E9437F097FD09C00E9437F08F3F910575
:1058E00009F034F40E9437F005C080E090E002C077
:1058F0008FEF90E026E0209FF001219FF00D112412
:10590000E15DFB4F95838483CCC50E940DDF182F8A
:1059100087FDC7C50091510E84E40E94BBF0882327
:1059200011F40C9444350E943BF06B017C0120E0A3
:1059300030E0A9010F941640882341F124E01202BF
:10594000F0011124E35BF14FC082D182E282F38245
:1059500020E030E0A90160914D0E70914E0E8091D3
:105960004F0E9091500E0F94164081110CC080E0A4
:1059700090E0A0EEBFE380934D0E90934E0EA09367
:105980004F0EB093500E01E00C94443580E08093AC
:10599000510E0E94C98085C50E940DDF87FD81C51B
:1059A0005FE7E52E52E0F52E05E71CE065E8C62E20
:1059B0006CE0D62ED7018D917D010E9472F0882374
:1059C00059F00E943BF00F949F48F8016083718367
:1059D000828393830E947EEB0C5F1F4FC016D1061B
:1059E00049F75FC50E940DDF87FD5BC54FE7E42ED9
:1059F00042E0F42E05E71CE0D7018D917D010E9465
:105A000072F0882339F00E943BF0F80164A375A37B
:105A100086A397A30C5F1F4FFCE005381F0761F7B3
:105A200040C58091211587FF02C00C944A358091B2
:105A300022158E7011F00C944A354091A90C5091AA
:105A4000AA0C6091AB0C7091AC0C8BE598E00E94B5
:105A5000FFF44091AD0C5091AE0C6091AF0C709181
:105A6000B00C81ED9CE10E94FFF44091B10C50918B
:105A7000B20C6091B30C7091B40C85ED9EE10E9464
:105A8000FFF48AE00E9427380CC58091201581FF21
:105A900002C00C9490358091211581FF02C00C94B6
:105AA0009035809122158C7011F00C949035F9C4CA
:105AB0003EE5E32E3EE0F32E10E088E5810F0E94E4
:105AC00072F0882359F00E943BF0D7016D937D93CB
:105AD0008D939C931397812F0E9467851F5FB4E07D
:105AE000EB0EF11C133049F70E94888ADAC483E573
:105AF0000E9472F0882351F00E943BF060930E04E4
:105B000070930F04809310049093110486E40E9414
:105B100072F0882381F00E943BF020E030E040E703
:105B200052E40F94264860931204709313048093F8
:105B30001404909315048AE50E9472F0882351F0B2
:105B40000E943BF06093160470931704809318042E
:105B50009093190487E50E9472F0882309F4A1C488
:105B60000E943BF0609322047093230480932404EA
:105B70009093250496C483E50E9472F0882351F027
:105B80000E943BF060931A0470931B0480931C04E2
:105B900090931D0486E40E9472F0882381F00E9495
:105BA0003BF020E030E040E752E40F942648609359
:105BB0001E0470931F04809320049093210482E5B7
:105BC0000E9472F0882381F00E943BF020E030E0D8
:105BD00040E752E40F94264860932A0470932B0404
:105BE00080932C0490932D0487E50E9472F0882303
:105BF00009F457C40E943BF0609326047093270475
:105C000080932804909329044CC483E50E9472F089
:105C1000882309F446C40E9427F080930D040E9453
:105C2000FADD3FC483E50E94BBF0882331F00E9477
:105C300037F090931102809310028091201590917B
:105C40002115A0912215B0912315892B8A2B8B2B1E
:105C500009F027C460911002709111028AE898E05F
:105C60000E9410F585E20E9427388AE00E942738BA
:105C700018C40E940DDFF82E87FD13C483E50E942F
:105C8000BBF00F2D0F2C000C110B882369F10E9423
:105C900037F0F801EE0FFF1FEA5EFD4F918380831E
:105CA000000F111F000F111FF801EC5DFD4F7F0168
:105CB000BC01990F880B990B0F941D402AE037ED1A
:105CC00043E25CE30F947C40F801E954FB4F2081F0
:105CD0003181428153810F947C40D7016D937D9334
:105CE0008D939C931397DDC30E9434F585E40E9445
:105CF000273880E38F0D0E942738000F111FF8010D
:105D0000EA5EFD4F608171818EE898E00E9410F597
:105D100085E20E9427388AE00E942738C2C380E5C6
:105D20000E9472F0882309F4BCC360E070E080E553
:105D30000E94C8F0F82E6FEF7FEF83E50E94C8F055
:105D40008C010196039708F0ACC3F7FCAAC38F2D12
:105D50000F947C30882339F00E9430F586E998E072
:105D60000E942CF49EC30E94B0EC60E08F2D0E9434
:105D70003CF90F3FBFEF1B0731F00130110571F007
:105D800000E010E00DC08F2D0F94433931E020E08A
:105D9000892B09F030E0032F122F02C001E010E040
:105DA0008F2D0F9443398017910709F47AC380E04F
:105DB0000E945339F5CF8AE50E94BBF0811106C0DD
:105DC00083E50E94BBF0882309F440C00E943BF0A9
:105DD00020E030E040E050EC0F94164087FDFFC615
:105DE0000E943BF020E030E040E050E40F948C490A
:105DF00018160CF4EEC60E943BF06B017C0184E0A7
:105E00000E948785811122C02091910C3091920CC3
:105E10004091930C5091940CC701B6010F947C40B3
:105E20000F9498482091A5063091A606260F371F9B
:105E30003093A6062093A5062091D50C3091D60C60
:105E4000620F731F7093D60C6093D50C809122154E
:105E500087FDCBC680912315837009F0C6C60E94CA
:105E600034F540913B0450913C0460913D047091A5
:105E70003E0485EA98E00E94FFF48AE00E942738F9
:105E800010C364E071E083E50E94B2E58C0168EE26
:105E900073E080E50E94B2E58938E3E19E0710F0E7
:105EA00088E893E1B8010E9417D6FBC285E40F94FD
:105EB000D007811173C080E50E9472F0882351F0F1
:105EC0000E943BF060933A0F70933B0F80933C0F1E
:105ED00090933D0F89E40E9472F0882381F00E9424
:105EE0003BF02CEA35EC47E25EE30F947C40609394
:105EF0003E0F70933F0F8093400F9093410F84E4C7
:105F00000E9472F0882381F00E943BF02CEA35EC6D
:105F100047E25EE30F9426486093420F7093430F6D
:105F20008093440F9093450F0E9434F540913A0FAF
:105F300050913B0F60913C0F70913D0F8AEB98E0C0
:105F40000E94FFF42CEA35EC47E25EE360913E0FDD
:105F500070913F0F8091400F9091410F0F94264810
:105F6000AB01BC0186EB98E00E94FFF42CEA35EC13
:105F700047E25EE36091420F7091430F8091440FBE
:105F80009091450F0F947C40AB01BC0182EB98E0EF
:105F90000E94FFF48AE00E94273883C20E9430F5F5
:105FA00088ED95E30E942CF47CC283E50E9472F098
:105FB000182F882371F00E943BF00F94984870933B
:105FC00029026093280221E0672B09F020E020934A
:105FD000810780E50E9472F0882359F02091280201
:105FE00030912902232B11F00E9427F08093810722
:105FF00058C2111156C20E9434F587ED98E00E94F4
:106000002CF480918107882319F080E198E202C086
:106010008EEB98E00E942CF4609128027091290286
:1060200086EC98E00E9410F582EC98E00E942CF437
:1060300038C20E94B0EC35C280912215867009F0FA
:10604000DAC50E9434F58AEE98E00E942CF4809123
:106050000A020E94D5F425C20F948C2722C20F9405
:10606000790781111EC207E219E321E531E139A365
:1060700028A3CE0101961C0174E9C72E78E2D72E21
:106080007C01F8016591759185919491A8A1B9A1C0
:106090008D909D90AD90BD90B9A3A8A3A50194014A
:1060A0000F942B472B013C01F7016083718382839E
:1060B000938320E030E040EA51EC0F948C4987FD57
:1060C0000AC020E030E040EA51E4C301B2010F947D
:1060D000164018162CF4F601849118160CF4A2C57B
:1060E000D7018D909D90AD90BD907D0120E030E076
:1060F00040EA51ECC501B4010F948C4987FD9DC560
:1061000020E030E040EA51E4C501B4010F941640AC
:1061100018160CF0A6C591C50E94FEE5C2C10F94E9
:10612000CA14BFC161E083E50E94D7F091E08927DE
:106130000E946D7DB6C181E0809301150F94F11529
:1061400010920115882309F4ACC10E9434F58DE347
:1061500099E00E942CF4A5C180913C1282FFA1C15C
:10616000806480933C129DC10E947EE29AC10E948D
:106170000DDF082F87FD95C185E50E9472F0882309
:10618000B1F1E02E002E000CFF080E943BF04B0105
:106190005C0120E030E0A9010F948C4987FF04C026
:1061A000B7FAB094B7F8B094C70153E0880F991FBD
:1061B0005A95E1F79C012B5F3B4F7901D9018D92F4
:1061C0009D92AD92BC92139720E030E048E453E4F6
:1061D000C501B4010F948C4918164CF480E090E08E
:1061E000A8E4B3E4F70180839183A283B3838CE4B2
:1061F0000E9472F0882309F454C1002E000C110B88
:106200000E943BF06B017C0120E030E0A9010F947B
:106210008C4987FF04C0F7FAF094F7F8F09420E077
:1062200030E048E453E4C701B6010F948C4998016B
:1062300043E0220F331F4A95E1F7F901EB5FFB4F73
:1062400018162CF0C482D582E682F7822AC180E03B
:1062500090E0A8E4B3E484839583A683B78321C147
:106260000E9450E11EC10E940DDF182F87FD19C149
:106270008AE50E94BBF0882349F040E050E0BA0173
:106280008AE50E94FF554B015C0106C0812C912CD0
:1062900090EAA92E91E4B92E412F64E083E00E9498
:1062A0007F6320E030E0A901C501B4010F948C495F
:1062B00018167CF580E090E0A0EAB0E489839A8328
:1062C000AB83BC832091591130915A1140915B11DD
:1062D00050915C11C501B4010F942C476B017C01F6
:1062E00020E030E04BE953E40F94164087FD06C0F0
:1062F000C12CD12C8BE9E82E83E4F82ECC8EDD8ED8
:10630000EE8EFF8EBE016F5F7F4FCE014C960E94D6
:10631000378A85E50E9472F0882329F00E943BF0BD
:106320006B017C010AC028E01202F0011124EB5F2E
:10633000FB4FC080D180E280F38020E030E0A901F3
:10634000C701B6010F948C4987FF04C0F7FAF09497
:10635000F7F8F094F7FAF094F7F8F094C982DA823B
:10636000EB82FC8264E0CE0101960F94EE0520E002
:1063700030E0A901C501B4010F948C4918165CF5F1
:1063800080E090E0A0EAB0E489839A83AB83BC8389
:10639000A50194016091591170915A1180915B117E
:1063A00090915C110F942B476B017C0120E030E051
:1063B000A9010F948C4918161CF0C12CD12C760120
:1063C000CC8EDD8EEE8EFF8EBE016F5F7F4FCE01D5
:1063D0004C960E94378A40E060E089E00E947F632B
:1063E00060C081E08093A1061092370D60E083E5E4
:1063F0000E94D7F0811155C00F94C41B52C083E591
:106400000E9472F0882339F00E9427F080932E04B6
:106410000E94F4F046C00E9434F588E499E00E949E
:106420002CF480912E040E94D5F43BC00E9436DFEC
:1064300038C00E943E8B6D3371058105910520F0B7
:1064400085E799E00F94B12281E799E00F94B1229A
:1064500084EE8093C1030E94ECF00E94A8998DE520
:1064600099E00E942CF489E19CE39093DD048093F1
:10647000DC0417C00F94BD0514C0109125150E94AF
:106480007BFA6093D80C7093D90C8093DA0C9093BC
:10649000DB0C112331F0812F0E9417C602C00F942C
:1064A000BD053DA5311102C00F94B41B8CA580938E
:1064B000E80D19C48090E20D9090E30DA090E40DDA
:1064C000B090E50D20915D1130915E1140915F110A
:1064D00050916011C501B4010F942B476B017C01F1
:1064E00020E030E0A9010F948C4987FFEFC32DEC29
:1064F0003CEC4CEC5DEBC701B6010F94164018164E
:106500005CF0C701B601905820E030E040E251E471
:106510000F94164018161CF40E943B86C2CF11E05F
:1065200020E030E0A901C701B6010F948C4918168C
:106530000CF010E08091EC028113EECF80925D119F
:1065400090925E11A0925F11B09260118DE591E181
:106550000E94C1EC20E030E0A901C701B6010F9410
:106560001640881F8827881F0E948AF19ACF20E052
:1065700030E0A901C701B6010F941640881F882793
:10658000881F181709F4A2C080E090E0A0E8BFEBD4
:1065900088A799A7AAA7BBA728A139A14AA15BA14F
:1065A000C501B4010F942B4720E030E040E05FE3E9
:1065B0000F947C4068A379A38AA39BA32CA13DA13F
:1065C0004EA15FA1C301B2010F942B4720E030E040
:1065D00040E05FE30F947C402B013C0128A139A1EE
:1065E0004AA15BA1CA01B9010F947C404B015C0137
:1065F000A3019201C301B2010F947C409B01AC0145
:10660000C501B4010F942C470F94DA494B015C018A
:106610009B01AC01C701B6010F942B476CA37DA36E
:106620008EA39FA3A5019401C701B6010F942C4727
:106630009B01AC016CA17DA18EA19FA10F947C4018
:106640006B017C0120E030E0A9010F948C4987FDAB
:1066500007C0C701B6010F94DA496B017C0103C082
:10666000C12CD12C7601C301B2019058A50194012F
:106670000F94264828A539A54AA55BA50F947C4010
:10668000A70196010F947C4028A139A14AA15BA1E2
:106690000F942C4769837A838B839C83A501940193
:1066A00068A179A18AA19BA10F94264828A539A5A4
:1066B0004AA55BA50F947C40A70196010F947C40EE
:1066C000A30192010F942C470C94D02280E090E01B
:1066D000A0E8BFE35DCF412FBE016F5F7F4F86ED26
:1066E0009DE00F940D1E0E947BFA6093D80C70936E
:1066F000D90C8093DA0C9093DB0CD3CE0E9430F54A
:1067000083E896E00E942CF4CCCE0E94B0ECE0909E
:10671000410E80E00E94D7F20E947BFA6093D80C71
:106720007093D90C8093DA0C9093DB0C8091560215
:1067300090915702A0915802B09159028093F802AB
:106740009093F902A093FA02B093FB028091100299
:10675000909111029093F7028093F60284E690E004
:10676000909311028093100281E08093D8040E94DC
:10677000338B8AE50E9472F0F82E88E50E9472F051
:10678000182F89E50E9472F018135DC0F11611F000
:10679000012F04C001E011E0FF24F39482E50E9480
:1067A000BBF0882319F00E943BF004C060E070E069
:1067B00080EA90E469837A838B839C8320E030E0D5
:1067C000A9010F941640882341F0111102C0002343
:1067D00071F0CE0101960F94D707112319F080E0D4
:1067E0000F946931002319F081E00F946931FF2083
:1067F00019F082E00F9469310E94868A8091D70453
:106800008093D8048E2D0E94D7F28091F802909147
:10681000F902A091FA02B091FB0280935602909384
:106820005702A0935802B09359028091F6029091BA
:10683000F702909311028093100283E080936E021E
:106840000E94888A2ECE082FA9CF88E50E9472F078
:1068500081115F9889E50E9472F081118A988AE51A
:106860000E9472F0882329F0809108018170809342
:10687000060185E40E9472F0882309F412CE129872
:1068800010CE60E081EE96E00E944ED65F988A9826
:1068900080910801817080930601129802CE0E94B7
:1068A00003F00E94B65BFDCD8DE40E94BBF088230F
:1068B000A9F00E9413F0813039F020F0823049F4C1
:1068C00062E003C060E001C061E0802F0E943CF9FB
:1068D00005C08BE597E00E942CF4E3CD83E50E9490
:1068E000BBF0882309F4DDCD0E9413F0F82EF9E007
:1068F000EF1203C080937007D4CD61E0802F0E9417
:106900003CF96F2D802F0E940DF96F2D70E0802FC4
:106910000E9478F9C6CD83E50E94BBF0882359F028
:106920000E943BF00F949848CB010E942CC661E076
:1069300080E00F94B4370F94F837B3CD83E50E940D
:10694000BBF0182F811105C082E50E94BBF088239F
:1069500041F10E943BF00F949848CB010E942CC655
:1069600061E081E00F94B4376091370F7091380F78
:10697000072E000C880B990B0F941D404B015C01F6
:106980004090330F5090340F6090350F7090360F59
:10699000A30192010F948C4918163CF1112361F068
:1069A00001E00F94F837002309F47BCD40E0612F1C
:1069B0008F2D0E9441C875CDA3019201C501B4017C
:1069C0000F948C4918168CF08BEC97E09F938F9363
:1069D0008BED97E09F938F931F920E94C7D60F90E5
:1069E0000F900F900F900F90DBCF85EC92E3EECFDE
:1069F00083E50E94BBF0882309F453CD0E943BF04D
:106A00000F949848CB010E94F5EF61E080E00F946D
:106A1000B43747CD83E50E94BBF0182F811106C023
:106A200082E50E94BBF0882309F43BCD0E943BF035
:106A30000F949848CB010E94F5EF60E081E00F943D
:106A4000B43760914A0E70914B0E072E000C880BE4
:106A5000990B0F941D402091460E3091470E4091A6
:106A6000480E5091490E0F948C49181654F080E04E
:106A700098E060E00E944ED660E0812F0E94AEC692
:106A800010CD83E198E0F5CF602F83E50E94D7F029
:106A90000C94C72C83E50E94BBF0882391F00E94E0
:106AA0003BF06093A90C7093AA0C8093AB0C90936D
:106AB000AC0C6093B10C7093B20C8093B30C9093B8
:106AC000B40C80E50E94BBF0882351F00E943BF09B
:106AD0006093A90C7093AA0C8093AB0C9093AC0CB0
:106AE00082E50E94BBF0882351F00E943BF0609346
:106AF000AD0C7093AE0C8093AF0C9093B00C84E50A
:106B00000E94BBF0882309F4CCCC0E943BF0609338
:106B1000B10C7093B20C8093B30C9093B40CC1CCB5
:106B200082E40E9472F0882351F00F94D124609384
:106B3000850C7093860C8093870C9093880C83E56A
:106B40000E9472F0882351F00E943BF06093B50CD4
:106B50007093B60C8093B70C9093B80C84E50E94A8
:106B600072F0882351F00E943BF06093B90C70934F
:106B7000BA0C8093BB0C9093BC0C8AE40E9472F018
:106B8000882309F48ECC0E943BF06B017C012AE043
:106B900037ED43E25CE30F948C4987FD13C02AE98B
:106BA00039E949E95EE3C701B6010F9416401816AA
:106BB0004CF0C0925407D0925507E0925607F092DD
:106BC00057076FCC0E9430F58BE698E00E942CF4BA
:106BD00068CCC12CD12CE12CF0E4FF2E10C9C12CC3
:106BE000D12CE12CE0ECFE2E0AC982E50E9472F065
:106BF000811135C956CC82E50E9472F0082F83E5D9
:106C00000E9472F0182F011103C0112309F449CC1E
:106C10000E9497EE112309F444CC0E9427F0809340
:106C20000A023FCCB7FAB094B7F8B094D7018D926E
:106C30009D92AD92BC92139753CA0E9430F58FE19A
:106C400099E00E942CF461E081E199E00E944ED627
:106C50000E943E4D68E270E088EC90E00E9417D6FA
:106C600020CC0C5F1F4FBFEFCB1ADB0AE9E30333E5
:106C70001E0709F006CA6EE5E62E6EE0F62E10E05D
:106C8000F10181919191A191B1911F01F70181933E
:106C90009193A193B1937F01812F0E9467851F5F1C
:106CA000133071F70E94888A60E08BEF98E00E94B1
:106CB0004ED663E972E084E690E00E9417D66AEB54
:106CC00072E084E690E00E9417D6EBCB2DEC3CEC12
:106CD0004CEC5DE3C701B6010F948C4987FD1CCCD9
:106CE000C701B60111CCAD960FB6F894DEBF0FBE4A
:106CF000CDBFDF91CF911F910F91FF90EF90DF906B
:106D0000CF90BF90AF909F908F907F906F905F904B
:106D10004F903F902F9008958091A70681110AC04F
:106D20008091380E813041F080913C1282FB88279F
:106D300080F9089580E0089581E00895129A0895F9
:106D40005F9A8091DA048E7F8093DA048A9A809128
:106D5000DA048D7F8093DA04809108018095817038
:106D6000809306018091DA048B7F8093DA040C947F
:106D70009E368F929F92AF92BF92CF92DF92EF9208
:106D8000FF920F931F93CF93DF93CDB7DEB760973A
:106D90000FB6F894DEBF0FBECDBF0E94DA84182F65
:106DA000809194118093931180939211809391110B
:106DB00084E6809390110E9470EB80ED93E09093B5
:106DC000730C8093720C11110E94E78481E0809310
:106DD000B9150E94B0EC81E00E9400EE6B017C01CD
:106DE00080E00E9400EE4B015C016093FF02709313
:106DF00000038093010390930203C0920303D09297
:106E00000403E0920503F092060382E00E9400EE84
:106E100060930703709308038093090390930A0318
:106E20008E010F5F1F4F20E1F80111922A95E9F7BB
:106E300089829A82AB82BC82CD82DE82EF82F88622
:106E400069877A878B879C8783E00E9400EE6B01BD
:106E50007C0120913F0730914007409141075091BC
:106E6000420769857A858B859C850F942B476987B6
:106E70007A878B879C87A701960160913B07709169
:106E80003C0780913D0790913E070F942C476D87FA
:106E90007E878F87988B8091410E882319F0C801D7
:106EA0000E9443EB80E1F801A1E5B1E101900D9270
:106EB0008A95E1F70E94868A60960FB6F894DEBF45
:106EC0000FBECDBFDF91CF911F910F91FF90EF903B
:106ED000DF90CF90BF90AF909F908F90089590914A
:106EE0003C1293FB882780F993FF06C081E09091C4
:106EF000A013911101C080E008958091A70681112F
:106F000010C08091380E823061F00E946F37882364
:106F100049F080913C1282FB882780F991E0892713
:106F2000089581E008951092700708958F929F92BE
:106F3000AF92BF92CF92DF92EF92FF920F93CF93D7
:106F4000DF931F92CDB7DEB75C016B017A01490177
:106F5000F501808191810F9446468983002311F0C9
:106F6000F6018083BE016F5F7F4FC4010F94940AC6
:106F7000F50180819181019691838083FFEFCF1A83
:106F8000DF0A81E0E81AF10819F780E00F90DF913D
:106F9000CF910F91FF90EF90DF90CF90BF90AF9087
:106FA0009F908F9008957F928F929F92AF92BF9201
:106FB000CF92DF92EF92FF920F931F93CF93DF93C5
:106FC0001F92CDB7DEB77C0159018B016B01C40E56
:106FD000D51E0C151D0559F1F70180809180F8012F
:106FE00071908F017982C4010F944646781691F012
:106FF000672DC4010F944E46C4010F9446469981F3
:10700000891741F00E9434F583E899E00E942CF43E
:1070100081E00EC0BE016F5F7F4FC5010F94940ADF
:10702000F70180819181019691838083D2CF80E0A6
:107030000F90DF91CF911F910F91FF90EF90DF9014
:10704000CF90BF90AF909F908F907F900895909138
:10705000C00095FFFCCF8093C60008958F929F9249
:10706000AF92BF92EF92FF920F931F93CF93DF9354
:10707000CDB7DEB7A0970FB6F894DEBF0FBECDBF79
:10708000611571058105910591F100E0842E912C27
:10709000A12CB12C102FEE24E394F12CEC0EFD1E4C
:1070A000E00EF11C07FDFA94A50194010F946C46C3
:1070B000F7016083B901CA010F5F61157105810590
:1070C000910541F71F3F31F1E1E0F0E0EC0FFD1FCA
:1070D000E10FF11D17FDFA9580818A3010F097E3DA
:1070E00001C090E3890F0E9427381150EBCF80E355
:1070F000A0960FB6F894DEBF0FBECDBFDF91CF9143
:107100001F910F91FF90EF90BF90AF909F908F9045
:107110000C942738A0960FB6F894DEBF0FBECDBFF3
:10712000DF91CF911F910F91FF90EF90BF90AF90A3
:107130009F908F900895CF92DF92EF92FF926B0114
:107140007C0197FF0BC08DE20E942738F094E094F9
:10715000D094C094C11CD11CE11CF11C4AE0C701B1
:10716000B601FF90EF90DF90CF900C942E388F9265
:107170009F92AF92BF92CF92DF92EF92FF92CF9306
:107180006B017C01B42E20E030E0A9010F94164081
:1071900087FF07C08DE20E942738F7FAF094F7F8CE
:1071A000F094C0E060E070E080E09FE3CB1541F038
:1071B0002DEC3CEC4CEC5DE30F947C40CF5FF6CFC4
:1071C0009B01AC01C701B6010F942C476B017C01F8
:1071D0000F949F484B015C014AE00E942E38CC235B
:1071E00089F1C501B4010F941B409B01AC01C7019B
:1071F000B6010F942B476B017C018EE20E94273869
:1072000020E030E040E251E4C701B6010F947C4039
:107210004B015C010F9498486B01770FEE08FF0853
:10722000C701B6010E949B38C701B6010F941D40EB
:107230009B01AC01C501B4010F942B476B017C018C
:10724000C150F1F6CF91FF90EF90DF90CF90BF90BB
:10725000AF909F908F9008958DE00E9427388AE02C
:107260000C942738CF93DF93EC018991882319F090
:107270000E942738FACFDF91CF910C942C3980915E
:107280002C1590912D15981759F0E92FF0E0E45D39
:10729000FA4E82819F5F9F7790932D1590E008951D
:1072A0008FEF9FEF08952F923F924F925F926F92D0
:1072B0007F928F929F92AF92BF92CF92DF92EF9286
:1072C000FF920F931F93CF93DF93CDB7DEB72A972B
:1072D0000FB6F894DEBF0FBECDBFF82E80919F068B
:1072E000843008F0E0C180919F06843008F001C12D
:1072F00080912C1590912D15891B8F7709F4F9C079
:107300000E943F3997FDEFCF8A3019F08D3009F098
:10731000E7C010920B038091AE159091AF15FC0160
:10732000E45FFC4F1082892B39F01092AF15109258
:10733000AE150CE013E003C00F949D2AD4CFF801E2
:107340008191803211F48F01FACF8E3409F06AC036
:107350000115110509F466C067EA7AE0C8010F94C7
:10736000943F6C01892B41F06EE470E0C8010496F3
:107370000F94864A009709F4C8014AE050E060E0A3
:1073800070E001960F94FC3C4B015C018091B015BC
:107390009091B115A091B215B091B3150196A11DB0
:1073A000B11D88169906AA06BB0631F0CD2821F436
:1073B00060E084E79AE049C06AE270E0C8010F9497
:1073C000B54A9C01009709F1982F901BE12C992355
:1073D00039F09150F801E90FF11D8081E826F7CFCF
:1073E0004AE050E060E070E0C90101960F94FC3C77
:1073F0004E2C512C612C712C641575058605970552
:1074000041F060E085E59AE020C060E08BE29AE020
:107410001CC08092B0159092B115A092B215B09296
:10742000B31516C080913C1280FF12C06DED70E361
:10743000C8010F94943F009729F0FC018381805389
:107440008A3030F460E08BE29AE00F94E01B51C088
:107450008091A1068130E1F067E470E0C8010F94EB
:10746000864A0097A9F04AE050E060E070E001969B
:107470000F94FC3C643071058105910548F484EB60
:1074800099E00E942CF460E08CEA99E00E944ED6CC
:1074900067EA79E0C8010F94543F892B21F41092D8
:1074A00023021092E70D62EA79E0C8010F94543F7D
:1074B000892B39F441E060E070E08BEE97E00E94A8
:1074C000A1F56DE979E0C8010F94543F892B11F4BF
:1074D0000E94B93661E08CE093E00F94381C03CF32
:1074E0002EEA35E14CE053E06BE073E00F94791B3A
:1074F000FACE80913C1282FFD6C01A82198211E026
:10750000409138125091391260913A1270913B12A9
:107510008091341290913512A0913612B0913712A9
:10752000481759076A077B0708F410E000E680E176
:10753000E82E99E6D92E80919F06843008F0B3C0DA
:107540001111B1C08091A5139091A613A091A7131A
:10755000B091A8138093381290933912A0933A12E5
:10756000B0933B1241E050E0BE016D5F7F4F8DE96B
:1075700093E10E945EBE019719F48B8190E002C0F6
:107580008FEF9FEF409038125090391260903A126E
:1075900070903B128090341290903512A090361269
:1075A000B090371211E0481459046A047B0408F4BF
:1075B00010E08F3FFFEF9F0761F4481459046A04FD
:1075C0007B0438F40E9430F58CEA9AE00E942CF497
:1075D000B2CF4091DB048A3079F08D3069F04814E5
:1075E00059046A047B0408F4A7C389819A8100972F
:1075F00019F001969A83898310926C0389819A818C
:10760000FC01049FE00DF11D1124E25EFA4F10828F
:10761000892BB1F01A82198280E00F940F1C80919F
:10762000381290913912A0913A12B0913B12809386
:10763000281590932915A0932A15B0932B1502C0F5
:107640000F949D2A481459046A047B0408F473CFEC
:107650000E94B0EC8DE993E10E946FC280913312D9
:107660008823E1F0815080933312D89EC001112409
:1076700062E08455994F0E942F9AE091331224E0E2
:10768000E29FF0011124E855F94F608171818281F8
:1076900093810E94B65B0E9428974DCF0E94179756
:1076A000E092A10648CF0E947BFA4B015C01F110E9
:1076B00050C38091A70681114CC310E04091F202A3
:1076C0005091F3026091F4027091F5024115510559
:1076D00061057105A1F08091D80C9091D90CA09111
:1076E000DA0CB091DB0C840F951FA61FB71FA50104
:1076F0009401281B390B4A0B5B0B57FF34C3809155
:107700006A0290916B02A0916C02B0916D02892B7C
:107710008A2B8B2B09F44FC0909193118091941177
:10772000981749F08092D80C9092D90CA092DA0C5C
:10773000B092DB0C40C011112BC30E947BFAC090A9
:10774000D80CD090D90CE090DA0CF090DB0C0091C2
:107750006A0210916B0220916C0230916D020C0D47
:107760001D1D2E1D3F1DDC01CB01801B910BA20BAB
:10777000B30BB7FD0DC38091770381111CC081E06D
:10778000809377035F9A8091DA048E7F8093DA0486
:107790008A9A8091DA048D7F8093DA0480910801BF
:1077A00080958170809306018091DA048B7F8093AD
:1077B000DA040E949E368091750390917603909929
:1077C00002C0019604C0181619062CF40197909374
:1077D00076038093750380917503909176038E3EB6
:1077E00092406CF00E9430F58BEB9AE00E942CF4F2
:1077F00040E060E070E080E090E00E94A1F58091C0
:10780000710390917203A0917303B0917403950179
:107810008401081B190B2A0B3B0B37FD23C19091E8
:10782000931180919411981751F0E09194111FE4F5
:10783000E19FF0011124E853F84F608102C060918C
:107840007007662311F070E002C060E070E089E02C
:107850000E9478F98091D70C882309F4F6C0E09053
:107860003502F09036020091370210913802609193
:10787000370F7091380F6E5F7F4F072E000C880B0B
:10788000990B0F941D409701A8010F94164087FD96
:10789000DCC030909411212C1C821D821E828091AC
:1078A0009311831509F467C0832D90E02FE4289F7E
:1078B000F001299FF00D1124EE57F84F45895689A4
:1078C0006789708D452B462B472B89F4418D528D4E
:1078D000638D748D452B462B472B49F4458D568D72
:1078E000678D70A1452B462B472B09F43FC04FE411
:1078F000489F9001499F300D1124C9018E57984F20
:107900006C01FC0161817281838194810F94DA4959
:107910002B013C01F60161A172A183A194A10F94F6
:107920001B406F83788789879A87F60165A176A1C6
:1079300087A190A50F941B409B01AC016F817885B6
:1079400089859A850F942648A30192010F947C4063
:107950003B016C01222D3C814D815E810F948C494D
:10796000181624F4262C7C82CD82DE8281E0830DE1
:107970008F70382E94CF20912D0230912E0240919D
:107980002F0250913002622D7C818D819E810F9457
:107990007C409701A8010F942C473B016C0120907B
:1079A00031023090320240903302509034029B01F9
:1079B000AC01B701C8010F948C4918166CF0910105
:1079C000A201B301C6010F948C4918161CF4710171
:1079D000820102C07301860140906D0350906E03D6
:1079E00060906F03709070039701A801C301B2010A
:1079F0000F948C491816C4F420E037ED43EA5CE399
:107A0000B701C8010F947C406B017C0128E431EE82
:107A10004AE75FE3C301B2010F947C40A7019601DE
:107A20000F942C477B018C01C701D80180936D0313
:107A300090936E03A0936F03B0937003B701C801D6
:107A40000F949848CB010E942CC6F4E68F0E911C2F
:107A5000A11CB11C8092710390927203A0927303D7
:107A6000B09274030F949D2A8091A106882309F493
:107A7000E4C180910A028823C9F08091650D8111CB
:107A800015C00E948C36811104C08091A7068823FE
:107A900069F08091940D87FD03C081508093940D0F
:107AA000959989C18091940D87FD75C180910901D7
:107AB000817011E0182700910102011709F44AC0F2
:107AC00090913C12906290933C12109301028111AC
:107AD0000DC064EF71E080E090E00E9408F40E9425
:107AE000D69780913C1283FD09C069C10E94179707
:107AF00080913C12877F806280933C12112309F4AD
:107B000061C1023028F460E08BE69BE00E944ED613
:107B100081E08093C0038DEB9BE19093260F8093CF
:107B2000250F1092280F1092270F83E080936E028A
:107B30000E947BFADC01CB018C599F4FAF4FBF4FA6
:107B40008093C4039093C503A093C603B093C70367
:107B5000111147C10E947BFA6B017C0180910002E8
:107B6000882359F18091E80D882339F140918003F1
:107B70005091810360918203709183039701860184
:107B8000041B150B260B370B37FD2AC0833079F009
:107B90003CF4813094F00E9434F58AE49BE00BC001
:107BA000843059F40E9434F58BE19BE004C00E94BC
:107BB00034F583E39BE00E942CF42091000230E036
:107BC000A8EEB3E00F94C046C60ED71EE81EF91EFD
:107BD000C0928003D0928103E0928203F0928303EB
:107BE0008091380E813009F06EC00E947BFA6B01E3
:107BF0007C0180917C0390917D03A0917E03B091E4
:107C00007F03A7019601281B390B4A0B5B0B57FD1D
:107C10003AC08090840D9090850DA090860DB09014
:107C2000870D0E943E8B6093840D7093850D809329
:107C3000860D9093870D0091CB041091CC04209178
:107C4000CD043091CE04081919092A093B09DC0139
:107C5000CB01800F911FA21FB31F8093CB04909381
:107C6000CC04A093CD04B093CE04D701C601805FAD
:107C7000984DAF4FBF4F80937C0390937D03A093AB
:107C80007E03B0937F038091780390917903A09154
:107C90007A03B0917B0397018601081B190B2A0B0D
:107CA0003B0B37FD10C010E8C10E1EEED11EE11CCB
:107CB000F11CC0927803D0927903E0927A03F0929B
:107CC0007B030E9481EA0E945BD20E944E6C8091ED
:107CD000F102882309F4B1C00E947BFA0091ED0201
:107CE0001091EE022091EF023091F002DC01CB0105
:107CF000801B910BA20BB30BB7FD9FC00E947BFAB8
:107D00006B017C012091F10230E0A8EEB3E00F940A
:107D1000C046C60ED71EE81EF91EC092ED02D092D4
:107D2000EE02E092EF02F092F00280E00E943CC688
:107D30008AE00E94273881C0049FA0011124425E7E
:107D40005A4F9E012F5F3F4F6CE673E00F94791BF3
:107D5000F2CB8092D80C9092D90CA092DA0CB0920F
:107D6000DB0C11E0ABCC0E9430F560913A0E7091C3
:107D70003B0E8EED9AE00E941DF58AE00E942738A6
:107D800040E060E070E080E090E00E94A1F5B7CCB8
:107D90001092770310CD81E08093650D8091A70646
:107DA000811106C083E89BE09093DD048093DC049E
:107DB0000E94B0EC7BCE85E08093940D73CE0023BF
:107DC00009F4C8CE023058F460E08CE59BE00E94D4
:107DD0004ED680913A0D811102C00E943E4D10E0B6
:107DE00097CE023009F0B6CE80913C1283FFB2CE1E
:107DF0000E94B996882379F081E00E94879649EB2A
:107E000050E06AE67EE08EE392E10E945EBE8EE381
:107E100092E10E946FC20E9404F1811107C00E948A
:107E2000ECF00E94A8991092311294CE8BE79BE05F
:107E30009093DD048093DC048DCE2A960FB6F894DF
:107E4000DEBF0FBECDBFDF91CF911F910F91FF908D
:107E5000EF90DF90CF90BF90AF909F908F907F90EA
:107E60006F905F904F903F902F900895CF92DF9248
:107E7000EF92FF92CF93DF936B017C01D42FC091DF
:107E8000E80D83E08093E80D81E08093E70DC11455
:107E9000D104E104F10431F00E947BFAC60ED71E32
:107EA000E81EF91E8091E70D882399F0C114D104D2
:107EB000E104F10421F48D2F0E945339F3CF0E9485
:107EC0007BFADC01CB018C199D09AE09BF09B7FD16
:107ED000F2CF1092E70DC093E80DDF91CF91FF90A4
:107EE000EF90DF90CF9008951F920F920FB60F92F0
:107EF00011240F900FBE0F901F9018951F920F9294
:107F00000FB60F9211240BB60F922F938F939F935E
:107F1000EF93FF939091C60020912D15E0912C15C1
:107F200081E08E0F8F77281729F0F0E0E45DFA4E9C
:107F30009283E82FE0932C15FF91EF919F918F9101
:107F40002F910F900BBE0F900FBE0F901F901895A2
:107F50008EBD0DB407FEFDCF08958FEF8EBD0DB41D
:107F600007FEFDCF8EB50895909164009B7F90939E
:107F70006400982F906A96959CBD80FD03C091E0A7
:107F8000863009F490E09DBD08950C947EEB0C942E
:107F90007EEB0C947EEB0C947EEBCF92DF92EF9213
:107FA000FF920F931F93CF93DF9361E081E00E94D4
:107FB000254CD091AE0DC0E0D1110BC08091AD0D1C
:107FC00081112AC08091A80D1092A80D81111EC0A8
:107FD00023C0D13061F48091AD0D813009F045C0EE
:107FE0008091A80D1092A80D811128C03EC0D230FA
:107FF00009F060C08091AD0D823009F08FC0809192
:10800000A80D1092A80D811172C088C00E94464D23
:108010008091CF0D81117CC180916E02882309F47B
:1080200040C081E09091AD0D911180E004E024E02A
:108030004EED56E36C2F0E943B5333C00E9448F72D
:10804000C12CD12CE12C10ECF12E09E714E420E036
:1080500030E040E85FE369E97CE08AE19CE00E946F
:10806000A6F68091CF0D811153C180916E028823B5
:10807000C1F011E08091AD0D813009F010E0609108
:10808000990C70919A0C80919B0C90919C0C0E9481
:10809000C64B00E09C014AE15CE06C2F812F0E94FE
:1080A0003E55CF5FDF5FC53009F086CF87E0809314
:1080B000A90D2EC1D33061F48091AD0D833009F04C
:1080C0006DC08091A80D1092A80D811150C066C09E
:1080D000D43009F03DC08091AD0D843009F09EC0D0
:1080E0008091A80D1092A80D811181C097C00E94A7
:1080F00048F7C12CD12CE12C10ECF12E09E714E447
:1081000020E030E040E85FE36DE97CE083E19CE063
:108110000E94A6F68091CF0D8111FAC080916E0267
:10812000882309F4BECF11E08091AD0D823009F0B3
:1081300010E060919D0C70919E0C80919F0C90912D
:10814000A00C0E94C64B00E09C0143E15CE0A5CF7F
:10815000D53009F03DC08091AD0D853009F08EC05D
:108160008091A80D1092A80D811172C087C00E9445
:1081700048F7C12CD12CE12C10ECF12E09E714E4C6
:1081800020E030E040E85FE361EA7CE08CE09CE0E6
:108190000E94A6F68091CF0D8111BAC080916E0227
:1081A000882309F47ECF11E08091AD0D833009F072
:1081B00010E06091A10C7091A20C8091A30C9091A1
:1081C000A40C0E94C64B00E09C014CE05CE065CF33
:1081D000D63009F066CF8091AD0D863009F07EC0B3
:1081E0008091A80D1092A80D811162C077C00E94E5
:1081F00048F7C12CD12CE12C10ECF12E09E714E446
:1082000020E030E040E85FE365EA7CE085E09CE068
:108210000E94A6F68091CF0D81117AC080916E02E6
:10822000882309F43ECF11E08091AD0D843009F030
:1082300010E06091A50C7091A60C8091A70C909114
:10824000A80C0E94C64B00E09C0145E05CE025CFF5
:108250000E9448F7C12CD12CE12C10ECF12E09E73B
:1082600014E420E030E0A90165EB7CE080E09CE0D4
:108270000E94A6F68091CF0D81114AC080916E02B6
:10828000882309F40ECF11E08091AD0D853009F0FF
:1082900010E06091B50C7091B60C8091B70C909184
:1082A000B80C0E94C64B00E09C0140E05CE0F5CEBB
:1082B0000E9448F7C12CD12CE12C10ECF12E09E7DB
:1082C00014E420E030E0A90169EB7CE084EF9BE05E
:1082D0000E94A6F68091CF0D81111AC080916E0286
:1082E000882309F4DECE11E08091AD0D863009F0CF
:1082F00010E06091B90C7091BA0C8091BB0C909118
:10830000BC0C0E94C64B00E09C0144EF5BE0C5CE74
:10831000DF91CF911F910F91FF90EF90DF90CF9061
:1083200008955F926F927F928F929F92AF92BF92C9
:10833000CF92DF92EF92FF920F931F93CF93DF9331
:1083400000D01F92CDB7DEB761E081E00E94254CDE
:108350006090AE0D712C43E0542E61100BC08091E3
:10836000AD0D81112AC08091A80D1092A80D811128
:108370001EC023C081E068120BC09091AD0D9130FA
:10838000C1F58091A80D1092A80D811127C031C0B0
:1083900082E068124AC08091AD0D823009F079C048
:1083A0008091A80D1092A80D811160C072C00E942A
:1083B000464D8091CF0D81111AC180916E028823A4
:1083C00061F181E09091AD0D911180E004E024E035
:1083D0004EED56E3672D0E943B531FC08091D70C92
:1083E00086258093D70C50926E028091CF0D81111B
:1083F000FEC080916E02882381F081E0913009F007
:1084000080E09091D70C91111FC02FEE36E301E070
:1084100048EE5BE0672D0E943E557394639485E0BF
:1084200078129BCF7092A90DE2C083E068120FC052
:108430008091AD0D833009F059C08091A80D109244
:10844000A80D811140C052C026EF36E3E0CF84E092
:108450006812E3CF8091AD0D843009F092C0809115
:10846000A80D1092A80D81115DC08BC0C12CD12C1C
:10847000E12CF12C02E813E420E030E0A90165E3EF
:1084800072E081EE9BE00E94A6F68091CF0D8111F3
:10849000AEC080916E02882309F4BFCF11E08091B5
:1084A000AD0D823009F010E0609135027091360216
:1084B00080913702909138020E94C64B00E09C01E7
:1084C00041EE5BE02CC0C12CD12CE12CF12C02E858
:1084D00013E420E030E0A90161E372E08AED9BE063
:1084E0000E94A6F68091CF0D811181C080916E020D
:1084F000882309F492CF11E08091AD0D833009F00B
:1085000010E06091310270913202809133029091BB
:1085100034020E94C64B00E09C014AED5BE0672DEF
:10852000812F79CF20E030E048EC52E460912D02B9
:1085300070912E0280912F02909130020F947C4016
:1085400020E030E0A9010F942C470F949F48812C24
:10855000912C80E5A82E81E0B82E6B0118EEE12E5B
:1085600013E0F12E00E010E020E030E0A9016DE220
:1085700072E08FEC9BE00F94240A8091CF0D811163
:1085800036C080916E02882309F447CF11E08091B4
:10859000AD0D843009F010E0C0902D02D0902E0275
:1085A000E0902F02F090300220E030E0A901C701F6
:1085B000B6010F94164087FD05C02DEB37E346E06A
:1085C00055E304C02DEB37E346E055EBC701B60198
:1085D0000F942C4769837A838B839C83CE01019609
:1085E0000E94C3CF00E09C014FEC5BE098CF0F905E
:1085F0000F900F900F90DF91CF911F910F91FF90EF
:10860000EF90DF90CF90BF90AF909F908F907F9032
:108610006F905F900895CF93DF9300D01F92CDB7F6
:10862000DEB70F949F480F941B4069837A838B8336
:108630009C83CE0101960E94F5CC0F900F900F9075
:108640000F90DF91CF9108958F929F92AF92BF923A
:10865000CF92DF92EF92FF92CF936B017C0120E0EB
:1086600030E0A9010F94164087FD05C06DEB77E35C
:1086700086E095E304C06DEB77E386E095EBA70118
:1086800096010F942C476B017C0120E030E0A9019A
:108690000F94164087FF1BC0C701B601905820E019
:1086A00030E040E251E40F947C4020E030E040E2D2
:1086B00051E40F947C404B015C0120E030E0A901C3
:1086C000C701B6010F948C491816FCF019C020E0C0
:1086D00030E040E251E4C701B6010F947C4020E055
:1086E00030E040E251E40F947C404B015C0120E01B
:1086F00030E0A901C701B6010F94164087FD05C0FF
:1087000060E070E080EA90E404C060E070E080EA3D
:1087100090ECA50194010F942C4720E030E040E25A
:1087200051E40F9426480F9498486B017C0180E235
:1087300080933B0D80E1C81687E2D806E104F1047E
:1087400094F0C701B60120E137E240E050E00F9419
:108750008E46CA01B9012AE030E040E050E00F94B3
:108760008E46605D01C060E260933C0D88EEC816E5
:1087700083E0D806E104F10494F0C701B60128EEC5
:1087800033E040E050E00F948E46CA01B9012AE080
:1087900030E040E050E00F948E46605D01C060E242
:1087A00060933D0D84E6C816D104E104F10494F011
:1087B000C701B60124E630E040E050E00F948E4659
:1087C000CA01B9012AE030E040E050E00F948E4643
:1087D000605D01C060E260933E0D8AE0882E912CBE
:1087E000A12CB12CC701B601A50194010F948E46AE
:1087F000C62FCA01B901A50194010F948E46605D90
:1088000060933F0D8EE28093400DC05DC093410D9B
:108810008BE39DE0CF91FF90EF90DF90CF90BF90E2
:10882000AF909F908F900895CF92DF92EF92FF923A
:10883000CF93DF9300D01F92CDB7DEB76B017C01E1
:1088400020E030E0A9010F94164087FD05C06DEBD4
:1088500077E386E095E304C06DEB77E386E095EB84
:10886000A70196010F942C4769837A838B839C839D
:10887000CE0101960E94F5CC0F900F900F900F90B3
:10888000DF91CF91FF90EF90DF90CF9008954F92BE
:108890005F926F927F928F929F92AF92BF92CF9290
:1088A000DF92EF92FF920F931F93CF93DF9300D04D
:1088B00000D0CDB7DEB7C090790CD0907A0CE090A4
:1088C0007B0CF0907C0C80917D0C90917E0CA091A3
:1088D0007F0CB091800C8C159D05AE05BF0510F482
:1088E000D701C601C090750CD090760CE090770C43
:1088F000F090780CBC01CD016C157D058E059F05AF
:1089000010F4C701B6010F941B402B013C0161E03C
:1089100081E00E94254C2091AE0D2E831D828E8118
:1089200081110BC08091AD0D81112CC08091A80DDB
:108930001092A80D811120C025C02E81213061F434
:108940008091AD0D813009F08DC08091A80D1092FD
:10895000A80D811129C086C08E81823009F0ABC07C
:108960008091AD0D823009F01FC18091A80D109249
:10897000A80D8111BFC018C10E94464D8091CF0D36
:1089800081118BC280916E02882309F487C081E037
:108990009091AD0D911180E004E024E04EED56E39E
:1089A0006D810E943B537AC00E9448F72AE037ED60
:1089B00043E25DE3C301B2010F947C4020E030E06C
:1089C000A9010F942C474B015C0120E030E040E00E
:1089D0005FE40F94164087FD05C0812C912CA12CDB
:1089E0005FE4B52E2AE037ED43E25DE36091A90C28
:1089F0007091AA0C8091AB0C9091AC0C0F947C40C0
:108A000020E030E0A9010F942C4720E030E040E85E
:108A10005FE30F942B470F949F4869837A838B837E
:108A20009C83C501B4010F9498487B018C0121E01F
:108A3000E21AF10801091109812C912C40EFA42EB2
:108A400041E0B42EC980DA8021E030E040E050E01F
:108A500069EA7CE081E89DE30F94240A8091CF0DC0
:108A600081111BC280916E028823C1F011E08091B8
:108A7000AD0D813009F010E06091A90C7091AA0C45
:108A80008091AB0C9091AC0C0E94144400E09C01CE
:108A900041E85DE36D81812F0E943E558D818F5F9E
:108AA0008D832E812F5F2E83853009F038CF88E0AB
:108AB0008093A90DF2C18E81833061F48091AD0D58
:108AC000833009F0F9C08091A80D1092A80D811192
:108AD00095C0F2C02E81243009F080C08091AD0D88
:108AE000843009F024C18091A80D1092A80D811145
:108AF0000CC11DC10E9448F76091810C7091820CDD
:108B00008091830C9091840C0F941B4020E030E006
:108B1000A9010F942C474B015C0120E030E040E0BC
:108B20005FE40F94164087FD05C0812C912CA12C89
:108B30003FE4B32E20E030E0A9016091AD0C7091CC
:108B4000AE0C8091AF0C9091B00C0F942C4720E0AC
:108B500030E048EC52E40F942B470F949F48698310
:108B60007A838B839C83C501B4010F9498487B0161
:108B70008C0124E6E21AF10801091109812C912CDB
:108B800026EDA22E21E0B22EC980DA8024E630E064
:108B900040E050E06DEA7CE088E49CE00F94240A19
:108BA0008091CF0D811179C180916E02882309F4E3
:108BB00075CF11E08091AD0D823009F010E0609129
:108BC000AD0C7091AE0C8091AF0C9091B00C0E94E6
:108BD000144400E09C0148E45CE05CCF8E81853069
:108BE00009F084C08091AD0D853009F0DEC0809120
:108BF000A80D1092A80D8111C6C0D7C00E9448F7D9
:108C00002AE037ED43E25DE3C301B2010F947C40FB
:108C100020E030E0A9010F942C474B015C0120E0DB
:108C200030E040E05FE40F94164087FD05C0812CE2
:108C3000912CA12C9FE4B92E2AE037ED43E25DE3AD
:108C40006091B10C7091B20C8091B30C9091B40C06
:108C50000F947C4020E030E0A9010F942C4720E0E5
:108C600030E040E85FE30F942B470F949F486983FF
:108C70007A838B839C83C501B4010F9498487B0150
:108C80008C0121E0E21AF10801091109812C912CD3
:108C900080EFA82E81E0B82EC980DA8021E030E094
:108CA00040E050E061EB7CE08DE39CE00F94240A0F
:108CB0008091CF0D8111F1C080916E02882309F45B
:108CC000EDCE11E08091AD0D833009F010E06091A0
:108CD000B10C7091B20C8091B30C9091B40C0E94C5
:108CE000144400E09C014DE35CE0D4CE2E8126309C
:108CF000D1F58091AD0D863009F085C08091A80D29
:108D00001092A80D81116DC07EC00E9448F705EC3D
:108D10001FE324E630E040E050E065E77CE086E3D6
:108D20009CE00F9437388091CF0D8111B6C08091AF
:108D30006E02882309F4B2CE11E08091AD0D84302B
:108D400009F010E06091750C7091760C8091770CB1
:108D50009091780C0F941B400E940B4300E09C0103
:108D600046E35CE097CE8E81873009F097CE809104
:108D7000AD0D873009F075C08091A80D1092A80D37
:108D800081115DC06EC00E9448F70BEC1FE324E622
:108D900030E040E050E069E77CE08FE29CE00F9437
:108DA00037388091CF0D811178C080916E02882371
:108DB00009F474CE11E08091AD0D853009F010E01A
:108DC0006091790C70917A0C80917B0C90917C0C65
:108DD0000F941B400E940B4300E09C014FE25CE0BB
:108DE00059CE0E9448F709EC1FE32AE030E040E04A
:108DF00050E06DE77CE088E29CE00F94373880918A
:108E0000CF0D81114AC080916E02882309F446CEAD
:108E100011E08091AD0D863009F010E060917D0C7D
:108E200070917E0C80917F0C9091800C0F941B4070
:108E30000E940B4300E09C0148E25CE02BCE0E94C4
:108E400048F707EC1FE324E630E040E050E061E83B
:108E50007CE081E29CE00F9437388091CF0D811146
:108E60001CC080916E02882309F418CE11E0809115
:108E7000AD0D873009F010E06091810C7091820C8B
:108E80008091830C9091840C0F941B400E940B43A3
:108E900000E09C0141E25CE0FDCD26960FB6F8941F
:108EA000DEBF0FBECDBFDF91CF911F910F91FF901D
:108EB000EF90DF90CF90BF90AF909F908F907F907A
:108EC0006F905F904F900895CF92DF92EF92FF9254
:108ED000CF93DF9300D01F92CDB7DEB76B017C013B
:108EE00020E030E0A9010F94164087FD05C06DEB2E
:108EF00077E386E095E304C06DEB77E386E095EBDE
:108F0000A70196010F942C4769837A838B839C83F6
:108F100060E2CE0101960E94A1CD0F900F900F90BC
:108F20000F90DF91CF91FF90EF90DF90CF90089559
:108F30006F927F928F929F92AF92BF92CF92DF9269
:108F4000EF92FF920F931F93CF93DF9361E081E045
:108F50000E94254CC091AE0D712C53E0652EC111BD
:108F60000BC08091AD0D81111BC08091A80D109296
:108F7000A80D81110FC014C0C13011F58091AD0D45
:108F8000813009F0C2C08091A80D1092A80D811106
:108F9000AFC0BBC00E94464D8091CF0D811128C14A
:108FA00080916E02882361F081E09091AD0D911166
:108FB00080E004E024E04EED56E3672D0E943B5331
:108FC0008091510E882371F0C23071F48091AD0D03
:108FD000823009F0EFC08091A80D1092A80D811188
:108FE000AFC0E8C0D2E001C0D3E0DC133AC080914A
:108FF000AD0D8D131BC08091A80D1092A80D882374
:10900000A9F00E9448F7C12CD12CE12CF12C08E4E6
:1090100013E420E030E0A90165E074E08BEA9BE016
:109020000E94A6F68091CF0D8111E2C080916E0260
:109030008823B9F011E08091AD0D8C1310E06091A0
:1090400005047091060480910704909108040E9421
:10905000C64B00E09C014BEA5BE0672D812F0E942C
:109060003E5581E08D0F8C133AC08091AD0D8C136D
:109070001BC08091A80D1092A80D8823A9F00E9412
:1090800048F7C12CD12CE12CF12C08E413E420E0AA
:1090900030E0A90169E074E080EA9BE00E94A6F656
:1090A0008091CF0D8111A4C080916E028823B9F008
:1090B00011E08091AD0D8C1310E060910904709166
:1090C0000A0480910B0490910C040E94C64B00E0AE
:1090D0009C0140EA5BE0672D812F0E943E5573940E
:1090E000CF5F85E078123BCFDE5FD093A90D80C0C3
:1090F0008091510E8C278093510E60926E020E94D7
:10910000C9808091CF0D811173C080916E02882338
:1091100009F456CF81E09091AD0D913009F080E0D7
:109120009091510E911103C02FEE36E302C026EF4D
:1091300036E301E045EC5BE0672D0E943E5540CFF1
:109140000E9448F720E030E04AE754E460914D0E79
:1091500070914E0E80914F0E9091500E0F947C4066
:1091600020E030E0A9010F942C4720E030E84BEBE1
:1091700054E40F942B470F949F4829EC822E20E84B
:10918000922E32E1A32E31E0B32E6B0116EDE12ECB
:1091900016E0F12E00E010E02CED35E040E050E06C
:1091A0006DE47EE086EB9BE00F94240A8091CF0D66
:1091B00081111EC080916E028823C1F0D1E08091A0
:1091C000AD0D823009F0D0E060914D0E70914E0EE1
:1091D00080914F0E9091500E0E94644700E09C01D8
:1091E00046EB5BE0672D8D2F0E943E55D3E039CFD3
:1091F000DF91CF911F910F91FF90EF90DF90CF9073
:10920000BF90AF909F908F907F906F900895FC01DA
:1092100084910895FC01808108959091410E81E030
:1092200089270C94D7F280916E02882351F06091C7
:10923000380D7091390D20E030E041E081E00C9470
:109240003B540895BF92CF92DF92EF92FF920F931B
:109250001F93CF93DF936B0189014A3009F49DC0BE
:10926000453109F06EC0DB011296ED91FC91139728
:10927000F280C681D78180910201809582708093AF
:10928000000188E28A950000E9F720E1B22EBF0CC8
:1092900038E2E32E88EF0E9411528E2D8A9500004D
:1092A000E9F7BFE1BF1508F45EC08F2D80778068B5
:1092B0000E9411528F2D8295807F0E9411528E2D17
:1092C0008A950000E9F780E80E94115280E00E9430
:1092D00011528E2D8A950000E9F78AEF0E941152F3
:1092E0008E2D8A950000E9F78E01005F1F4F88815F
:1092F000807F0E94115289918295807F0E94115235
:10930000C017D107A1F78E2D8A950000E9F7F394D5
:10931000BF10C0CF80910201827080930001F601DE
:10932000C281D381CE010E94B88C8111D3C1DF915B
:10933000CF911F910F91FF90EF90DF90CF90BF9052
:109340000895DB011296CD91DC911397842F90E064
:10935000FC017497E433F105F0F48827EE58FF4FD1
:109360008F4F0D94114710EE1F0D1068812F807FD5
:109370000E941152812F8295807F0E9411528E2D62
:109380008A950000E9F780E80E94115280E89FCF9B
:109390008981F901808381E0CACF809101018260D7
:1093A000809301018091020182708093000180917D
:1093B000010181608093010180910201817080939D
:1093C0000001099A119A8091020180958270809320
:1093D000000188E28A950000E9F788E790E02EE92D
:1093E0003FE0CEE9DFE0F9013197F1F70197C9F7E6
:1093F00088EF0E94115218E2812F8A950000E9F748
:1094000080E20E94115280E00E941152812F8A95C1
:109410000000E9F780E00E94115280E80E9411529A
:10942000812F8A950000E9F780E00E94115280E1C7
:109430000E941152812F8A950000E9F7CE01019711
:10944000F1F7CE010197F1F7CE010197F1F7CE01C7
:109450000197F1F7CE010197F1F7CE010197F1F7EE
:10946000CE010197F1F7CE010197F1F7CE010197F7
:10947000F1F7CE010197F1F7CE010197F1F7CE0197
:109480000197F1F7CE010197F1F7CE010197F1F7BE
:109490002197F1F780E20E94115280E40E9411525C
:1094A000812F8A950000E9F780E20E94115280E640
:1094B0000E9411521A950000E9F7D0E0C8E218E2C4
:1094C0008D2F807780680E9411528D2F8295807F2A
:1094D0000E9411528C2F8A950000E9F780E80E94C3
:1094E000115280E00E9411528C2F8A950000E9F7FA
:1094F0008AEF0E9411528C2F8A950000E9F790E2C2
:10950000119880910201817080930001119A0000EE
:10951000119880910201817080930001119A0000DE
:10952000119880910201817080930001119A0000CE
:10953000119880910201817080930001119A0000BE
:10954000119880910201817080930001119A0000AE
:10955000119880910201817080930001119A00009E
:10956000119880910201817080930001119A00008E
:10957000119880910201817080930001119A00007E
:10958000119880910201817080930001119A00006E
:10959000119880910201817080930001119A00005E
:1095A000119880910201817080930001119A00004E
:1095B000119880910201817080930001119A00003E
:1095C000119880910201817080930001119A00002E
:1095D000119880910201817080930001119A00001E
:1095E000119880910201817080930001119A00000E
:1095F000119880910201817080930001119A0000FE
:109600008C2F8A950000E9F7915009F079CF88EF07
:109610000E941152812F8A950000E9F7DF5FD03256
:1096200009F04ECF80E00E94115280EC0E9411524E
:1096300088E28A950000E9F78091020182708093A8
:10964000000181E074CE4D8150E0440F551F60E071
:1096500070E08E819F810F94614ACE010E94CE8C72
:1096600081E065CEF90181819381913009F46EC06A
:10967000933009F040C048EF480F91E02B81241748
:1096800008F490E021E03A81831708F420E031E00B
:10969000841708F030E0492F432B242319F4932337
:1096A00009F479CED8011296FC90EE24EA94D12CDC
:1096B00044C0B901CE010E94D58C81E038CEF901B9
:1096C00010828A8181838D81815082838B81838303
:1096D00081E02DCE4D8150E0440F551F60E070E0D9
:1096E0008E819F810F94614A81E021CE8D81D901C5
:1096F0008C9381E01CCE2B81281708F44CCE2A8154
:10970000821708F448CEF2809130C9F1D8F1923036
:10971000B9F4E12CDD24DA9410C0B801CE010E9426
:10972000D58CF8018181D8019C919D0D9C938E0D63
:1097300011968C93FF0C09F42ECEF7FEF4CFEDCFEB
:10974000933009F4B2CFE12CD12CF7CF48E0480F89
:1097500091E02B81281708F490E021E03A8143172B
:1097600008F420E031E0481708F030E0492F432B9F
:10977000242319F4932309F40ECEF801F280EE2489
:10978000E39495CFE12CDD24D394D7CFCF92DF9211
:10979000EF92FF926B017C0120E030E0A9010F9471
:1097A000164087FD05C06DEB77E386E095E304C0C6
:1097B0006DEB77E386E095EBA70196010F942C47BC
:1097C0006B017C0120E030E0A9010F94164087FD79
:1097D00005C020E030E040E05FE304C020E030E07E
:1097E00040E05FEBC701B6010F942C470F949848F7
:1097F000CB01FF90EF90DF90CF900C940ED10F93A0
:10980000CF93DF93CDB7DEB700E22EE349855A85CB
:1098100068858F810E943B53DF91CF910F9108950E
:1098200063E972E084E690E00E9417D66AEB72E08A
:1098300084E690E00C9417D681110C94104C68EBE0
:1098400071E084E190E00C9417D6282F1092B90DA6
:109850008091BF0D9091C00DA091C10DB091C20D2E
:10986000B7FF08C01092BF0D1092C00D1092C10D2D
:109870001092C20D8091C203882331F08091BF0DF8
:109880008093AD0D1092CF0D8091A90D1816FCF4A8
:10989000082E000C990B821B91092091AD0D022E10
:1098A000000C330B2817390794F097FF02C080E0B3
:1098B00090E08093AD0D092E000CAA0BBB0B80939A
:1098C000BF0D9093C00DA093C10DB093C20D8091B8
:1098D000AD0D6623A9F09091AE0D891714F4809315
:1098E000AE0D2091AE0D022E000C330B2C5F3F4FBE
:1098F000482F082E000C550B241735071CF48450F4
:109900008093AE0D08958091931190919411891BCD
:109910008F7011F40C948C3681E008958F929F9291
:10992000AF92BF92CF92DF92EF92FF920F931F936D
:10993000CF93DF93EC01042F122F8091D5119091DA
:10994000D6118C179D0709F48CC02091C10327FD07
:109950001092C1036B01E12CF12C20E6CC34D2072C
:10996000A1F48C569F46B9F50E947BFADC01CB012D
:109970008E519B4FAF4FBF4F8093B5039093B6036B
:10998000A093B703B093B80326C02FE6CC36D20716
:1099900009F043C08C54904609F050C00E947BFAF5
:1099A0008090B5039090B603A090B703B090B80331
:1099B000DC01CB0188199909AA09BB09B7FF3EC090
:1099C0008091DA048770873031F40E94834C8823B9
:1099D00011F0C6E3DDE8D093D611C093D511C09243
:1099E000BF0DD092C00DE092C10DF092C20D009358
:1099F000AE0D1093A90DCC56DF4621F410923A0D0E
:109A00001092B40382E080936E0281E08093CF0DC8
:109A10001092C3031092FE1424C0D093D611C093A9
:109A2000D511C092BF0DD092C00DE092C10DF09241
:109A3000C20D0093AE0D1093A90DE4CF8CE69FE606
:109A40009093D6118093D511C092BF0DD092C00DC6
:109A5000E092C10DF092C20D0093AE0D1093A90DCE
:109A6000CDCFDF91CF911F910F91FF90EF90DF90BD
:109A7000CF90BF90AF909F908F90089520E040E0EE
:109A800060E070E08CE69FE60C948E4CE091B403AD
:109A9000EE2389F0E150E093B40388E0E89FF00101
:109AA0001124EC57FC4F62817381278146818081AC
:109AB00091810C948E4C0C943E4D0F931F93CF9339
:109AC000DF93FC01EB018091BF0D9091C00DA0913F
:109AD000C10DB091C20DB7FF08C01092BF0D10921A
:109AE000C00D1092C10D1092C20D8091C30D9091C6
:109AF000C40DA091C50DB091C60D4091BF0D509100
:109B0000C00D6091C10D7091C20D84179507A60715
:109B1000B70744F48093BF0D9093C00DA093C10D7F
:109B2000B093C20D80916E02882301F14091BF0D68
:109B30005091C00D6091C10D7091C20D8091C70D03
:109B40009091C80DA091C90DB091CA0D8A019B01D9
:109B5000080F191F2A1F3B1FC901B8011995BC0125
:109B60008091CD0D9091CE0D0E94B9548091A80D99
:109B7000811108C08091BC0D8823D1F180916E02C3
:109B80008823B1F18091CB0D9091CC0D0097B1F06D
:109B90000091BF0D1091C00D2091C10D3091C20DEB
:109BA0004091C70D5091C80D6091C90D7091CA0DBB
:109BB000400F511F621F731FFE011995E091BD0DEB
:109BC000F091BE0D309741F08091BC0D811103C022
:109BD0008091A80D811119958091A80D1092A80D62
:109BE000882331F0DF91CF911F910F910C94464D56
:109BF000DF91CF911F910F910895E091B403E6306A
:109C000010F581E08E0F8093B4034091BF0D509109
:109C1000C00D6091C10D7091C20D9091AE0D8091FB
:109C2000A90D28E0E29FF0011124EC57FC4F209190
:109C3000D5113091D61131832083428353836483BD
:109C4000758396838783089510923A0D0C94464D40
:109C5000AF92BF92CF92DF92EF92FF920F931F933A
:109C6000CF93DF93EC015B018A01FB01199587FD1E
:109C700005C090E0A0E0B0E0219628C1982F907E2A
:109C8000903CC9F48F7190E0A0E0B0E06C017D01E0
:109C900026E0CC0CDD1CEE1CFF1C2A95D1F7CE0172
:109CA0000196F50119958F73A7019601282BDA010A
:109CB000C90122960BC1982F907F903E29F58F7095
:109CC000C82ED12CE12CF12C86E0CC0CDD1CEE1C36
:109CD000FF1C8A95D1F7CE010196F50119958F7376
:109CE000C82A96E0CC0CDD1CEE1CFF1C9A95D1F71F
:109CF000CE010296F50119958F73A7019601282BC5
:109D0000DA01C9012396E2C0982F987F903F91F520
:109D10008770C82ED12CE12CF12CF6E0CC0CDD1C88
:109D2000EE1CFF1CFA95D1F7CE010196F5011995AD
:109D30008F73C82AA6E0CC0CDD1CEE1CFF1CAA9574
:109D4000D1F7CE010296F50119958F73C82AB6E0B6
:109D5000CC0CDD1CEE1CFF1CBA95D1F7CE0103968E
:109D6000F50119958F73A7019601282BDA01C90116
:109D70002496ACC0982F9C7F983F09F03FC0837019
:109D8000C82ED12CE12CF12C56E0CC0CDD1CEE1CA5
:109D9000FF1C5A95D1F7CE010196F50119958F73E5
:109DA000C82A66E0CC0CDD1CEE1CFF1C6A95D1F7BE
:109DB000CE010296F50119958F73C82A76E0CC0C76
:109DC000DD1CEE1CFF1C7A95D1F7CE010396F50140
:109DD00019958F73C82AE6E0CC0CDD1CEE1CFF1C25
:109DE000EA95D1F7CE010496F50119958F73A70175
:109DF0009601282BDA01C901259668C0982F9E7F0D
:109E00009C3F09F04CC08170C82ED12CE12CF12C64
:109E100086E0CC0CDD1CEE1CFF1C8A95D1F7CE0130
:109E20000196F50119958F73C82A96E0CC0CDD1CBC
:109E3000EE1CFF1C9A95D1F7CE010296F5011995FB
:109E40008F73C82A26E0CC0CDD1CEE1CFF1C2A9563
:109E5000D1F7CE010396F50119958F73C82A36E024
:109E6000CC0CDD1CEE1CFF1C3A95D1F7CE010496FC
:109E7000F50119958F73C82A46E0CC0CDD1CEE1C49
:109E8000FF1C4A95D1F7CE010596F50119958F7300
:109E9000A7019601282BDA01C901269617C0982F31
:109EA000907C903841F4807C803869F42196CE0112
:109EB000F5011995F8CF8E7F8D3F28F02196CE01C0
:109EC000F5011995F8CF80E090E0DC01011511054E
:109ED00029F0F80180839183A283B383CE01DF91BF
:109EE000CF911F910F91FF90EF90DF90CF90BF9097
:109EF000AF9008956F927F928F929F92AF92BF9290
:109F0000CF92DF92EF92FF920F931F93CF93DF9345
:109F100000D01F92CDB7DEB7862E6A01122F2EEF2A
:109F2000621305C038E5A32E3CE0B32E04C024E83C
:109F3000A22E22E4B22E082F992E86E0E82EF12CD4
:109F40009AE0792E11160CF08DC0AE014F5F5F4F75
:109F500067E079E4802F992D0E94284E082F992ED2
:109F600069817A818B819C816115710581059105DB
:109F700009F478C06D3371058105910509F45BC062
:109F80006E3771058105910509F455C06A32710576
:109F900081059105C1F0643271058105910579F45F
:109FA000C114D10461F086E01802B0011124C60189
:109FB0000E947B53B7010F94FD46161BC3CF0E942E
:109FC000CA521150BFCF87FC38C065E470E080E012
:109FD00090E00E94CA52115009F443C061E08981A7
:109FE0009A81AB81BC81CD97A105B10509F460E0F0
:109FF000862F880D8A3094F0672D0F94DB46692EEA
:10A00000682F880F770B605D7F4F072E000C880B41
:10A01000990B0E94CA52115021F1862D682F880F8A
:10A02000770B605D7F4F072E000C880B990B0E9409
:10A03000CA5211500DC087FED1CF86E01802B00180
:10A040001124C5010E947B53B7010F94FD46161BD6
:10A05000112339F026E01202B0011124802F992D2E
:10A06000A7CF10E0812F0F900F900F900F90DF91EE
:10A07000CF911F910F91FF90EF90DF90CF90BF9005
:10A08000AF909F908F907F906F9008951F93CF9384
:10A09000DF9300D01F92CDB7DEB710E0AE014F5F67
:10A0A0005F4F6AE079E40E94284E49815A816B81B2
:10A0B0007C81452B462B472B11F01F5FEFCF812F63
:10A0C0000F900F900F900F90DF91CF911F910895F7
:10A0D0001F93CF93DF9300D01F92CDB7DEB710E070
:10A0E000AE014F5F5F4F67E079E40E94284E4981DF
:10A0F0005A816B817C81452B462B472B11F01F5FCA
:10A10000EFCF812F0F900F900F900F90DF91CF9195
:10A110001F9108952F923F924F925F926F927F927C
:10A120008F929F92AF92BF92CF92DF92EF92FF9267
:10A130000F931F93CF93DF9300D0CDB7DEB74C01C1
:10A140003B015A012B83232E28014091BF0D5091D2
:10A15000C00D6091C10D7091C20D41155105610591
:10A16000710579F081E0141615060CF080E08093FB
:10A17000FE141092BF0D1092C00D1092C10D1092DE
:10A18000C20D1091FE143090A80D1092A80D311040
:10A1900005C080916E02882309F478C0C2010E9434
:10A1A0006850082FC114D10409F46EC0C6010E9482
:10A1B00068501A821982E114F104B1F4402F50E082
:10A1C000282F30E0CA01820F931F46976CF485E177
:10A1D00090E0841B950B821B930B97FD0196959540
:10A1E00087958A8381E0898301E027E039E4A20131
:10A1F000BE016F5F7F4FCE0102960E94BA8FE114BD
:10A20000F10491F08A81882321F01A8289818F5F7D
:10A21000898300E02AE039E4A701BE016F5F7F4F28
:10A22000CE0102960E94BA8FC114D10459F000E009
:10A2300027E039E4A601BE016F5F7F4FCE01029691
:10A240000E94BA8F41E04127B30181E00F948B094E
:10A25000C4010E946850412FB40194E1981B892FDA
:10A260000F948B09332061F0111102C0AB80B22C26
:10A27000A114B10419F0F501199502C00E94464DD0
:10A2800081E080933A0D02C080E093CF0F900F9051
:10A290000F90DF91CF911F910F91FF90EF90DF9082
:10A2A000CF90BF90AF909F908F907F906F905F9076
:10A2B0004F903F902F900895089580E090E008958A
:10A2C000DF92EF92FF920F931F93CF93DF93EC01F6
:10A2D000D62E1CAD0BAD7C0184E0E80EF11CE98D9F
:10A2E000FA8DC7011995412F480F2D2D602FC701F9
:10A2F0000E9418969BAD890F8BAF81E090E0DF91B3
:10A30000CF911F910F91FF90EF90DF9008959F9252
:10A31000AF92BF92CF92DF92EF92FF920F931F9373
:10A32000CF93DF93EC018B01942EC52E8A859B85FC
:10A330008617970731F0888199810E94C8941B87FE
:10A340000A8788859985019691F00E811F81692D74
:10A350007C2D888199810F943E09080F111D8885F5
:10A3600099858017910718F481E090E026C0DC8081
:10A370001A819E81190FA880B980D5015596ED915B
:10A38000FC915697C5011995D80EE92CFC2C00E0DC
:10A39000D7012D917D01222341F04D2D612FC50163
:10A3A0000E941896180F080FF3CF8E819F81800F9F
:10A3B000911D9F838E8380E090E0DF91CF911F916C
:10A3C0000F91FF90EF90DF90CF90BF90AF909F9054
:10A3D0000895EF92FF920F931F93CF93DF93EC01B9
:10A3E0008B017A018A859B858617970731F08881D2
:10A3F00099810E94C8941B870A87B7018881998137
:10A400000F943E092E813F81280F311D3F832E83FB
:10A4100080E090E0DF91CF911F910F91FF90EF903E
:10A42000089511989091020187FD64C091709093F6
:10A430000001119A0000119890910201382F330FFA
:10A4400086FD56C0917090930001119A00001198FA
:10A4500080910201232F220F36FD48C08170809326
:10A460000001119A0000119880910201922F990F1A
:10A4700026FD3AC0817080930001119A0000119866
:10A4800080910201292F220F96FD2CC081708093AC
:10A490000001119A0000119880910201922F990FEA
:10A4A00026FD1EC0817080930001119A0000119852
:10A4B00080910201292F220F96FD10C08170809398
:10A4C0000001119A000011988091020126FD8095EB
:10A4D000817080930001119A000008958095EECF5D
:10A4E0008095E0CF8095D2CF8095C4CF8095B6CFB0
:10A4F0009095A8CF90959ACF9CE0899F802D1124AC
:10A5000091E0980F9093670D2CE0280F2093660D33
:10A5100030E02E5F3F4F40910F1250E02417350777
:10A5200014F480E00895292F30E04091111250E09A
:10A5300024173507B4F7662341F08E5F0F94720934
:10A540008091660D8E5F0F9472098091660D9091D7
:10A550000F12891730F3209111129091670D29176E
:10A5600000F3109212128093131281E00895482F85
:10A5700050E02091BB03022E000C330B421753070F
:10A5800041F08093BB036BEE7DE08BED91E10C9489
:10A59000C8940895CF92DF92EF92FF920F931F938A
:10A5A000CF93DF93CDB7DEB72C970FB6F894DEBF0D
:10A5B0000FBECDBF6F3F71058105910509F060F4B5
:10A5C00087ED91E10E946051E091DF11F091E0117F
:10A5D0003196849190E040C0F0901212E0901312F6
:10A5E0002091C003211109C04BEC5DE06E2D8F2D31
:10A5F0000F94AE2E80E090E029C0C090DF11D09083
:10A60000E0112BED31E13A8329832F2D30E03C839B
:10A610002B832E2D30E03E832D8318861F822FEF53
:10A620003FEF3A8729871C861B8607E811E59E01C4
:10A630002F5F3F4FAB01BC01C6010F949B0EB601CB
:10A640008BED91E10E94C8948F819885F80EF0926D
:10A650001212E092131299272C960FB6F894DEBFCF
:10A660000FBECDBFDF91CF911F910F91FF90EF9063
:10A67000DF90CF9008950F93CF93DF93982F862F7D
:10A68000EA01692F0E947C52882389F14091AA0D2A
:10A690005091AB0D24E16091AC0DCE010E947A4F38
:10A6A00096E0899FE0011124C730D10548F060E2AF
:10A6B00070E080E090E00E94CA52C81BD90BF4CF32
:10A6C0008091660D9AE79093121280931312602F77
:10A6D000000F770B880B990B0E94CA5260E270E062
:10A6E00080E090E0DF91CF910F910C94CA52DF91FE
:10A6F000CF910F910895CF92DF92EF92FF920F9337
:10A700001F93CF93DF93CDB7DEB72C970FB6F89496
:10A71000DEBF0FBECDBFF0901212E0901312209159
:10A72000C003211109C04BEC5DE06E2D8F2D0F94FD
:10A73000AE2E80E090E028C0C090DF11D090E011F4
:10A740002BED31E13A8329832F2D30E03C832B839D
:10A750002E2D30E03E832D8318861F827A876987ED
:10A760001C861B8607E811E59E012F5F3F4F47E0DF
:10A7700059E4BC01C6010F94692EB6018BED91E13D
:10A780000E94C8948F819885F80EF0921212E09280
:10A79000131299272C960FB6F894DEBF0FBECDBFCB
:10A7A000DF91CF911F910F91FF90EF90DF90CF90AD
:10A7B00008956FEF7FEF0C947B53CF92DF92EF926F
:10A7C000FF920F931F93CF93DF93CDB7DEB72C97F4
:10A7D0000FB6F894DEBF0FBECDBFF0901212E0901E
:10A7E00013122091C003211109C04BEC5DE06E2DC6
:10A7F0008F2D0F94AE2E80E090E028C0C090DF1126
:10A80000D090E0112BED31E13A8329832F2D30E0F8
:10A810003C832B832E2D30E03E832D8318861F82B0
:10A820007A8769871C861B8607E811E59E012F5FE2
:10A830003F4F4AE059E4BC01C6010F94692EB601AE
:10A840008BED91E10E94C8948F819885F80EF0926B
:10A850001212E092131299272C960FB6F894DEBFCD
:10A860000FBECDBFDF91CF911F910F91FF90EF9061
:10A87000DF90CF900895BF92CF92DF92EF92FF9238
:10A880000F931F93CF93DF938B01F42EE90141FBCC
:10A89000662760F90E947C52882309F45CC0011588
:10A8A000110529F0C8010E946850B82E01C0B12CD2
:10A8B000209729F0CE010E944650E82E01C0E12CDD
:10A8C000F0FE1EC085E190E08B199109B7FC9395CD
:10A8D0008E199109E7FC939597FD019695958795BB
:10A8E000F82E30E8C32ED12CFA94F7FC0CC060E2AD
:10A8F00070E080E090E00E94CA52C81AD90AF4CFF2
:10A9000080E8C82ED12CBB2099F0C60166E070E02B
:10A910000F94E946262F4091AA0D5091AB0D6091FE
:10A92000AC0DC8010E947A4F96E0899F6001112406
:10A93000EE2031F0B601CE010E94DD53C81AD90ACB
:10A9400087E0C816D10438F060E270E080E090E063
:10A950000E94CA52F3CFDF91CF911F910F91FF90C8
:10A96000EF90DF90CF90BF9008956FEF7FEF0C9442
:10A97000DD53AF92BF92CF92DF92EF92FF920F938F
:10A980001F93CF93DF935C016B010E946850E82E08
:10A99000C6010E944650F12C03E110E0081B11098A
:10A9A0000E151F0514F0C5E201C0CFE18C2F90E019
:10A9B000AC014E5F5F4F20910F1230E042175307FA
:10A9C0003CF009972091111230E028173907DCF587
:10A9D000D0E0C114D10409F446C06AE370E080E01D
:10A9E00090E00E94CA520E151F0584F4C45F809146
:10A9F0000F12C817C0F12C2F30E029503109809177
:10AA0000111290E0821793071CF42DC0DD2359F139
:10AA1000802F880F080F000F00931212C09313129B
:10AA200060E270E080E090E00E94CA52C601DF91CF
:10AA3000CF911F910F91FF90EF90DF90CF90BF903B
:10AA4000AF900C94B5544091AA0D5091AB0D60910C
:10AA5000AC0D10921212C093131225E1C5010E9491
:10AA60007A4FD1E0B6CFDF91CF911F910F91FF9038
:10AA7000EF90DF90CF90BF90AF9008958F929F920C
:10AA8000AF92BF92CF92DF92EF92FF920F931F93FC
:10AA9000CF93DF93CDB7DEB72C970FB6F894DEBF18
:10AAA0000FBECDBF982F862F5A017901D02E692F66
:10AAB0000E947C52882309F488C0C701002361F0FA
:10AAC0000E946850C82E8090DF119090E011809114
:10AAD000C00381110EC00BC00E944650C82E80904A
:10AAE000DF119090E0118091C003811113C02FEF0E
:10AAF0002BC09E012F5F3F4F8CE0F90111928A9588
:10AB0000E9F78BED91E19A83898309EE11E547E03E
:10AB100059E410C09E012F5F3F4F8CE0F901119264
:10AB20008A95E9F78BED91E19A83898309EE11E526
:10AB30004AE059E4B701C4010F94692EB4018BEDCA
:10AB400091E10E94C8942F81122F23E12C1940918A
:10AB5000AA0D5091AB0D6091AC0DC5010E947A4FCA
:10AB6000CC2099F1F6E08F9F500111246AE370E048
:10AB700080E090E00E94CA5257E0A516B10448F068
:10AB800060E270E080E090E00E94CA52A81AB90A20
:10AB9000F3CF4091660D212F30E0E6E0CE9EC0015C
:10ABA00011242E5F3F4F281739070CF49C0180E8D1
:10ABB000821B8093121240931312C701DD2019F0FB
:10ABC0000E94D95302C00E94B5542C960FB6F89437
:10ABD000DEBF0FBECDBFDF91CF911F910F91FF90D0
:10ABE000EF90DF90CF90BF90AF909F908F9008959F
:10ABF000E7EDF1E183AF64AFCA010C94B554CF9295
:10AC0000DF92EF92FF926A017B010E94BBF08823E2
:10AC100031F0FF90EF90DF90CF900C943BF0C701A4
:10AC2000B601FF90EF90DF90CF9008952F923F9262
:10AC30004F925F926F927F928F929F92AF92BF924C
:10AC4000CF92DF92EF92FF920F931F93CF93DF93F8
:10AC5000CDB7DEB7E7970FB6F894DEBF0FBECDBF16
:10AC600060E070E085E40E94C8F08823E1F081EAAA
:10AC70009DE0E7960FB6F894DEBF0FBECDBFDF9123
:10AC8000CF911F910F91FF90EF90DF90CF90BF90E9
:10AC9000AF909F908F907F906F905F904F903F907C
:10ACA0002F900C942CF465E070E083E40E94C8F0CF
:10ACB0008EA360E085E50E94D7F08DAB40E050E0C8
:10ACC0006EE373E483E50E94FF556B017C0160E055
:10ACD00084E99DE00E94E2D6C701B6010F9498482E
:10ACE000072E000C880B990B0F941D40162F7D83A7
:10ACF0008E83292E0E947BFA2B013C016091210258
:10AD0000709122026F507109072E000C880B990B6D
:10AD10000F941D409B01AC01612F7D818E81922D8E
:10AD20000F948C4918162CF489E69DE00E942CF4AF
:10AD300027C2A3019201205C33464F4F5F4F29ABDE
:10AD40003AAB4BAB5CAB85E59DE00E942CF40E94D6
:10AD5000A5CB8FE78093390F81E0809323024D8A42
:10AD60005E8A6F8A788E48A659A66AA67BA68FE768
:10AD700090E0A0E0B0E08F839887A987BA871D8E06
:10AD80001E8E1F8E18A2198E1A8E1B8E1C8E812C61
:10AD9000912C54011D8690E49E87ACE1AF87B6E408
:10ADA000B88B198A1A8A1B8A1C8A1CA68DA69EA695
:10ADB000AFA6B8AAFFE7CF2ED12CE12CF12C1AA216
:10ADC0001BA21CA21DA221E029A31C861B86312CDC
:10ADD00000E01EAA1FAA4EA1042E000C550B5FA373
:10ADE0004EA380912302882309F4C8C10E947BFAF4
:10ADF00069837A838B839C838091D40C882309F4A4
:10AE000090C00E9458CC3090330F0091340F509175
:10AE1000350F5EAB8091360F8FAB29893A894B890C
:10AE20005C89632D702F8EA99FA90F948C491816E9
:10AE300034F4398A0A8B9EA99B8BAFA9AC8B2D85E4
:10AE40003E854F855889632D702F8EA99FA90F9439
:10AE5000164087FF06C03D860E87BEA9BF872FA973
:10AE6000288B39A1232D3323E9F1302F4EA95FA977
:10AE7000612F7D818E81922D0F94164087FF51C0E6
:10AE800049815A816B817C8144195509660977098A
:10AE9000DB01CA0188589341A109B109B7FD41C03E
:10AEA0008F819885A985BA858C199D09AE09BF093E
:10AEB000B595A795979587958093390F4AA35BA37E
:10AEC0006CA37DA3198B4D814A8B5E815B8B2C8A91
:10AED00089819A81AB81BC818D8B9E8BAF8BB88F22
:10AEE00019A21FC0302F4EA95FA9612F7D818E81CD
:10AEF000922D0F948C491816A4F489819A81AB8104
:10AF0000BC812D893E894F89588D821B930BA40BE0
:10AF1000B50BAC01BD01485853416109710977FF78
:10AF200049C120E030E040EF51E4612F7D818E8106
:10AF3000922D0F942C47232D302F4EA95FA90F94EB
:10AF4000164087FF03C089E69DE0A8C089819A81E9
:10AF5000AB81BC8128A539A54AA55BA5821B930BB3
:10AF6000A40BB50BB7FD7EC080E00E943CC68AE012
:10AF70000E94273889819A81AB81BC818053984F88
:10AF8000AF4FBF4F88A799A7AAA7BBA79CA59111B0
:10AF90004EC02DA53EA54FA558A9632D702F8EA993
:10AFA0009FA90F948C4918167CF520E030E040E012
:10AFB00050E4632D702F8EA99FA90F942C476DA785
:10AFC0007EA78FA798AB29813A814B815C81205C59
:10AFD00033464F4F5F4F29AB3AAB4BAB5CAB20E0F6
:10AFE00030E040EE50E4612F7D818E81922D0F94F0
:10AFF0002B47232D302F4EA95FA90F941640881F91
:10B000008827881F8CA72EC089819A81AB81BC813B
:10B0100029A93AA94BA95CA9821B930BA40BB50BD8
:10B02000B7FD20C047EB52E466EC72E418C020E0A4
:10B0300030E040EF51E4612F7D818E81922D0F949D
:10B040002B479B01AC01632D702F8EA99FA90F94F4
:10B05000164087FF07C043EF52E461E073E480E0ED
:10B060000F943F2A8D899E89AF89B88D481659065D
:10B070006A067B0610F4D301C20129813A814B8113
:10B080005C81281B390B4A0B5B0BDA01C901813843
:10B090009F44A241B10528F08EEE9CE00E942CF462
:10B0A0006DC04EA15FA18B859C85481759070CF098
:10B0B00062C003970CF45FC081E99CE00E942CF40D
:10B0C00084E79CE00E942CF4B501A4018DE89CE08B
:10B0D0000E94FFF48AE00E94273884E79CE00E94E7
:10B0E0002CF4498D5A8D6B8D7C8D89E89CE00E94F3
:10B0F000FFF48AE00E94273884E79CE00E942CF449
:10B100004D8D5E8D6F8D78A185E89CE00E94FFF4E7
:10B110008AE00E9427389DA9992391F180923A0FE5
:10B1200090923B0FA0923C0FB0923D0F2CEA35EC71
:10B1300047E25EE3698D7A8D8B8D9C8D0F947C4008
:10B1400060933E0F70933F0F8093400F9093410F99
:10B150002CEA35EC47E25EE36D8D7E8D8F8D98A1F4
:10B160000F9426486093420F7093430F8093440FCF
:10B170009093450F05C00E944E6C33CE0E94A5CB24
:10B18000E7960FB6F894DEBF0FBECDBFDF91CF912B
:10B190001F910F91FF90EF90DF90CF90BF90AF90F5
:10B1A0009F908F907F906F905F904F903F902F90E7
:10B1B0000D94CB054B855C85452B09F407C14AA04E
:10B1C0005BA06CA07DA0480E591E6A1E7B1E2AA1A2
:10B1D0003BA14CA15DA1281B390B4A0B5B0BC7019E
:10B1E000B6010F945C46A30192010F948E46CF8066
:10B1F000D884E984FA84C20ED31EE41EF51E54E1FD
:10B20000C516D104E104F1040CF18CEEC816D1048A
:10B21000E104F1043CF490E8C916D104E104F1041E
:10B2200034F422C04BEEC42ED12CE12CF12CCF8271
:10B23000D886E986FA862EEF30E040E050E02C19FF
:10B240003D094E095F0969017A0112C084E190E06D
:10B25000A0E0B0E08F839887A987BA8734E1C32E36
:10B26000D12CE12CF12C04C0CF82D886E986FA8655
:10B270008DE49DE00E942CF46F81788589859A8504
:10B280000E949B3888E49DE00E942CF4C701B6011F
:10B290000E949B384D855E856F85788981E49DE0AD
:10B2A0000E94FFF449895A896B897C898AE39DE071
:10B2B0000E94FFF4AB85BC8513970CF487C0C701CF
:10B2C000B6010F941D4020E030E040E850E40F94B8
:10B2D0007C404B015C012D853E854F8558896989ED
:10B2E0007A898B899C890F942B472BED3FE049E4A9
:10B2F00050E40F947C4020E030E040E05FE30F94A6
:10B300007C409B01AC01C501B4010F9426484B0160
:10B310005C01C301B2010F941D402FE632E143E806
:10B320005AE30F947C402B013C01B501A40184E356
:10B330009DE00E94FFF4B301A2018EE29DE00E9415
:10B34000FFF42AE939E949E15FE3C501B4010F944B
:10B350007C404B015C019B01AC01C301B2010F9425
:10B360007C4020E030E040E05EE30F947C406D8F55
:10B370007E8F8F8F98A3A5019401C501B4010F940E
:10B380002C47A30192010F942648698F7A8F8B8FE7
:10B390009C8F8CE09DE00E942CF4B501A40188E212
:10B3A0009DE00E94FFF4498D5A8D6B8D7C8D82E269
:10B3B0009DE00E94FFF44D8D5E8D6F8D78A18CE134
:10B3C0009DE00E94FFF48AE00E9427388F819885D3
:10B3D000A985BA858C0D9D1DAE1DBF1DB595A79580
:10B3E000979587958093390F2B853C852F5F3F4F2D
:10B3F0003C872B871D873D813E874E814F87288A5A
:10B4000049805A806B807C8051E059A38ACD2F926D
:10B410003F924F925F926F927F928F929F92AF92E4
:10B42000BF92CF92DF92EF92FF920F931F93CF9331
:10B43000DF93D62FC72FFC0180809180A280B3803C
:10B44000C501B40120E831E541E050E00F946C46BD
:10B45000C9016DE671E00F94E9466B017C01C501FD
:10B46000B40120E13EE040E050E00F946C46CA0198
:10B47000B90128E130E040E050E00F946C46362EF0
:10B48000272E062F172F8CE3482E512C612C712C60
:10B49000C501B401A30192010F946C46B62EA72EEC
:10B4A000CA01B901A30192010F946C46CB01C114EA
:10B4B000D104D9F0AF92BF927F936F932F923F92B6
:10B4C000FF92EF92DF92CF9280E69CE09F938F9362
:10B4D000CF93DF930F94AE3F8DB79EB70E960FB606
:10B4E000F8949EBF0FBE8DBF5CC0E114F104C9F09B
:10B4F000AF92BF927F936F932F923F92FF92EF9202
:10B5000084E69CE09F938F93CF93DF930F94AE3F9D
:10B51000EDB7FEB73C960FB6F894FEBF0FBEEDBF79
:10B5200040C0012BB9F0AF92BF927F936F932F92DF
:10B530003F9288E69CE09F938F93CF93DF930F9485
:10B54000AE3F8DB79EB70A960FB6F8949EBF0FBE5A
:10B550008DBF27C0892BA9F0AF92BF927F936F93C5
:10B560008CE69CE09F938F93CF93DF930F94AE3F35
:10B57000EDB7FEB738960FB6F894FEBF0FBEEDBF1D
:10B5800010C0AF92BF9280E79CE09F938F93CF93C0
:10B59000DF930F94AE3F0F900F900F900F900F908E
:10B5A0000F908D2F9C2FDF91CF911F910F91FF90C6
:10B5B000EF90DF90CF90BF90AF909F908F907F9053
:10B5C0006F905F904F903F902F9008958F929F9231
:10B5D000AF92BF92CF92DF92EF92FF920F931F93A1
:10B5E000CF93DF93CDB7DEB7E6970FB6F894DEBF03
:10B5F0000FBECDBF0091B9031091BA03F8010190BD
:10B600000020E9F731976F01C01AD10AF801CF0184
:10B61000801B910B8C159D0534F480818F3209F4C9
:10B6200010823196F4CF8BE1E9E5F2E1DE015C9620
:10B6300001900D928A95E1F7E12CF12CEC14FD04B8
:10B640000CF07AC0F801EE0DFF1D8081811103C05E
:10B650008FEFE81AF80A48018E0C9F1CF4018081D4
:10B66000882309F469C0FFEFEF1AFF0AF801EE0D15
:10B67000FF1D7F01E01AF10A81918111FACFCE01FD
:10B680004C960E94F3C48BE1FE017C96DE0111967C
:10B6900001900D928A95E1F7B401CE0101960E94C6
:10B6A0000499CE0101960E940EF18FE20E94273884
:10B6B0008091F60D811103C082ED92E002C086EF09
:10B6C0009DE05C01F50181915F01882319F00E94E2
:10B6D0002738F8CF80913C1284FF2EC019821C823B
:10B6E00021E0A401BE01645E7F4FCE0101960E945D
:10B6F00078C281110FC08AE00E9427380E9434F579
:10B70000B40185E891E30E941DF5CE0101960E94E7
:10B710000EF112C0CE014C960E946FC28BE1FE0169
:10B720003196DE015C9601900D928A95E1F7CE018B
:10B7300001960E940EF182CF8AE00E942738CE0146
:10B740004C960E940EF1E6960FB6F894DEBF0FBE3F
:10B75000CDBFDF91CF911F910F91FF90EF90DF90C0
:10B76000CF90BF90AF909F908F900895AB01BC0198
:10B77000409338125093391260933A1270933B12EF
:10B780008DE993E10C9445BCCF93DF93EC01CB01A1
:10B79000BA010F941D4020E030E0A9010F942C471E
:10B7A0000F94984879836883DF91CF9108950C9422
:10B7B000464DCF92DF92EF92FF920F931F938AE351
:10B7C000C82E86E3D82EE12CF12C0CEB19E127EDE5
:10B7D0003BE545EB56ED6CED7AE38BEC99E10E948D
:10B7E0008A501F910F91FF90EF90DF90CF900895B6
:10B7F0000E943E4D86EB99E19093DD048093DC043A
:10B8000008950E94ECF00E94A899109231120C94B5
:10B810003E4D9F92AF92BF92CF92DF92EF92FF92F6
:10B820000F931F93CF93DF9381E080933A0D61E0F4
:10B830000E94254CD091AE0DC0E09924939401E074
:10B840001CE58CEBE82E89E1F82E98EFC92E9BE5DC
:10B85000D92E2AE6A22E28E1B22ED1112BC0992092
:10B86000D9F08091AD0D1816BCF04091BF0D5091EC
:10B87000C00D6091C10D7091C20D4F5F5F4F6F4F52
:10B880007F4F4093BF0D5093C00D6093C10D7093D7
:10B89000C20D8F5F8093AD0D80916E02882309F4F5
:10B8A00041C020E030E041E06EE478E18C2F0E945E
:10B8B0003B5438C0D13059F48091AD0D8130D1F472
:10B8C0008091A80D1092A80D81110EC013C0D23026
:10B8D00049F58091AD0D8230A1F58091A80D1092AF
:10B8E000A80D811128C02DC00E94F85B8091CF0D5A
:10B8F000811137C080916E02882399F0DF92CF9238
:10B90000BF92AF92CF9381E09091AD0D913039F518
:10B910008F930E94FF4B0F900F900F900F900F90FE
:10B920000F90912CCF5FDF5FC53009F096CF83E099
:10B930008093A90D16C00E94015C8091CF0D8111EA
:10B9400010C080916E02882361F31F930F93FF92C2
:10B95000EF92CF9381E09091AD0D9230C9F280E0EB
:10B96000D7CFDF91CF911F910F91FF90EF90DF9094
:10B97000CF90BF90AF909F900895EF92FF920F935A
:10B980001F93CF93DF93CDB7DEB765970FB6F894CB
:10B99000DEBF0FBECDBF8091A80D1092A80D8823E9
:10B9A00019F00E94464D7AC060E085E00E94254C67
:10B9B0000091AE0D10E08AE3F82E90E2E92E01111D
:10B9C0000AC080916E02882361F120E030E043E0FC
:10B9D00069E470E323C0013051F480916E02882342
:10B9E00001F120E030E041E061EC7FE217C002307D
:10B9F00051F480916E028823A1F020E030E041E014
:10BA00006EE679E10BC00330E9F580916E02882380
:10BA100041F020E030E041E063E478E1812F0E94D2
:10BA20003B54F982EA8242E150E067EC7FE2CE01CA
:10BA300003960F94853F8C8987FD1C8A053059F445
:10BA400080916E028823A9F09E012F5F3F4F41E055
:10BA500063E679E10BC0063061F480916E028823C1
:10BA600041F020E030E041E061E579E1812F0E9482
:10BA70003B541F5F0F5F153009F0A1CF87E0809323
:10BA8000A90D0CC0043069F680916E02882349F23A
:10BA900020E030E041E06CEA7FE2C0CF65960FB66F
:10BAA000F894DEBF0FBECDBFDF91CF911F910F91F4
:10BAB000FF90EF900895EF92FF920F931F93CF9313
:10BAC000DF93CDB7DEB765970FB6F894DEBF0FBE34
:10BAD000CDBF8091A80D1092A80D882319F00E9467
:10BAE000464D75C060E085E00E94254C0091AE0D8A
:10BAF00010E08AE3F82E90E2E92E01110CC080914B
:10BB00006E02882341F020E030E043E067E479E111
:10BB1000812F0E943B54F982EA8242E150E060E4C6
:10BB200079E1CE0103960F94853F8C8987FD1C8AAD
:10BB3000013069F480916E02882349F09E012F5FE5
:10BB40003F4F41E06AE379E1812F0E943B54F98243
:10BB5000EA8242E150E066E379E1CE0103960F9478
:10BB6000853F8C8987FD1C8A023069F480916E02C2
:10BB7000882349F09E012F5F3F4F41E06CE279E15D
:10BB8000812F0E943B54F982EA8242E150E062E256
:10BB900079E1CE0103960F94853F8C8987FD1C8A3D
:10BBA000033069F480916E02882349F09E012F5F73
:10BBB0003F4F41E06CE179E1812F0E943B541F5FD0
:10BBC0000F5F153009F099CF84E08093A90D659639
:10BBD0000FB6F894DEBF0FBECDBFDF91CF911F919E
:10BBE0000F91FF90EF900895EF92FF920F931F93A4
:10BBF000CF93DF93CDB7DEB765970FB6F894DEBF6E
:10BC00000FBECDBF8091A80D1092A80D882319F00A
:10BC10000E94464DB5C060E085E00E94254C009131
:10BC2000AE0D10E08AE3F82E90E2E92E01110CC06F
:10BC300080916E02882341F020E030E042E06DE028
:10BC400079E1812F0E943B54F982EA8242E150E07F
:10BC500064ED78E1CE0103960F94853F8C8987FDD2
:10BC60001C8A013069F480916E02882349F09E019C
:10BC70002F5F3F4F40E064E079E1812F0E943B5409
:10BC8000F982EA8242E150E060E079E1CE01039678
:10BC90000F94853F8C8987FD1C8A023059F480916E
:10BCA0006E02882309F19E012F5F3F4F40E067EF4E
:10BCB00078E117C0033051F480916E028823A1F01F
:10BCC00020E030E040E065EE78E10BC0043061F444
:10BCD00080916E02882341F020E030E042E066ED82
:10BCE00078E1812F0E943B54F982EA8242E150E0E0
:10BCF00064ED78E1CE0103960F94853F8C8987FD32
:10BD00001C8A053069F480916E02882349F09E01F7
:10BD10002F5F3F4F40E064E079E1812F0E943B5468
:10BD2000F982EA8242E150E062ED78E1CE010396C9
:10BD30000F94853F8C8987FD1C8A063059F48091C9
:10BD40006E028823A9F09E012F5F3F4F40E067EF0E
:10BD500078E10BC0073061F480916E02882341F0D6
:10BD600020E030E040E065EE78E1812F0E943B5416
:10BD70001F5F0F5F153009F059CF88E08093A90D40
:10BD800065960FB6F894DEBF0FBECDBFDF91CF91A1
:10BD90001F910F91FF90EF9008952F923F924F9235
:10BDA0005F926F927F928F929F92AF92BF92CF924B
:10BDB000DF92EF92FF920F931F93CF93DF93CDB754
:10BDC000DEB7A1970FB6F894DEBF0FBECDBF80914E
:10BDD000A80D1092A80D882319F00E94464D19C194
:10BDE0008091C7049091C80499A388A3A091C90425
:10BDF000B091CA04BF8FAE8F4090CB045090CC045A
:10BE00006090CD047090CE048091CF049091D004C6
:10BE1000A091D104B091D2048A8F9B8FAC8FBD8F3B
:10BE20008090D3049090D404A090D504B090D60410
:10BE300060E085E00E94254C0091AE0D10E0DE012F
:10BE400011967D018AE0C82ED12C9AE7292E98E11F
:10BE5000392E01110DC080916E028823D9F188A17D
:10BE600099A10F94CD379C0140E061EC78E12FC09F
:10BE7000013069F480916E02882361F18E8D9F8D6F
:10BE80000F94CD379C0140E066EB78E120C0023092
:10BE900051F480916E028823E9F020E030E040E028
:10BEA00066EA78E114C0033009F053C080916E0255
:10BEB000882381F04E8A5F8A688E798EB701CE0121
:10BEC00046960E94075A9C0140E063EA78E1812F80
:10BED0000E943B5420E030E048EC52E4C501B4013C
:10BEE0000F9426480F949848CB01B6010F94FD4655
:10BEF0009F938F9320E030E04AE754E4C501B401FA
:10BF00000F9426480F9498489F938F937F936F9335
:10BF10003F922F92FF92EF920F94AE3F0FB6F8949C
:10BF2000DEBF0FBECDBF073059F480916E0288236B
:10BF300039F0970140E063EA78E1812F0E943B5499
:10BF40001F5F0F5F153009F084CF88E08093A90D43
:10BF500060C0043059F480916E02882309F4BACF8E
:10BF600020E030E040E061E978E118C00530D1F42C
:10BF700080916E02882309F4ADCF8A8D9B8DAC8DA4
:10BF8000BD8D8E8B9F8BA88FB98FB701CE01469642
:10BF90000E94075A9C0140E063EA78E1812F0E94E9
:10BFA0003B540DC0063009F095CF80916E02882376
:10BFB00031F020E030E040E062E878E188CF20E036
:10BFC00030E048EC52E4C501B4010F9426480F94C8
:10BFD0009848CB01B6010F94FD469F938F9320E0C4
:10BFE00030E04AE754E4C501B4010F9426480F94A9
:10BFF00098489F938F937F936F933F922F92FF92D6
:10C00000EF920F94AE3F0FB6F894DEBF0FBECDBFD8
:10C0100097CFA1960FB6F894DEBF0FBECDBFDF91CC
:10C02000CF911F910F91FF90EF90DF90CF90BF9035
:10C03000AF909F908F907F906F905F904F903F90C8
:10C040002F9008950F941D4020E030E0A9010F9437
:10C050002C470F949848CB010C940ED164EC7BE5EF
:10C0600082E290E60C945D4D8CE89AE10C94A2DC9F
:10C070008CE39AE10C94A2DC8FE69AE10C94A2DCAA
:10C0800087EC9AE10C94A2DC8BEA9AE10C94A2DC96
:10C0900088E19AE10C94A2DC2F923F924F926F922A
:10C0A0007F928F929F92AF92BF92CF92DF92EF9248
:10C0B000FF920F931F93CF93DF930E948C36382EFD
:10C0C00080913C1283FBDD27D0F983FF04C00E94DE
:10C0D0006F37282E01C0212C61E081E00E94254CA1
:10C0E0001091AE0D412C83EE682E8CEC782E97E8E3
:10C0F000E92E96EDF92E2CEFC22E29E1D22E36EE46
:10C10000A32E39E1B32E42EE842E49E1942E111173
:10C110000BC08091AD0D81113BC08091A80D109294
:10C12000A80D81112FC034C0332009F443C0113051
:10C1300061F48091AD0D813009F090C18091A80D1E
:10C140001092A80D811184C189C1123061F48091CF
:10C15000AD0D823009F0A3C08091A80D1092A80DFA
:10C16000811195C09CC0133009F092C18091AD0D32
:10C17000833009F097C18091A80D1092A80D81110C
:10C1800089C190C10E94464D8091CF0D8111D8C1C7
:10C1900080916E02882361F081E09091AD0D911144
:10C1A00080E004E024E04DE05AE1642D0E943B531E
:10C1B00031106EC10E947D37882371F0113071F407
:10C1C0008091AD0D813009F083C18091A80D10924E
:10C1D000A80D811177C17CC1C1E001C0C2E0C113CB
:10C1E00022C08091AD0D8C130EC08091A80D1092CD
:10C1F000A80D882341F08AE391E00E94A9908091E4
:10C20000CF0D81119DC180916E02882361F081E084
:10C210009091AD0D911380E003E02EE34FE05CE3DD
:10C22000642D0E943B53CF5FC11322C08091AD0D9E
:10C230008C130EC08091A80D1092A80D882341F098
:10C2400081EA92E90E94A9908091CF0D811178C175
:10C2500080916E02882361F081E09091AD0D911381
:10C2600080E003E02EE347E051E3642D0E943B535E
:10C2700081E08C0F811326C08091AD0D81134CC1DC
:10C280008091A80D1092A80D81113EC145C189ED84
:10C290009BE50E94A9908091CF0D811151C18091A1
:10C2A0006E02882309F44AC181E09091AD0D92306D
:10C2B00009F080E003E02EE34CEB59E1642D0E948D
:10C2C0003B53C4E082E08C0F811322C08091AD0DFE
:10C2D00081130EC08091A80D1092A80D882341F003
:10C2E0008CEC98ED0E94A9908091CF0D811128C10E
:10C2F00080916E02882361F081E09091AD0D9113E1
:10C3000080E003E02EE348E85AE3642D0E943B53AB
:10C3100083E08C0F811322C08091AD0D81130EC07C
:10C320008091A80D1092A80D882341F082EB92E62F
:10C330000E94A9908091CF0D811102C180916E025F
:10C34000882361F081E09091AD0D911380E003E0CE
:10C350002EE345EA59E1642D0E943B5384E08C0FA3
:10C3600031106EC0DD2309F44CC0211069C0811367
:10C3700020C09091AD0D91130EC08091A80D109228
:10C38000A80D882341F09092DD048092DC04809116
:10C39000CF0D8111D5C080916E02882351F081E0CC
:10C3A000911380E000E22EE340ED59E1642D0E94FC
:10C3B0003B5385E08C0F811322C08091AD0D81131A
:10C3C0000EC08091A80D1092A80D882341F080ED39
:10C3D00091E00E94A9908091CF0D8111B1C0809110
:10C3E0006E02882361F081E09091AD0D911380E0A1
:10C3F00003E02EE348E85CE3642D0E943B5386E0B3
:10C400001EC081131BC08091AD0D811302C010921C
:10C41000A80D90916E02992389F01F921F92BF92EE
:10C42000AF924F9291E0811390E09F930E94FF4B57
:10C430000F900F900F900F900F900F9085E08C0F42
:10C4400043941F5F95E0491262CE8093A90D78C096
:10C450000E9487D68091CF0D811172C080916E02AB
:10C46000882309F46BC0FF92EF92DF92CF924F9234
:10C4700081E09091AD0D913009F080E08F930E94A2
:10C48000FF4B0F900F900F900F900F900F9056C092
:10C49000C4E0CACE87EB90E90E94A9908091CF0DAD
:10C4A00081114EC080916E02882309F447C081E05B
:10C4B0009091AD0D933009F080E003E02EE344EF5E
:10C4C00059E1FCCE0E94E3CC8091CF0D811138C0A0
:10C4D00080916E028823B1F07F926F928AE698E194
:10C4E0009F938F934F9281E09091AD0D913009F021
:10C4F00080E08F930E94FF4B0F900F900F900F9052
:10C500000F900F90C2E08FCE8AE39AED0E94A9901F
:10C510008091CF0D811114C080916E02882309F49F
:10C52000D1CE81E09091AD0D911380E003E02EE338
:10C530004CE558E1642D0E943B53C4CEC4E098CE34
:10C54000DF91CF911F910F91FF90EF90DF90CF90EF
:10C55000BF90AF909F908F907F906F904F903F9043
:10C560002F9008950F93CF93DF9361E081E00E94B5
:10C57000254CD091AE0DC0E0D1110BC08091AD0D16
:10C58000811129C08091A80D1092A80D81111DC0A4
:10C5900022C0D13059F48091AD0D813091F5809158
:10C5A000A80D1092A80D811124C02BC0D23009F023
:10C5B00041C08091AD0D823009F05EC08091A80D20
:10C5C0001092A80D811150C057C00E94464D809115
:10C5D000CF0D811190C080916E02882319F181E006
:10C5E0009091AD0D911180E004E024E04FE251E321
:10C5F00016C08DEB9CE50E94A9908091CF0D811112
:10C600007AC080916E02882369F081E09091AD0D2F
:10C61000913009F080E003E02EE345EA59E16C2F08
:10C620000E943B53CF5FDF5FC53009F0A5CFC093B9
:10C63000A90D61C0D33059F48091AD0D833099F5C7
:10C640008091A80D1092A80D811125C02CC0D43066
:10C6500049F78091AD0D8430F1F58091A80D1092CD
:10C66000A80D811130C037C08BE59DE50E94A990CF
:10C670008091CF0D81113FC080916E02882391F28D
:10C6800081E09091AD0D923009F080E003E02EE35F
:10C6900049E959E1C4CF84EF9DE50E94A9908091BA
:10C6A000CF0D811128C080916E02882309F4BACF82
:10C6B00081E09091AD0D933009F080E003E02EE32E
:10C6C0004BE859E1ACCF8DEC9EE50E94A99080919A
:10C6D000CF0D811110C080916E02882309F4A2CF82
:10C6E00081E09091AD0D943009F080E003E02EE3FD
:10C6F00049E759E194CFDF91CF910F9108956111EE
:10C70000609302024093BC03082E000C990BAA0B05
:10C71000BB0B8C30910570F5FC018827EA55FF4F63
:10C720008F4F0D94114788E390E61BC089ED9DED76
:10C7300016C085ED9DED13C080E490E612C084E440
:10C7400090E60FC088E490E60CC081ED9DED07C037
:10C750001092E60D80EA97ED02C08DED9DED0097F9
:10C7600049F021E020933A0D20E040E060E070E0E5
:10C770000C948E4C0C943E4D84E390E6F2CF8CE307
:10C7800090E6EFCFE091AC0D86E0E802F0011124D5
:10C79000E15DFB4F8091B10D90E095838483089516
:10C7A0003F924F925F926F927F928F929F92AF9241
:10C7B000BF92CF92DF92EF92FF920F931F93CF938E
:10C7C000DF93CDB7DEB728970FB6F894DEBF0FBE64
:10C7D000CDBF3090AC0D61E081E00E94254C2091EE
:10C7E000AE0D28871F8211E0232D30E0C901880F8C
:10C7F000991FAC014D5F534C5A83498346E0429FD9
:10C80000C001439F900D1124FC01E15DFB4F3F01EE
:10C810009F012C5F3F4F3C832B832F0132E0430E5F
:10C82000511CAC014F5C5B4F5E834D8358855111A9
:10C830002CC01123D9F08091AD0D1816BCF0409199
:10C84000BF0D5091C00D6091C10D7091C20D4F5F31
:10C850005F4F6F4F7F4F4093BF0D5093C00D60935C
:10C86000C10D7093C20D8F5F8093AD0D80916E02EC
:10C87000882381F1E981FA816591749120E030E0AB
:10C8800043E08F810E943B5425C08885813011F59B
:10C890008091AD0D813061F48091A80D1092A80DAA
:10C8A000882331F00E94464D8091CF0D81112BC11C
:10C8B00080916E02882369F081E09091AD0D9130F6
:10C8C00009F080E004E024E04CE558E16F810E942B
:10C8D0003B5310E0EB81FC8180818093B10DF885A2
:10C8E000F23071F43092AC0D8091AD0D823009F0D0
:10C8F0003EC08091A80D1092A80D81112EC037C0A6
:10C900002885233061F48091AD0D833009F07FC01C
:10C910008091A80D1092A80D81114DC078C0F885A6
:10C92000F43061F48091AD0D843009F0B2C0809193
:10C93000A80D1092A80D81117EC0ABC0F885F5300E
:10C9400069F58091AD0D853009F0BEC08091A80DCC
:10C950001092A80D8111B2C0B7C062EC73E684E1F9
:10C9600091E30F9401398091CF0D8111CCC080915A
:10C970006E02882391F011E08091AD0D823009F0B4
:10C9800010E08091B10D0E9473D100E09C0144E160
:10C9900051E36F81812F0E943E5510E02F812F5F60
:10C9A0002F8338853F5F3887253009F03FCF86E0F9
:10C9B0008093A90DA8C0F3016081718180E090E0AF
:10C9C0000F941B4020E030E0A9010F942C4720E099
:10C9D00030E040EA50E40F942B470F949F48812C9D
:10C9E000912C2AEBA22E28EDB22E6B01E12CF12C1A
:10C9F0008701EA9425E030E040E050E0B30184E2B2
:10CA000091E30F94240A8091CF0D81117CC0809115
:10CA10006E02882311F211E08091AD0D833009F090
:10CA200010E0F301808191810E9444D100E09C01DB
:10CA300044E251E3AECFF2016081718180E090E089
:10CA40000F941B4020E030E0A9010F942C4720E018
:10CA500030E040EA50E40F942B470F949F48812C1C
:10CA6000912C8AEBA82E88EDB82E6B011EE6E12EE4
:10CA7000F12C00E010E025E030E040E050E06D8176
:10CA80007E8184E892E40F94240A8091CF0D811175
:10CA90003AC080916E02882309F47FCF11E0809123
:10CAA000AD0D843009F010E0F201808191810E9487
:10CAB00044D100E09C0144E852E46BCF0E94C6CC14
:10CAC0008091CF0D81111FC080916E02882309F4DF
:10CAD00064CF26EC3CEC3F932F938AEC96E39F9334
:10CAE0008F93FF81FF9381E09091AD0D953009F018
:10CAF00080E08F930E94FF4B0F900F900F900F904C
:10CB00000F900F904ACF28960FB6F894DEBF0FBE55
:10CB1000CDBFDF91CF911F910F91FF90EF90DF90EC
:10CB2000CF90BF90AF909F908F907F906F905F90CD
:10CB30004F903F90089581E080933A0D1092DA046F
:10CB40001092AE0420E040E060E070E081EB95E6FA
:10CB50000E948E4C84E89CE39093DD048093DC0477
:10CB6000089580916E02882341F020E030E041E09A
:10CB700063E27BE182E00E943B548091AE048770C7
:10CB8000873041F420E040E060E070E084EE95E61C
:10CB90000C948E4C089520E040E060E070E087E265
:10CBA00096E60E948E4C81E08093BE038091BF0385
:10CBB000811103C088E09BE102C08EEF91E4909365
:10CBC000DD048093DC04089580916E02882341F097
:10CBD00020E030E041E06FE07BE181E00E943B54E7
:10CBE0008091A80D1092A80D882321F01092BF0308
:10CBF0000C94CB65089581E080933A0D8091DA041E
:10CC00008770873051F01092DA041092AE0484E8F5
:10CC10009CE39093DD048093DC048091410E80932B
:10CC2000BD0380E00E94D7F220E040E060E070E0C9
:10CC300080E592E00C948E4C6091B10D7091B20D34
:10CC40008091B30D9091B40D41E00C94F2F20F93EA
:10CC50001F93CF93DF93CDB7DEB72A970FB6F89423
:10CC6000DEBF0FBECDBF80916E028823F1F01F9210
:10CC700089E08F938091BF0390E001969F938F93FB
:10CC800080E09BE19F938F938E010F5F1F4F1F9357
:10CC90000F930F94AE3FB80182EF9AE10E94B9540E
:10CCA0000FB6F894DEBF0FBECDBF84E080936E0256
:10CCB0008091BE03811108C020E040E060E070E098
:10CCC0008FE696E60E948E4C2A960FB6F894DEBF49
:10CCD0000FBECDBFDF91CF911F910F910895CF92DD
:10CCE000DF92EF92FF920F931F93CF93DF9300D0C9
:10CCF0001F92CDB7DEB78091A80D1092A80D8823A2
:10CD0000E1F08091BF038F5F8093BF03893090F083
:10CD100081E08093BE0320E040E060E070E080E3CB
:10CD200097E60E948E4C8EEF91E49093DD04809301
:10CD3000DC0489C00E94CB6586C06091BF0D7091F4
:10CD4000C00D8091C10D9091C20D611571058105D5
:10CD5000910509F448C00F941D402DEC3CEC4CECBF
:10CD60005CE30F947C402091591130915A1140910D
:10CD70005B1150915C110F942C477B018C0120E0DA
:10CD800030E040E050EC0F94164087FD0FC020E0EB
:10CD900030E040E050E4B701C8010F948C49181608
:10CDA0004CF4E12CF12C00E010E404C0E12CF12C57
:10CDB00000E010ECC701D8018093591190935A11EB
:10CDC000A0935B11B0935C118BE892E00E945F89A5
:10CDD00082E080936E021092BF0D1092C00D1092EF
:10CDE000C10D1092C20D80916E02882361F1C09036
:10CDF0005911D0905A11E0905B11F0905C1120E035
:10CE000030E0A901C701B6010F94164087FD05C0A7
:10CE100027E137EB41ED58E304C027E137EB41ED63
:10CE200058EBC701B6010F942C4769837A838B8333
:10CE30009C836BE2CE0101960E94A1CDBC0184EFE0
:10CE400099E30E94B9540F900F900F900F90DF91CB
:10CE5000CF911F910F91FF90EF90DF90CF900895A9
:10CE60008091BE03811104C00E94244E0E94104C88
:10CE700080916E02882341F020E030E041E06FEDC8
:10CE80007AE181E00E943B5482E080936E02089533
:10CE90002F923F924F925F926F927F928F929F92CA
:10CEA000AF92BF92CF92DF92EF92FF920F931F93B8
:10CEB000CF93DF9300D0CDB7DEB78091DA048770CF
:10CEC00089830E94DBF3682E61E081E00E94254C9B
:10CED0002091AE0D2A83712C4BED442E4CEC542E38
:10CEE0005AEC252E56E3352E8A8181110BC0809194
:10CEF000AD0D811195C18091A80D1092A80D8111E1
:10CF000089C18EC19A81913061F48091AD0D8130DB
:10CF100009F09CC18091A80D1092A80D81118EC1BD
:10CF200095C12981273011F082E02FC06620E1F3FE
:10CF30009A81923049F52091410E2B838091AD0D5D
:10CF4000823031F48091A80D1092A80D811190C10A
:10CF500080916E02882309F4B1C181E09091AD0DFA
:10CF6000923009F080E09B81911103C02FEE36E3EF
:10CF700002C026EF36E301E04DE15CE3672D0E943D
:10CF80003E5523E02B8302C083E08B8380913D0ECE
:10CF900090913E0EA0913F0EB091400E8093B10D46
:10CFA0009093B20DA093B30DB093B40D9B812A81E1
:10CFB00092133DC08091AD0D89131DC08091A80DC5
:10CFC0001092A80D8823B9F00E9448F72CE1C22ED8
:10CFD00026E6D22EE12CF12C08EC12E420E030E021
:10CFE000A90161EB7DE083E49BE10E94A6F68091BC
:10CFF000CF0D811176C180916E028823C1F011E0BE
:10D000008091AD0D9A81891310E06091B10D7091FE
:10D01000B20D8091B30D9091B40D0E94C64B00E00B
:10D020009C0143E45BE1672D812F0E943E558B817B
:10D030008F5F2A8182135CC08091AD0D82133CC04A
:10D040008091A80D1092A80D8823B1F120E030E066
:10D050004AE754E460913B0470913C0480913D04A4
:10D0600090913E040F947C4020E030E0A9010F94A1
:10D070002C4720E030E04AE754E40F942C470F940B
:10D080009F48812C912C82E1A82E81E0B82E6B0163
:10D0900010EDE12E17E0F12E00E010E028E13CEF6A
:10D0A0004FEF5FEF6BE374E089E291E30F94240AA2
:10D0B0008091CF0D811115C180916E028823C1F03E
:10D0C00011E08091AD0D9A81891310E060913B04CD
:10D0D00070913C0480913D0490913E040E9464470D
:10D0E00000E09C0149E251E3672D812F0E943E55EB
:10D0F0008B818E5F2A81821323C08091AD0D8213B4
:10D100000EC08091A80D1092A80D882341F08BEFDE
:10D1100095E60E94A9908091CF0D8111E2C0809187
:10D120006E02882369F081E09091AD0D2A819213FF
:10D1300080E003E02EE342E35BE1672D0E943B5376
:10D140008B818D5F9A8189132AC08091AD0D8913DF
:10D150000CC08091A80D1092A80D882331F00E9478
:10D16000DBCC8091CF0D8111BCC080916E028823F1
:10D17000B1F05F924F928AEB96E39F938F937F92E9
:10D1800081E09091AD0D2A81921380E08F930E94EF
:10D19000FF4B0F900F900F900F900F900F908B817F
:10D1A0008C5F9A8189132AC08091AD0D89130CC0C0
:10D1B0008091A80D1092A80D882331F00E94C6CC52
:10D1C0008091CF0D81118DC080916E028823B1F0C6
:10D1D00086EC9CEC9F938F933F922F927F9281E0FD
:10D1E0009091AD0D2A81921380E08F930E94FF4BA6
:10D1F0000F900F900F900F900F900F9073948A8163
:10D200008F5F8A8395E079126FCE2B812B5F2093FD
:10D21000A90D67C00E94464D8091CF0D811161C05C
:10D2200080916E02882399F181E09091AD0D91116A
:10D2300080E004E024E04FE05CE316C08BE995E673
:10D240000E94A9908091CF0D81114BC080916E02F8
:10D250008823E9F081E09091AD0D913009F080E0F4
:10D2600003E02EE343E55BE1672D0E943B530FC0D3
:10D270008B8191E089278B8323E020936E020E94AB
:10D280000D498091CF0D882309F462CE2AC099817F
:10D29000973009F44BCE80913D0E90913E0EA091B7
:10D2A0003F0EB091400E8093B10D9093B20DA093BC
:10D2B000B30DB093B40D82E08B83B9CE80913D0E57
:10D2C00090913E0EA0913F0EB091400E8093B10D13
:10D2D0009093B20DA093B30DB093B40D23E02B83C4
:10D2E000A6CE0F900F900F90DF91CF911F910F91CD
:10D2F000FF90EF90DF90CF90BF90AF909F908F9076
:10D300007F906F905F904F903F902F9008958F92F5
:10D310009F92AF92BF92CF92DF92EF92FF92CF9304
:10D320006B017C0120E030E0A9010F94164087FDDD
:10D3300005C06DEB77E386E095E304C06DEB77E322
:10D3400086E095EBA70196010F942C476B017C01B9
:10D3500020E030E040E251E40F947C4020E030E0F7
:10D3600048EC52E40F947C404B015C0120E030E03B
:10D37000A901C701B6010F94164087FD05C020E042
:10D3800030E040EA50E404C020E030E040EA50ECF5
:10D39000C501B4010F942C4720E030E040E251E495
:10D3A0000F9426480F9498486B017C0197FF0AC0A0
:10D3B000F094E094D094C094C11CD11CE11CF11CE9
:10D3C0008DE201C08BE280933B0DC701B60120E1E5
:10D3D00037E240E050E00F948E468AE0882E912C90
:10D3E000A12CB12CCA01B901A50194010F948E465C
:10D3F000605D60933C0DC701B60128EE33E040E06C
:10D4000050E00F948E46CA01B901A50194010F9412
:10D410008E46605D60933D0DC701B60124E630E0A5
:10D4200040E050E00F948E46CA01B901A501940175
:10D430000F948E46605D60933E0D8EE280933F0DAB
:10D44000C701B601A50194010F948E46C62FCA01EB
:10D45000B901A50194010F948E46605D6093400D63
:10D46000C05DC093410D8BE39DE0CF91FF90EF90A5
:10D47000DF90CF90BF90AF909F908F9008957F9254
:10D480008F929F92AF92BF92CF92DF92EF92FF92D4
:10D490000F931F93CF93DF9361E081E00E94254CAF
:10D4A000D091AE0DC0E0A3E07A2ED1110BC08091D7
:10D4B000AD0D811129C08091A80D1092A80D811188
:10D4C0001DC022C0D13059F48091AD0D8130D1F50D
:10D4D0008091A80D1092A80D811127C033C0D230C1
:10D4E00009F04FC08091AD0D823009F099C0809154
:10D4F000A80D1092A80D811164C092C00E94464DE3
:10D500008091CF0D8111BCC180916E02882381F181
:10D5100081E09091AD0D911180E004E024E04CE5B4
:10D5200058E16C2F0E943B5323C080910D048D273E
:10D5300080930D0470926E020E94FADD8091CF0DEF
:10D5400081119EC180916E02882391F081E09091BB
:10D55000AD0D913009F080E090910D0491111FC044
:10D560002FEE36E301E04CEA5BE16C2F0E943E5562
:10D57000CF5FDF5FC53009F098CF87E08093A90DBA
:10D580007FC1D33079F48091AD0D833009F077C03D
:10D590008091A80D1092A80D81115CC070C026EF7B
:10D5A00036E3E0CFD43009F086C08091AD0D8430F1
:10D5B00009F0CDC08091A80D1092A80D811198C0DE
:10D5C000C6C020E030E048EC52E460910E04709157
:10D5D0000F0480911004909111040F947C4020E07E
:10D5E00030E0A9010F942C470F949F48812C912C77
:10D5F000E6ECAE2EE8EDBE2E6B0110E1E12E17E257
:10D60000F12E00E010E020E030E0A9016EE074E0CF
:10D610008BE99BE10F94240A8091CF0D811130C1D9
:10D6200080916E02882309F4A3CF11E08091AD0DA3
:10D63000823009F010E060910E0470910F04809127
:10D640001004909111040E94876900E09C014BE94D
:10D650005BE12EC0C12CD12CE12C10ECF12E09E79E
:10D6600014E420E030E040E85FE362E174E08BE83E
:10D670009BE10E94A6F68091CF0D811101C180919E
:10D680006E02882309F474CF11E08091AD0D8330D0
:10D6900009F010E060911204709113048091140459
:10D6A000909115040E94C64B00E09C014BE85BE1A1
:10D6B0006C2F812F5BCFD53061F48091AD0D85301B
:10D6C00009F095C08091A80D1092A80D811159C044
:10D6D0008EC0D63009F04CCF8091AD0D863009F068
:10D6E000B5C08091A80D1092A80D81119AC0AEC04E
:10D6F00020E030E048EC52E4609116047091170489
:10D7000080911804909119040F947C4020E030E03F
:10D71000A9010F942C470F949F48812C912C36EC33
:10D72000A32E38EDB32E6B011CE3E12E16E8F12E8B
:10D7300001E010E020E030E0A90166E174E081E85A
:10D740009BE10F94240A8091CF0D811199C08091A3
:10D750006E02882309F40CCF11E08091AD0D843066
:10D7600009F010E06091160470911704809118047C
:10D77000909119040E94876900E09C0141E85BE1F7
:10D7800097CF20E030E048EC52E460911A047091A9
:10D790001B0480911C0490911D040F947C4020E098
:10D7A00030E0A9010F942C4720E030E44CE156E42E
:10D7B0000F942C470F949F48812C912C96ECA92E06
:10D7C00098EDB92E6B0110E2E12E1EE4F12E00E07F
:10D7D00010E020EF38ED4FEF5FEF6AE174E081E792
:10D7E0009BE10F94240A8091CF0D811149C0809153
:10D7F0006E02882309F4BCCE11E08091AD0D853016
:10D8000009F010E060911A0470911B0480911C04CF
:10D8100090911D040E94876900E09C0141E75BE153
:10D8200047CFC12CD12CE12C10ECF12E09E714E4E8
:10D8300020E030E040E85FE36EE174E081E69BE1E8
:10D840000E94A6F68091CF0D81111AC080916E02C0
:10D85000882309F48DCE11E08091AD0D863009F05A
:10D8600010E060911E0470911F048091200490913B
:10D8700021040E94C64B00E09C0141E65BE118CF09
:10D88000DF91CF911F910F91FF90EF90DF90CF909C
:10D89000BF90AF909F908F907F9008954F925F922E
:10D8A0006F927F928F929F92AF92BF92CF92DF92B0
:10D8B000EF92FF920F931F93CF93DF9300D01F92AD
:10D8C000CDB7DEB70E947BFA4B015C0110910902D3
:10D8D0001F3FE9F10E947BFAC090F903D090FA0350
:10D8E000E090FB03F090FC03DC01CB018C199D0957
:10D8F000AE09BF09B7FD2BC080919311909194118F
:10D900008F5F8F70891719F1143060F524E0129F32
:10D91000F0011124ED57FD4F80819181A281B381E7
:10D9200089839A83AB83BC83C12CD12C76018E0171
:10D930000F5F1F4F2DE531E149E551E165E571E1EB
:10D9400081E591E10E9468B98FEF809309020E94FE
:10D9500007D78091C803811191C18091FE1582FD86
:10D9600006C08CC180E090E0A8E4B2E4D9CF8091F9
:10D97000040481110CC081E0809304049091E70DB0
:10D9800089278093A80D1092E70D0F945230809153
:10D99000C4039091C503A091C603B091C703A5012C
:10D9A0009401281B390B4A0B5B0B57FF05C0809174
:10D9B000C303882309F40DC2D501C4018C599F4FBC
:10D9C000AF4FBF4F8093C4039093C503A093C6038A
:10D9D000B093C7036091E00C062E000C770B77FF25
:10D9E00003C07195619571099091E00C80910304D9
:10D9F000981347C1633008F044C11092E00C809145
:10DA0000E00C80930304643028F48091A80D811108
:10DA100087C097C08091B90D882309F45AC0C0907F
:10DA2000B50DD090B60DE090B70DF090B80DC114C3
:10DA3000D104E104F10409F43FC070E080E090E01B
:10DA40000F941B4020E030E040E85EE30F947C4000
:10DA50002B013C01C501B4016C197D098E099F0998
:10DA60000F941B409B01AC01C301B2010F942648E7
:10DA700020E030E04AE754E40F947C406B017C01E5
:10DA800020E030E040EA52E40F948C4987FF0FC059
:10DA900020E030E040EF51E4C701B6010F948C491B
:10DAA00087FD0AC02AE030E040E050E009C024E6EB
:10DAB00030E040E050E004C021E030E040E050E0E1
:10DAC0008092B50D9092B60DA092B70DB092B80DA0
:10DAD00004C021E030E040E050E0A091E00C0A2ECC
:10DAE000000CBB0B0F94B84624E030E040E050E05F
:10DAF0000F948E468091BF0D9091C00DA091C10DE5
:10DB0000B091C20D820F931FA41FB51F8093BF0D4C
:10DB10009093C00DA093C10DB093C20D1092E00C74
:10DB2000D501C4018856954CAF4FBF4F8093FF037A
:10DB300090930004A0930104B093020481E08093C9
:10DB40006E028091D5119091D6113FE68C369307E5
:10DB500029F480915502882351F0C6C0805D914020
:10DB6000B9F480915502882309F49BC0BDC08CE0B4
:10DB7000809355028091FD039091FE03009729F058
:10DB800001979093FE038093FD0381E080936E02E2
:10DB90000E94DA84C0906C07D0906D07E0906E0709
:10DBA000F0906F0781110E94E784D701C6013AE027
:10DBB000B695A795979587953A95D1F7009751E037
:10DBC000A507B10520F08FEF9FEFA0E0B0E096959C
:10DBD000879520916E02211105C03091C303311148
:10DBE000F4C03FC0009739F04091FD035091FE030F
:10DBF00048175907B0F58091C303882309F478C00A
:10DC000083E00E94B75281E08093FB11E091D5112F
:10DC1000F091D61119951092C2038091C30381111E
:10DC200074C01092A80D8091D5119091D6118C5688
:10DC30009F46F9F40E947BFADC01CB01881999090F
:10DC4000AA09BB09C090FD03D090FE03E12CF12C82
:10DC5000C816D906EA06FB0620F49093FE038093CB
:10DC6000FD038091D5119091D6118C569F4609F4F1
:10DC70009DC080913A0D811199C07EC0109204041C
:10DC800086CE633009F0BBCE8091E00C87FD02C0E8
:10DC900081E001C08FEF880F880F8093E00C64E073
:10DCA000AECE84E0809355028091D00D8F5F80933B
:10DCB000D00D9091D10D981728F41092D00D8CE0D2
:10DCC0008093550281E080936E02D501C40188568D
:10DCD000954CAF4FBF4F8093FF0390930004A093E8
:10DCE0000104B093020454CF81508093550250CF69
:10DCF0002230C0F0243028F02430A1F410926E02BB
:10DD000011C081E080936E020DC08BED91E10F9404
:10DD1000690E91E0811101C090E09093C3038111DD
:10DD20000BC07FCF87ED91E10F943C2F81E0809372
:10DD3000C2038093C30364CF8091D5119091D61113
:10DD40008C569F4609F045C00E947BFADC01CB014E
:10DD500088199909AA09BB09C090FD03D090FE0358
:10DD6000E12CF12CC816D906EA06FB0690F5909333
:10DD7000FE038093FD032DC08091FF03909100046A
:10DD8000A0910104B0910204881A990AAA0ABB0A58
:10DD9000B7FE0E943E4D8091C30381111AC080914D
:10DDA0006E028130B1F410926E0213C058E9850EF4
:10DDB0005AE3951EA11CB11C8092FF0390920004AF
:10DDC000A0920104B0920204E6CF009709F418CFA4
:10DDD0000BCF0F900F900F900F90DF91CF911F916D
:10DDE0000F91FF90EF90DF90CF90BF90AF909F90FA
:10DDF0008F907F906F905F904F900895CF92DF92B9
:10DE0000EF92FF92CF93C82F0E947BFA6B017C01A7
:10DE100024EA30E74DE75FE3609105027091060266
:10DE200080910702909108020F94164087FD05C06B
:10DE30008AEF90E0A0E0B0E003C080E090E0DC0179
:10DE4000C80ED91EEA1EFB1EC092F903D092FA0337
:10DE5000E092FB03F092FC03C0930902CF91FF9084
:10DE6000EF90DF90CF900895CF92DF92EF92FF92E4
:10DE70000F931F930E947BFA0091CA031091CB036A
:10DE80002091CC033091CD036B017C01C01AD10AE3
:10DE9000E20AF30AF7FC13C02091C90320952093EE
:10DEA000C903DC01CB018A549C4FAF4FBF4F809315
:10DEB000CA039093CB03A093CC03B093CD0381E02E
:10DEC0009091C903911101C080E01F910F91FF90C3
:10DED000EF90DF90CF9008954F925F926F927F9274
:10DEE0008F929F92AF92BF92CF92DF92EF92FF926A
:10DEF0000F931F93CF93DF93CDB7DEB72C970FB659
:10DF0000F894DEBF0FBECDBF1092B90D8091A80D61
:10DF10001092A80D8823B1F020E040E060E070E0AE
:10DF20008CE490E60E948E4C81E08093C0038DEBE0
:10DF30009BE19093260F8093250F1092280F10924B
:10DF4000270F0EC620911002309111024091BF0D93
:10DF50005091C00DC901840F951F2436310559F425
:10DF60004730510514F0069723C04A3F5F4F0CF02D
:10DF70003AC306961DC0243631052CF4853691052A
:10DF80000CF031C305C0843691050CF42CC303C0DA
:10DF90008A3091053CF0883EE3E09E072CF087EE46
:10DFA00093E002C08AE090E02817390731F411C0ED
:10DFB0008A30910584F78AE090E090931102809373
:10DFC00010021092BF0D1092C00D1092C10D109250
:10DFD000C20D8091C203882309F419C26091370FE2
:10DFE0007091380F072E000C880B990B0F941D4071
:10DFF00011E02091330F3091340F4091350F509143
:10E00000360F0F948C4918160CF010E060914A0EF0
:10E0100070914B0E072E000C880B990B0F941D402E
:10E020002091460E3091470E4091480E5091490E76
:10E030000F948C4918160CF412601093F803209179
:10E04000651130916611409167115091681160918E
:10E0500055117091561180915711909158110F944C
:10E060002C474B015C012091691130916A1140915C
:10E070006B1150916C116091591170915A118091EE
:10E080005B1190915C110F942C476B017C012091E6
:10E09000611130916211409163115091641160914E
:10E0A00051117091521180915311909154110F940C
:10E0B0002C4769837A838B839C838D829E82AF8277
:10E0C000B886C986DA86EB86FC8620E030E040E23E
:10E0D00051E4C701B6010F947C4020E030E048ECE9
:10E0E00052E40F947C404B015C0120E030E0A90138
:10E0F000C701B6010F94164087FF05C020E030E04D
:10E1000040EA50EC04C020E030E040EA50E4C501B1
:10E11000B4010F942C4720E030E040E251E40F942A
:10E1200026480F9498486B017C0197FF0AC0F09431
:10E13000E094D094C094C11CD11CE11CF11C8DE270
:10E1400001C080E280933B0DF0E1CF16F7E2DF06DD
:10E15000E104F10494F0C701B60120E137E240E0A8
:10E1600050E00F948E46CA01B9012AE030E040E049
:10E1700050E00F948E46605D01C060E260933C0DFC
:10E1800028EEC21623E0D206E104F10494F0C701A0
:10E19000B60128EE33E040E050E00F948E46CA010D
:10E1A000B9012AE030E040E050E00F948E46605D17
:10E1B00001C060E260933D0DC701B60124E630E086
:10E1C00040E050E00F948E466AE0862E912CA12C00
:10E1D000B12CCA01B901A50194010F948E46605D6E
:10E1E00060933E0DC701B601A50194010F948E46C0
:10E1F000162F662381F08EE280933F0DCA01B9018C
:10E20000A50194010F948E46605D6093400D105DF2
:10E210001093410D17C0CA01B901A50194010F94D3
:10E220008E46662339F08EE280933F0D605D6093E9
:10E23000400D05C080E28093400D80933F0D80E249
:10E240008093410D6BE37DE080EF93E00F94914A62
:10E25000CE0101960E94BDCEBC018BEE93E00F94DF
:10E26000914ACE0105960E94BDCEBC0186EE93E098
:10E270000F94914A1091C1031F7739F50E946F37AF
:10E28000882319F18091341290913512A0913612A1
:10E29000B09137120097A105B105B9F0BC01CD01CD
:10E2A0006D597F4F8F4F9F4F24E630E040E050E0A4
:10E2B0000F946C46609138127091391280913A1225
:10E2C00090913B120F946C46122F0E943E8B062FAA
:10E2D000972E5C01F62E80910402811709F43FC04D
:10E2E0001093040238E4139FB001112480E090E001
:10E2F0000F941B402AE037ED43E25CE30F947C402F
:10E300000F949F486093E503111103C01092E0033E
:10E3100026C0143630F0812F64E60F94CF46805D1E
:10E3200001C080E280933F0D1A3048F02AE0812F2F
:10E33000622F0F94CF460F94CF46905D01C090E2BC
:10E340009093400D812F6AE00F94CF46905D90939B
:10E35000410D6FE37DE080EE93E00F94914A809150
:10E360000302F81609F453C000930302602F792DBD
:10E37000C50120E13EE040E050E00F946C466901A9
:10E380007A014CE3442E512C612C712C602F792D95
:10E39000C501A30192010F946C46CA01B901A30102
:10E3A00092010F946C4644E6C416D104A8F47F93FE
:10E3B0006F93DF92CF928DEB9CE19F938F9380EDD3
:10E3C00093E09F938F930F94AE3F0FB6F894DEBF08
:10E3D0000FBECDBF85E014C07F936F93DF92CF92C5
:10E3E00083EB9CE19F938F9380ED93E09F938F93BA
:10E3F0000F94AE3F0FB6F894DEBF0FBECDBF86E0E0
:10E400009AEF899F802D112480588093CF030E941A
:10E41000346F182F81E00E94B75280910F1284311F
:10E4200028F480911112883008F0E0C08091F80340
:10E43000282F227081FF03C048E00CE002C042E1B7
:10E4400002E080910F1290E044977CF480911112C9
:10E45000841758F02111D7C089E59CE17C0123E0A5
:10E4600060E58BED91E10F94950880910F12843156
:10E47000B8F480911112823098F0112309F4C6C0CB
:10E4800080917007882309F4C1C083E29CE17C017C
:10E4900002E123E042E068E68BED91E10F949508FC
:10E4A00080910F128C31B0F59091F8038090330F6A
:10E4B0009090340FA090350FB090360FC090370F6A
:10E4C000D090380F843128F480911112883008F0F0
:10E4D00050C280910F12883008F42BC280910F1225
:10E4E0008C3108F42DC2C090460ED090470EE090BB
:10E4F000480EF090490E80910F12883008F426C221
:10E5000080910F128C3108F428C280910F128C3147
:10E5100008F429C20E946F37882349F080910F12B6
:10E52000843328F4809111128A3208F072C08091ED
:10E530000F12853328F480911112813308F091C0B5
:10E5400080910F12843328F480911112823308F0E5
:10E550008FC080910F128033D8F4809111128832CD
:10E56000B8F08091E003882361F040EE53E060E36F
:10E5700087E30E94F85565E270E080E090E00E9439
:10E58000CA5240ED53E060E38091CF030E94F855FA
:10E5900080910F12883298F4809111128D3178F0A9
:10E5A0002BE040E86DE180E00F94E70880910F12C6
:10E5B000873228F4809111128F3108F063C0809166
:10E5C0000F12833328F4809111128B3208F016C198
:10E5D00080910F12813408F0C3C2809111128633EA
:10E5E00008F030C1BDC284E690E0D5CC83E8E82EC7
:10E5F0008CE1F82E0CE024E048E060E08BED91E146
:10E600000F94950813CF8FE59CE128CF8DEE9BE109
:10E610003ECF07E028E04AE26AE28BED91E10F94F9
:10E62000210905E022E04CE262E38BED91E10F94D9
:10E63000210924E04AE061E38AE20F94E70860914F
:10E64000DD117091DE1182E38093F7118BE28093EC
:10E65000F81127EF31E142E38BED91E10E94C49480
:10E6600066CF24E04AE461E386E30F94E70868CFCD
:10E6700002E02091E50342E367E38BED91E10F9423
:10E68000210967CF83E08093121206E200931312F0
:10E6900068E570E080E090E00E94CA528BE08093D1
:10E6A000121200931312112329F08BEE93E00E94B3
:10E6B000B55424C08091AE0480FD18C03BEEE32E1B
:10E6C00033E0F32EF70161917F016623B9F06F32D9
:10E6D00034F4062E000C770B880B990B04C06FE303
:10E6E00070E080E090E00E94CA52ECCF8091DA04A2
:10E6F00080FDDBCF8CEC9CE10E94D95388E28093B3
:10E70000121206E20093131269E570E080E090E0D7
:10E710000E94CA5280E380931212009313121123B5
:10E7200029F086EE93E00E94B55426C08091AE0495
:10E73000869580FD18C026EEE22E23E0F22EF7012A
:10E7400061917F016623C1F06F3234F4062E000C14
:10E75000770B880B990B04C06FE370E080E090E0CA
:10E760000E94CA52ECCF8091DA04869580FDD9CF01
:10E770008CEC9CE10E94D9538DE48093121206E246
:10E78000009313126AE570E080E090E00E94CA52A4
:10E7900085E58093121200931312112329F080EF64
:10E7A00093E00E94B5540BCF8091AE048695869578
:10E7B00080FD19C090EFE92E93E0F92EF7016191E9
:10E7C0007F01662309F4FBCE6F3234F4062E000C71
:10E7D000770B880B990B04C06FE370E080E090E04A
:10E7E0000E94CA52EBCF8091DA048695869580FD0F
:10E7F000D6CF89EC9CE10E94D953E1CE83E00E9400
:10E80000B75283E08093121283E38093131266E081
:10E8100070E080E090E00E94CA5281E00E94B7520E
:10E8200080911002909111020E940ED1AC0163E31D
:10E830008CE00E94F85565E270E080E090E00E9474
:10E84000CA52C6CE109212128EE38093131282EE39
:10E850009CE00E944650082F863178F482EE9CE0BE
:10E860000E94B554053109F47BC160E270E080E09C
:10E8700090E00E94CA520F5FF5CFE090E10C8E2D20
:10E8800090E09C012E51334F7901C9010E944650FE
:10E89000082F60E870E0C7010E94DD53053130F5B4
:10E8A0006EE270E080E090E00E94CA520431F1F024
:10E8B0006EE270E080E090E00E94CA520331B1F055
:10E8C000202F30E02E5F3F4F4AEF4203B001439FBD
:10E8D000700D112460587F4F82EE9CE00E94DD5342
:10E8E00060E270E080E090E00E94CA528091CE0326
:10E8F000181709F435C11093CE0382EE9CE00E94F4
:10E9000046509091E10C981788F481E0890F21E03E
:10E91000280FE82FF0E0EE51F34F9081907C903873
:10E9200011F4822FF4CF8093E10C1AC11092E10C04
:10E9300017C111112FC0809108168111CFCD2AC0A7
:10E9400080911112843108F058C0CDCD111184C0CE
:10E95000809103168111D4CD7FC080911112843132
:10E9600008F0B1C0D2CD80911112843108F0DAC024
:10E97000D1CD90FD0CC08DEB9BE17C010CE022E041
:10E9800048E060E28BED91E10F949508A2CD85ED12
:10E990009BE1F3CFB601DD0C880B990B0F941D4062
:10E9A00020E030E040E05FE30F942C470F9498485C
:10E9B000CB010E940ED1FC0180818032E1F4818183
:10E9C000803211F092E001C091E043E050E0491B39
:10E9D00051094E0F5F1F892F880F980F892F81953E
:10E9E00067E0895D0E94F85569E070E080E090E0A2
:10E9F0000E94CA5273CD93E0E8CF20E030E040E0BF
:10EA00005FE3C501B4010F942C470F949848CB01E4
:10EA10000E940ED1FC0180818032E1F4818180323C
:10EA200011F092E001C091E043E050E0491B510930
:10EA30004E0F5F1F892F880F980F892F81956CE1EA
:10EA4000895D0E94F85569E070E080E090E00E94E6
:10EA5000CA5249CD93E0E8CF60914A0E70914B0EB7
:10EA6000072E000C880B990B0F941D4020E030E01E
:10EA700040E05FE30F942C470F949848CB010E942D
:10EA80000ED1FC0180818032E1F48181803211F06D
:10EA900092E001C091E043E050E0491B51094E0F64
:10EAA0005F1F892F880F980F892F819567E0865AFD
:10EAB0000E94F85569E070E080E090E00E94CA5240
:10EAC0001FCD93E0E8CF20E030E040E05FE3C701F6
:10EAD000B6010F942C470F949848CB010E940ED199
:10EAE000FC0180818032E1F48181803211F092E07A
:10EAF00001C091E043E050E0491B51094E0F5F1FF8
:10EB0000892F880F980F892F81956CE1865A0E9472
:10EB1000F85569E070E080E090E00E94CA52F5CCC0
:10EB200093E0E8CF80917007882309F4F3CCF4E6F2
:10EB30008F9FC001112481589F4F6FEF70E00F9499
:10EB4000FD46CB010E940ED1AC016CE187E60E942C
:10EB5000F85565E270E080E090E00E94CA52DACC9D
:10EB60002C960FB6F894DEBF0FBECDBFDF91CF91CC
:10EB70001F910F91FF90EF90DF90CF90BF90AF90DB
:10EB80009F908F907F906F905F904F9008950F931C
:10EB90000FB70F9300916E000F930B7F00936E00E1
:10EBA00000916F000D7F00936F000F930BB70F93D1
:10EBB0000CB70F921F922F933F934F935F936F93D6
:10EBC0007F938F939F93AF93BF93EF93FF93112402
:10EBD0000E944376FF91EF91BF91AF919F918F91EA
:10EBE0007F916F915F914F913F912F911F900F9067
:10EBF0000CBF0F910BBF0F910260F89400936F0050
:10EC00000F9100936E000F910FBF0F911895809197
:10EC1000D90480FF03C089988FEF02C0899A81E0F0
:10EC2000809364048091D904869580FF03C08F98F7
:10EC30008FEF02C08F9A81E0809365048091D904A0
:10EC40008695869580FF08C080910B018095827023
:10EC5000809309018FEF06C080910B018270809331
:10EC6000090181E0809366048091D9048695869598
:10EC7000869580FF03C0169A8FEF02C0169881E038
:10EC80008093670408952F923F924F925F926F9204
:10EC90007F928F929F92AF92BF92CF92DF92EF922C
:10ECA000FF920F931F93CF93DF9300D01F92CDB7A6
:10ECB000DEB78FEF9FEF90938900809388000AE082
:10ECC0000983212C312C78948091AA049091AB0473
:10ECD000A091AC04B091AD04892B8A2B8B2B71F0E1
:10ECE0008091AA049091AB04A091AC04B091AD04C2
:10ECF000892B8A2B8B2B09F063C5DAC18091B9155A
:10ED00008823D1F01092B9158091B7159091B8155C
:10ED1000892B91F01092B8151092B71510926304D8
:10ED20009091931180919411981731F080919411E2
:10ED30008F5F8F70809394118091B7159091B81563
:10ED4000892B71F2C090A604D090A704E090A8048B
:10ED5000F090A9044091A2045091A3046091A404EE
:10ED60007091A5040091940410E020E030E0DB01F4
:10ED7000CA018C199D09AE09BF09081719072A078E
:10ED80003B0710F4D901C801E82F8C0D9D1DAE1D65
:10ED9000BF1D8093A6049093A704A093A804B093EA
:10EDA000A9041B821A82F1E0C0906C04D0906D041B
:10EDB000E0906E04F0906F0480917C0490917D044B
:10EDC000A0917E04B0917F04C80ED91EEA1EFB1EDE
:10EDD000C0927C04D0927D04E0927E04F0927F0485
:10EDE000F7FC31C080916404082E000C990BAA0B2B
:10EDF000BB0B4091C6155091C7156091C815709115
:10EE0000C915840F951FA61FB71F8093C615909331
:10EE1000C715A093C815B093C91580916804909147
:10EE20006904A0916A04B0916B04A7019601281BA4
:10EE3000390B4A0B5B0B20937C0430937D04409389
:10EE40007E0450937F04009170041091710420910E
:10EE50007204309173048091800490918104A09198
:10EE60008204B0918304080F191F2A1F3B1F0093CF
:10EE7000800410938104209382043093830437FD2F
:10EE800031C080916504082E000C990BAA0BBB0BB6
:10EE90004091CA155091CB156091CC157091CD154C
:10EEA000840F951FA61FB71F8093CA159093CB158B
:10EEB000A093CC15B093CD1580916804909169040E
:10EEC000A0916A04B0916B04B901A801481B590BC9
:10EED0006A0B7B0B409380045093810460938204FF
:10EEE000709383044091740450917504609176048A
:10EEF000709177048091840490918504A091860498
:10EF0000B0918704480F591F6A1F7B1F40938404E8
:10EF100050938504609386047093870477FD31C015
:10EF200080916604082E000C990BAA0BBB0B8090F5
:10EF3000CE159090CF15A090D015B090D115880D1A
:10EF4000991DAA1DBB1D8093CE159093CF15A0933C
:10EF5000D015B093D1158091680490916904A09167
:10EF60006A04B0916B042A013B01481A590A6A0AE3
:10EF70007B0A4092840450928504609286047092C9
:10EF800087048090780490907904A0907A04B090DF
:10EF90007B048091880490918904A0918A04B091A7
:10EFA0008B04880D991DAA1DBB1D80938804909326
:10EFB0008904A0938A04B0938B04B7FD31C080907C
:10EFC0006704082C000C9908AA08BB084090D215C9
:10EFD0005090D3156090D4157090D515840C951C65
:10EFE000A61CB71C8092D2159092D315A092D4156E
:10EFF000B092D5158090680490906904A0906A043E
:10F00000B0906B042C013D01481859086A087B0830
:10F01000409288045092890460928A0470928B0412
:10F02000F1110CC0A0908400B09085006A807B80B4
:10F03000A618B708F2E0AF16B104A0F3F7FE889A5D
:10F0400037FF8E9A77FD06C0F0910B01F095F870AE
:10F05000F0930901B7FF149A409084005090850006
:10F060005B824A82A0908400B09085006A807B8099
:10F07000A618B708F2E0AF16B104A0F3F7FE88981F
:10F0800037FF8E9877FD05C020910B0128702093E3
:10F090000901B7FF1498EE2331F04090840050909E
:10F0A00085005B824A82E150F0E009F07DCE18CE07
:10F0B000E091B715F091B815309709F407C5809124
:10F0C000A6049091A704A091A804B091A90440912E
:10F0D000A2045091A3046091A4047091A504841724
:10F0E0009507A607B707D0F01092B8151092B7157C
:10F0F000109263049091931180919411981709F4E0
:10F10000E5C4809194118F5F8F7080939411F0ED1E
:10F11000CF2EF7E0DF2EE12CF12C69C140919E0447
:10F1200050919F046091A0047091A1044817590761
:10F130006A077B0708F470C040919A0450919B04C1
:10F1400060919C0470919D0481A992A9A3A9B4A97E
:10F150005524499F612C5A9F90016A9F300D699FE9
:10F16000200D311D4A9F600C211D351D599F600CDB
:10F17000211D351D689F600C211D351D589F610C98
:10F18000251D351D6694251D351DB49F200D311D8F
:10F19000B59F300D112482AD93ADA4ADB5AD820FF6
:10F1A000931FA11DB11D8093960490939704A09383
:10F1B0009804B093990406A917A920AD31AD08179A
:10F1C00019072A073B0740F400939604109397040D
:10F1D000209398043093990480909604909097041B
:10F1E000A0909804B09099040090950404C0880CF5
:10F1F000991CAA1CBB1C0A94D2F78EEE97E221E060
:10F20000FC01C590D590E590F490C814D904EA04A7
:10F21000FB0408F425C32FC340919004509191043E
:10F220006091920470919304481759076A077B070D
:10F2300008F06CC040918C0450918D0460918E0454
:10F2400070918F0481A992A9A3A9B4A94424499FCC
:10F25000512C5A9F90016A9F300D699F200D311DDE
:10F260004A9F500C211D341D599F500C211D341DE7
:10F27000689F500C211D341D589F510C241D341DB6
:10F280005694241D341DB49F200D311DB59F300DA3
:10F290001124C901A0E0B0E08090960490909704FA
:10F2A000A0909804B0909904FE9688159905AA0537
:10F2B000BB0580F40081118122813381881A990A6B
:10F2C000AA0ABB0A80169106A206B30638F44801C2
:10F2D000590104C080809180A280B3800090950481
:10F2E00004C0880C991CAA1CBB1C0A94D2F78EEE91
:10F2F00097E221E0FC01C590D590E590F490C81408
:10F30000D904EA04FB0408F41EC328C380910B024D
:10F3100090910C02A0910D02B0910E02B7FF5FC058
:10F3200086A997A9A0ADB1AD0090950404C0880F3F
:10F33000991FAA1FBB1F0A94D2F72EEE37E241E0B5
:10F34000F901C590D590E590F490C816D906EA0663
:10F35000FB0658F4B695A79597958795440F2C5FB3
:10F360003F4FF8E22A303F0759F740939404803228
:10F370009105A105B10508F47CC38097A109B109E5
:10F38000811508E09007A105B10508F44FC314E00A
:10F39000919F9001112422513C4DF90132964591E3
:10F3A0005491EE27859FB001849F610D7E1F0694C6
:10F3B0006E1F7E1F1124CB01A0E0B0E0F901459142
:10F3C000549160E070E0481B590B6A0B7B0B409333
:10F3D0000B0250930C0260930D0270930E02C090CA
:10F3E0000B02D0900C02E0900D02F0900E02809182
:10F3F000B7159091B815892B09F0DAC10E941B83CB
:10F400009093B8158093B715892B09F4D1C1E09179
:10F41000B715F091B815808183FF44C0858D968D16
:10F42000A78DB0A1418D528D638D748D058916898C
:10F430002789308D0093C6151093C7152093C815E2
:10F440003093C9154093CA155093CB156093CC15D2
:10F450007093CD158093CE159093CF15A093D015B2
:10F46000B093D11581A192A1A3A1B4A18093D2158B
:10F470009093D315A093D415B093D5151092B815C9
:10F480001092B7151092630490919311809194118A
:10F49000981709F4B3CF809194118F5F8F70809388
:10F4A0009411ACCFDF01A55BBF4F8D919D910D9065
:10F4B000BC91A02D80931A0F90931B0FA0931C0F4B
:10F4C000B0931D0F85889688A788B08C81E0811441
:10F4D0009104A104B10409F480E0C18CD28CE38CC6
:10F4E000F48CC114D104E104F10409F08260058DAB
:10F4F000168D278D30A1011511052105310509F063
:10F5000084608093630410928C0410928D04109296
:10F510008E0410928F0410929A0410929B04109201
:10F520009C0410929D0446A957A960AD71AD80E07E
:10F5300042389BE159076105710560F4440F551F7E
:10F54000661F771F4238ABE15A076105710580F7E6
:10F550008F5FEECF80939504482E512C5B824A82B8
:10F5600045A156A167A170A5082E04C0440F551FE0
:10F57000661F771F0A94D2F74093A2045093A30406
:10F580006093A4047093A504442455243201441AC2
:10F59000550A660A770A40927C0450927D04609274
:10F5A0007E0470927F0440928004509281046092A5
:10F5B0008204709283044092840450928504609285
:10F5C0008604709287044092880450928904609265
:10F5D0008A0470928B0441A052A063A074A0440CD2
:10F5E000551C661C771C880C991CAA1CBB1C80929D
:10F5F0006C0490926D04A0926E04B0926F04CC0CD7
:10F60000DD1CEE1CFF1CC0927004D0927104E092CD
:10F610007204F0927304000F111F221F331F009316
:10F620007404109375042093760430937704409209
:10F6300078045092790460927A0470927B04440FAB
:10F64000551F661F771F40936804509369046093A9
:10F650006A0470936B041092A6041092A70410928F
:10F66000A8041092A90441A552A563A574A5082E6B
:10F6700004C0440F551F661F771F0A94D2F74093AA
:10F680009E0450939F046093A0047093A10445A529
:10F6900056A567A570A93A014B0104C0660C771CFA
:10F6A000881C991C8A95D2F76092900470929104FC
:10F6B000809292049092930485A99091D90489171D
:10F6C00021F08093D9040E9407768091D80481119B
:10F6D0000E94AF8A88248A94982C540180920B024D
:10F6E00090920C02A0920D02B0920E02E091B7151A
:10F6F000F091B81582AD93ADA4ADB5AD80939604ED
:10F7000090939704A0939804B09399040A8004C03E
:10F71000880F991FAA1FBB1F0A94D2F72EEE37E25B
:10F7200041E0F901C590D590E590F490C816D9064E
:10F73000EA06FB0670F4B695A79597958795440F52
:10F740002C5F3F4F6AE0462E68E2562E4216530663
:10F7500041F74093940480329105A105B10508F466
:10F76000B0C18097A109B109811508E09007A105F2
:10F77000B10508F483C114E0919F90011124225136
:10F780003C4DF901329645915491EE27859FB00189
:10F79000849F610D7E1F06946E1F7E1F1124F90148
:10F7A000C590D490E12CF12CC61AD70AE108F108D3
:10F7B000C092AA04D092AB04E092AC04F092AD04E3
:10F7C0008091AA049091AB04A091AC04B091AD04D7
:10F7D0008F3F2FEF9207A105B10528F04FEF5FEFA4
:10F7E00060E070E002C0AC01BD01841B950BA60B6C
:10F7F000B70B8093AA049093AB04A093AC04B0938E
:10F80000AD04F89480918400909185004096098120
:10F8100001500983002339F0240E351E28163906BD
:10F8200008F451CA01C01C0130928900209288005E
:10F8300078940F900F900F900F90DF91CF911F91C0
:10F840000F91FF90EF90DF90CF90BF90AF909F907F
:10F850008F907F906F905F904F903F902F90089582
:10F86000B694A79497948794220F049618E28A304E
:10F87000910709F0C5CC2093940420E282169104EC
:10F88000A104B10408F459C000E2801A9108A1084B
:10F89000B108811418E09106A104B104F8F024E045
:10F8A000929EC001112482519C4DFC0132962591FB
:10F8B0003491F82DEE27F39FD001F29FA10DBE1FCA
:10F8C0000694AE1FBE1F1124FC01C590D490E12CFC
:10F8D000F12CCA1ADB0AE108F10822C0D501C401E3
:10F8E000B695A79597958795FC01EC7FCF0182513E
:10F8F000904EFC01C590D490FC0132962591349134
:10F90000E82DE770E29FC001E39F900D1124E3E032
:10F9100096958795EA95E1F7C81AD90AE12CF12C5A
:10F920004C0D5D1D6E1D7F1D40939A0450939B04EA
:10F9300060939C0470939D045ACDA0E28A2E912C72
:10F94000A12CB12CA1CFB694A79497948794220FA1
:10F95000049638E28A30930709F0CCCC20939404C3
:10F9600080E288169104A104B10408F459C000E2B1
:10F97000801A9108A108B108811418E09106A10429
:10F98000B104F8F024E0929EC001112482519C4DF4
:10F99000FC01329625913491F82DEE27F39FD0018A
:10F9A000F29FA10DBE1F0694AE1FBE1F1124FC01C5
:10F9B000C590D490E12CF12CCA1ADB0AE108F108B9
:10F9C00022C0D501C401B695A79597958795FC01EE
:10F9D000EC7FCF018251904EFC01C590D490FC0188
:10F9E000329625913491E82DE770E29FC001E39FA4
:10F9F000900D112423E0969587952A95E1F7C81A72
:10FA0000D90AE12CF12C4C0D5D1D6E1D7F1D40931C
:10FA10008C0450938D0460938E0470938F04E7CC14
:10FA2000E0E28E2E912CA12CB12CA1CFAC01BD0116
:10FA30007695679557954795FA01EC7F9F0122517E
:10FA4000304EF90145915491F901329665917491C6
:10FA50008770869F9001879F300D1124C90113E0A4
:10FA6000969587951A95E1F7481B590B60E070E071
:10FA7000AECC80E290E0A0E0B0E07FCCAC01BD0174
:10FA80007695679557954795FA01EC7F9F0122512E
:10FA9000304EF901C590D490F901329645915491B8
:10FAA0008770849F9001859F300D1124C90103E068
:10FAB000969587950A95E1F7C81AD90AE12CF12C99
:10FAC00077CE80E290E0A0E0B0E04BCE80EDC82E93
:10FAD00087E0D82EE12CF12C91CCAF92BF92CF923F
:10FAE000DF92EF92FF920F931F93CF93C82F811154
:10FAF00002C00E9434F587ED9FE10E942CF481ED55
:10FB00009FE10E942CF48AE00E942738C11102C0B4
:10FB10000E9434F584EB9FE10E942CF48AE00E945D
:10FB20002738C11114C040E061EA7FE180E00F9402
:10FB3000AE148091510E882321F08AE00E9427386C
:10FB400004C086E99FE10E942CF40E9434F5609184
:10FB5000510E70E08DE89FE10E9410F540914D0E2E
:10FB600050914E0E60914F0E7091500E8AE89FE1B9
:10FB70000E94FFF48AE00E94273841E06AE77FE1B3
:10FB80008C2F0F94AE146FEF81E08C270F94962486
:10FB900041E06DE57FE18C2F0F94AE14C11102C0DE
:10FBA0000E9434F54091990C50919A0C60919B0CF5
:10FBB00070919C0C84E59FE10E94FFF440919D0CA4
:10FBC00050919E0C60919F0C7091A00C89E79AE374
:10FBD0000E94FFF44091A10C5091A20C6091A30CE3
:10FBE0007091A40C85E39EE10E94FFF44091A50C66
:10FBF0005091A60C6091A70C7091A80C85E29CE036
:10FC00000E94FFF48AE00E94273841E063E37FE12D
:10FC10008C2F0F94AE14C11102C00E9434F5609174
:10FC2000750C7091760C8091770C9091780C0F94F4
:10FC30001B40AB01BC018AE29FE10E94FFF460918E
:10FC4000790C70917A0C80917B0C90917C0C0F94C4
:10FC50001B40AB01BC0189E79AE30E94FFF460916D
:10FC60007D0C70917E0C80917F0C9091800C0F9494
:10FC70001B40AB01BC0185E39EE10E94FFF4609153
:10FC8000810C7091820C8091830C9091840C0F9464
:10FC90001B40AB01BC0185E29CE00E94FFF48AE0BE
:10FCA0000E94273841E061EE7EE18C2F0F94AE1464
:10FCB000C11102C00E9434F54091A90C5091AA0CC8
:10FCC0006091AB0C7091AC0C88ED9EE10E94FFF44A
:10FCD0004091AD0C5091AE0C6091AF0C7091B00C96
:10FCE00081ED9CE10E94FFF44091B10C5091B20C67
:10FCF0006091B30C7091B40C85ED9EE10E94FFF40D
:10FD00008AE00E94273841E061E87EE18C2F0F9461
:10FD1000AE14C11102C00E9434F56091850C70913F
:10FD2000860C8091870C9091880C0F941B40AB013E
:10FD3000BC0188E79EE10E94FFF44091B50C509110
:10FD4000B60C6091B70C7091B80C80E89BE00E94F3
:10FD5000FFF44091B90C5091BA0C6091BB0C7091BA
:10FD6000BC0C85ED9EE10E94FFF440915407509138
:10FD70005507609156077091570785E79EE10E94ED
:10FD8000FFF48AE00E94273841E068E67EE18C2F8C
:10FD90000F94AE14C11102C00E9434F540915E0E62
:10FDA00050915F0E6091600E7091610E8FE59EE143
:10FDB0000E94FFF44091620E5091630E6091640EB8
:10FDC0007091650E89E79AE30E94FFF44091660EF8
:10FDD0005091670E6091680E7091690E85E39EE107
:10FDE0000E94FFF48AE00E94273841E06CE47EE143
:10FDF0008C2F0F94AE14C11102C00E9434F5609193
:10FE0000410E70E083E49EE10E9410F540913D0EAA
:10FE100050913E0E60913F0E7091400E85E39EE141
:10FE20000E94FFF48AE00E9427380E94DBF38823B7
:10FE300009F44EC08FE3C82E84E0D82E00E010E015
:10FE40005601E12CF12CC11102C00E9434F5B7011A
:10FE500088E39EE10E9410F5B80185E79EE10E94CB
:10FE600010F585E39EE10E942CF4F501608171811B
:10FE70008281938145E00E94B7388AE00E9427384A
:10FE8000FFEFEF1AFF0A8CE0A80EB11CE3E0EE16BC
:10FE9000F104C9F60F5F1F4FF4E0CF0ED11C033001
:10FEA000110571F6C11102C00E9434F58DE29EE188
:10FEB0000E942CF460913B0470913C0480913D04BD
:10FEC00090913E0445E00E94B7388AE00E942738AE
:10FED00041E061E17EE18C2F0F94AE140FE214E05B
:10FEE000E12CF12CC11102C00E9434F5B70188E069
:10FEF0009EE10E9410F5F8016081718185E09EE12C
:10FF00000E94F2F4F801628173818EE79EE10E9403
:10FF1000F2F4F8016481758182E09EE10E94F2F4BE
:10FF20008AE00E942738FFEFEF1AFF0A0A5F1F4F8F
:10FF300082E0E816F104B1F641E064EF7DE18C2F38
:10FF40000F94AE14C11102C00E9434F540913A0FD3
:10FF500050913B0F60913C0F70913D0F8BEE9DE1F6
:10FF60000E94FFF42CEA35EC47E25EE360913E0F1D
:10FF700070913F0F8091400F9091410F0F94264850
:10FF8000AB01BC0180E49EE10E94FFF42CEA35EC59
:10FF900047E25EE36091420F7091430F8091440FFE
:10FFA0009091450F0F947C40AB01BC018AE89FE122
:10FFB0000E94FFF48AE00E94273841E066ED7DE16F
:10FFC0008C2F0F94AE14C11102C00E9434F56091C1
:10FFD0002E0470E08DEC9DE10E9410F58AE00E94F5
:10FFE000273841E067EA7DE18C2F0F94AE14C111F0
:10FFF00002C00E9434F540910E0450910F046091AC
:020000021000EC
:100000001004709111048EE99DE10E94FFF440916B
:1000100022045091230460912404709125048BE9FB
:100020009DE10E94FFF420E030E040E752E460915F
:1000300012047091130480911404909115040F948C
:100040007C40AB01BC0182E09EE10E94FFF4409144
:10005000160450911704609118047091190485E3F7
:100060009EE10E94FFF48AE00E94273841E06DE79C
:100070007DE18C2F0F94AE14C11102C00E9434F5A3
:1000800040911A0450911B0460911C0470911D044E
:1000900084E79DE10E94FFF44091260450912704DB
:1000A00060912804709129048BE99DE10E94FFF47E
:1000B00020E030E040E752E460911E0470911F049C
:1000C00080912004909121040F947C40AB01BC01ED
:1000D00082E09EE10E94FFF48AE00E94273841E01E
:1000E00067E27DE18C2F0F94AE14C11102C00E9413
:1000F00034F560910D0470E08EE19DE10E9410F5F1
:100100008AE00E94273841E060E07DE18C2F0F9467
:10011000AE14C11102C00E9434F584ED9CE10E942E
:100120002CF44091090450910A0460910B047091E1
:100130000C048AED9FE30E94FFF440910504509166
:10014000060460910704709108048DEF9CE10E9401
:10015000FFF48AE00E94273841E065EE7CE18C2FB5
:100160000F94AE14C11102C00E9434F560910A02CE
:1001700070E08CED9CE10E9410F58AE0CF911F9118
:100180000F91FF90EF90DF90CF90BF90AF900C94C5
:100190002738CF92DF92EF92FF928091510E882301
:1001A00071F1C0904D0ED0904E0EE0904F0EF09039
:1001B000500E20E030E0A901C701B6010F941640AF
:1001C0008823E9F020E030E040E05FE3C701B601BA
:1001D0000F947C409B01AC010F947C402BED3FE0E1
:1001E00049E450E40F947C409B01AC0160E070E076
:1001F00080E89FE30F9426486B017C0106C0C12C68
:10020000D12C80E8E82E8FE3F82EC092B704D0926C
:10021000B804E092B904F092BA04609116027091A9
:100220001702072E000C880B990B0F941D402AE033
:1002300037ED43E25CE30F947C40A70196010F94F5
:100240007C40609324027093250280932602909351
:100250002702FF90EF90DF90CF900895CF93C82FA3
:10026000CB01009711F00E942CF484EB92E40E94E1
:100270002CF4C11103C08EE098E202C083E198E241
:100280000E942CF48AE0CF910C9427384F925F9211
:100290006F927F928F929F92AF92BF92CF92DF9296
:1002A000EF92FF920F931F93CF93DF93CDB7DEB7FB
:1002B00068970FB6F894DEBF0FBECDBF8C015B010F
:1002C0005A834983DC01D6966D917D918D919C91E5
:1002D000D9970F941B406B017C01F501208131817E
:1002E000428153810F947C400F940A480F949F4899
:1002F00069877A878B879C87A981BA812D913D91E7
:100300004D915C91C701B6010F947C400F940A484F
:100310000F949F486D877E878F87988B29853A85B4
:100320004B855C85283731054105510540F488E748
:1003300090E0A0E0B0E089879A87AB87BC872D85E5
:100340003E854F855889283731054105510540F4D0
:1003500088E790E0A0E0B0E08D879E87AF87B88BFC
:10036000F801EE5BFF4F2081318142815381298367
:100370003A834B835C83CA01B9010F941D402B0162
:100380003C0169857A858B859C850F941B40698B20
:100390007A8B8B8B9C8B20E030E0A901C301B201EA
:1003A0000F941640882329F1A7019601C701B601D1
:1003B0000F947C404B015C0129893A894B895C8907
:1003C000CA01B9010F947C409B01AC01C501B40185
:1003D0000F942B474B015C01A3019201C301B201B1
:1003E0000F942C479B01AC01C501B4010F94264822
:1003F00003C060E070E0CB010F940A480F949F485F
:100400006D837E838F83988769817A818B819C81BC
:1004100090958095709561957F4F8F4F9F4F0F946A
:100420001D404B015C016D857E858F8598890F94F9
:100430001B4069837A838B839C8320E030E0A90191
:10044000C501B4010F941640882349F129813A81EE
:100450004B815C81CA01B9010F947C406D8B7E8B0E
:100460008F8B988FA7019601C701B6010F947C402E
:100470009B01AC016D897E898F89988D0F942B47E4
:100480006B017C01A5019401C501B4010F942C47B7
:100490009B01AC01C701B6010F94264803C060E080
:1004A00070E0CB010F94CE48D80195968D909D9029
:1004B000AD90BC909897750164012D813E814F816C
:1004C0005885C21AD30AE40AF50A0F949F48C61A3F
:1004D000D70AE80AF90AF7FE75C020E030E0A90162
:1004E000C301B2010F941640882309F443C0C5012B
:1004F000B4010F941B406B017C01A3019201C30165
:10050000B2010F942C479B01AC01C701B6010F94B7
:100510007C406B017C0129893A894B895C89CA013D
:10052000B9010F947C409B01AC01C701B6010F9447
:100530002B476B017C0129813A814B815C81CA0187
:10054000B9010F947C409B01AC01C701B6010F9427
:100550002C476B017C0120E030E040E850E4C3010F
:10056000B2010F947C409B01AC01C701B6010F940E
:10057000264803C060E070E0CB010F940A487B017D
:100580008D83998320E030E0A9010F948C491816DF
:1005900024F0E12CF12C1D821982B7018D81998103
:1005A0000F949F486D837E838F8398878616970666
:1005B000A806B90620F48D829E82AF82B886C12C2F
:1005C000D12C76018D819E81AF81B885F80181A7FC
:1005D00092A7A3A7B4A7C80ED91EEA1EFB1EC5A6E4
:1005E000D6A6E7A6F0AA29853A854B855C8522AF79
:1005F00033AF44AF55AFFE962D853E854F85588964
:10060000208331834283538368960FB6F894DEBF0C
:100610000FBECDBFDF91CF911F910F91FF90EF9053
:10062000DF90CF90BF90AF909F908F907F906F9012
:100630005F904F900895CF93DF93809193119091A5
:100640009411891B8F7009F445C0909190119923E2
:1006500051F0833030F48FEF890F19F080939011AF
:100660003BC010929011E09194118FE4E89FF0014B
:100670001124EE57F84F808180FD2EC080916C07C9
:1006800090916D07A0916E07B0916F07EF01C95B64
:10069000DF4F488159816A817B81841B950BA60BB2
:1006A000B70B80936C0790936D07A0936E07B09380
:1006B0006F07809194118F5F8F708093911190914B
:1006C00094118091921198130AC080919111809396
:1006D000921105C00E9470EB80E090E001C0CF0154
:1006E000DF91CF9108952F923F924F925F926F9238
:1006F0007F928F929F92AF92BF92CF92DF92EF92B2
:10070000FF920F931F93CF93DF93CDB7DEB762971E
:100710000FB6F894DEBF0FBECDBF788B6F87DC01BC
:100720008D909D90AD90BC90139714962D913D9116
:100730004D915C9117972D833E834F83588720E01E
:1007400030E040E251E4C501B4010F942B4726ED9F
:1007500039EB42EF5BE30F947C400F9498481616F8
:1007600014F461E002C067FD60E0E62E660FFF084A
:10077000F701EE0FFF1FEE0FFF1FEB5DFD4E4080F8
:1007800051806280738087010F5F1F4F20E030E04F
:1007900040E251E46D817E818F8198850F942B47D3
:1007A00025E338E74EE05CE30F947C400F949848D3
:1007B000161614F461E002C067FD60E0E62F660FD4
:1007C000FF0BFA8BE98BEE0FFF1FEE0FFF1FEB5DA8
:1007D000FD4E208131814281538129833A834B83AD
:1007E0005C8329883A883FEF231A330AB701660FE2
:1007F000771FAB014E0D5F1D5A874987FA01898922
:100800009A89E80FF91FEE0FFF1FEE0FFF1FE15C43
:10081000FB4FC080D180E280F380F801EE0FFF1F14
:10082000EE0FFF1FEB5DFD4EA30192016081718110
:10083000828193810F942B476B877C878D879E875E
:10084000A3019201C501B4010F942B472B013C0178
:10085000C801880F991F080F191FA989BA89A00F0D
:10086000B11FAA0FBB1FAA0FBB1FA15CBB4FA701E3
:1008700096016D917D918D919C910F942B472B85C5
:100880003C854D855E850F942648A30192010F9407
:100890007C40A70196010F942C476B017C01E985F0
:1008A000FA85E20DF31DEE0FFF1FEE0FFF1FE15C57
:1008B000FB4F80809180A280B380020D131DF80150
:1008C000EE0FFF1FEE0FFF1FE15CFB4FA501940130
:1008D00060817181828193810F942B472B853C85A8
:1008E0004D855E850F942648A30192010F947C40AC
:1008F000A50194010F942C47A70196010F942B4753
:100900004B015C01F101EE0FFF1FEE0FFF1FEB5DCE
:10091000FD4E29813A814B815C81608171818281A8
:1009200093810F942B479B01AC01C501B4010F9437
:1009300026484B015C0129813A814B815C816D81A4
:100940007E818F8198850F942B479B01AC01C50157
:10095000B4010F947C40A70196010F942C47EF85BA
:10096000F88920813181428153810F947C4020910C
:100970003B0430913C0440913D0450913E040F945F
:100980002C4762960FB6F894DEBF0FBECDBFDF9145
:10099000CF911F910F91FF90EF90DF90CF90BF907C
:1009A000AF909F908F907F906F905F904F903F900F
:1009B0002F90089590916F0081E091FD02C080E03A
:1009C000089590916F009D7F90936F000895EFE6DA
:1009D000F0E080818260808308958F929F92AF9231
:1009E000BF92CF92DF92EF92FF92CF93DF93EC0111
:1009F00080903D0E90903E0EA0903F0EB090400E25
:100A000020E030E0A901C501B4010F94164088230D
:100A100009F44AC0C880D980EA80FB80A70196010A
:100A2000C501B4010F94164018160CF042C0209175
:100A3000B3043091B4044091B5045091B604C70199
:100A4000B6010F941640882331F1C092B304D092BE
:100A5000B404E092B504F092B6042091AF04309152
:100A6000B0044091B1045091B204688179818A81C7
:100A70009B810F947C409B01AC0160E070E080E8BA
:100A80009FE30F942B47609312027093130280939D
:100A900014029093150260911202709113028091DA
:100AA00014029091150208C060E070E080E89FE3B6
:100AB00003C060E070E0CB01DF91CF91FF90EF9039
:100AC000DF90CF90BF90AF909F908F900895CF937D
:100AD000DF9324E0829FC0011124EC01CF59DE4E48
:100AE000FC01E25AF14FDC01AE5AB14F2D913D911C
:100AF0004D915C9160817181828193810F942C472B
:100B0000688379838A839B83DF91CF91089580FFE7
:100B100004C09091AE0490FD8E7F81FF04C090913F
:100B2000AE0491FD8D7F82FF04C09091AE0492FDD2
:100B30008B7F0895CF92DF92EF92FF921F93CF9316
:100B4000DF9320910F02222309F48DC0EC01109154
:100B5000AE0410FF2CC0C0903902D0903A02E09051
:100B60003B02F0903C02288139814A815B81C701B8
:100B7000B6010F948C49181624F4C882D982EA82EF
:100B8000FB82C0904502D0904602E0904702F09070
:100B90004802288139814A815B81C701B6010F94DF
:100BA000164087FF04C0C882D982EA82FB8211FF07
:100BB0002CC0C0903D02D0903E02E0903F02F090E9
:100BC00040022C813D814E815F81C701B6010F94A7
:100BD0008C49181624F4CC82DD82EE82FF82C0900C
:100BE0004902D0904A02E0904B02F0904C022C81D6
:100BF0003D814E815F81C701B6010F94164087FF8A
:100C000004C0CC82DD82EE82FF8212FF2CC0C09035
:100C10004102D0904202E0904302F09044022885C5
:100C200039854A855B85C701B6010F948C49181632
:100C300024F4C886D986EA86FB86C0904D02D090FF
:100C40004E02E0904F02F0905002288539854A8587
:100C50005B85C701B6010F94164087FF04C0C886A4
:100C6000D986EA86FB86DF91CF911F91FF90EF90A6
:100C7000DF90CF9008952F923F924F925F926F92A4
:100C80007F928F929F92AF92BF92CF92DF92EF921C
:100C9000FF920F931F93CF93DF93CDB7DEB7A69745
:100CA0000FB6F894DEBF0FBECDBF86ED9DE00E946B
:100CB0009A858091740C83FD83C020915D113091E1
:100CC0005E1140915F11509160116091E20D709141
:100CD000E30D8091E40D9091E50D0F94164088236B
:100CE00009F46EC080918107811119C06091330FA2
:100CF0007091340F8091350F9091360F0F94984872
:100D000020912802309129026217730744F40E944F
:100D100034F58DE295E30E942CF411E001C010E05F
:100D200020915D1130915E1140915F1150916011E1
:100D30006091E20D7091E30D8091E40D9091E50DCD
:100D40000F942B476B017C0120E030E0A9010F9448
:100D50008C4987FF04C0F7FAF094F7F8F0942091DB
:100D60002402309125024091260250912702C701AA
:100D7000B6010F947C4020E030E048E453E40F9447
:100D80008C4918163CF40E9434F58EE095E30E94DD
:100D90002CF402C01123A1F08091E20D9091E30D9B
:100DA000A091E40DB091E50D80935D1190935E11DB
:100DB000A0935F11B093601182EE9DE00E94C1ECA0
:100DC0002AE037ED43E25CE36091560270915702EE
:100DD00080915802909159020F947C406B017C01E4
:100DE0006091100270911102072E000C880B990B74
:100DF0000F941D409B01AC01C701B6010F947C40CC
:100E0000698B7A8B8B8B9C8B8091410E882309F4A4
:100E10008CC0C0903D0ED0903E0EE0903F0EF09002
:100E2000400E20E030E0A901C701B6010F94164042
:100E3000882379F02091DE0D3091DF0D4091E00D97
:100E40005091E10DC701B6010F948C4918160CF0B2
:100E50006CC0209151113091521140915311509119
:100E600054116091D60D7091D70D8091D80D90914D
:100E7000D90D0F942B476D8B7E8B8F8B988F209184
:100E80005511309156114091571150915811609160
:100E9000DA0D7091DB0D8091DC0D9091DD0D0F94DA
:100EA0002B47698F7A8F8B8F9C8F209159113091AE
:100EB0005A1140915B1150915C116091DE0D70915F
:100EC000DF0D8091E00D9091E10D0F942B476D8F18
:100ED0007E8F8F8F98A320915D1130915E1140918C
:100EE0005F11509160116091E20D7091E30D80915E
:100EF000E40D9091E50D0F942B476B017C0120E0F0
:100F000030E0A9016D897E898F89988D0F941640F4
:100F100081113DC020E030E0A901698D7A8D8B8D73
:100F20009C8D0F941640811132C0C12CD12C7601BA
:100F30008E010F5E1F4F22EE3DE04EED5DE06AED4B
:100F40007DE086ED9DE00E9468B980E1E6EDFDE080
:100F5000A1E5B1E101900D928A95E1F7A6960FB651
:100F6000F894DEBF0FBECDBFDF91CF911F910F91DF
:100F7000FF90EF90DF90CF90BF90AF909F908F90B9
:100F80007F906F905F904F903F902F9008952D89A4
:100F90003E894F89588DCA01B9010F947C404B019D
:100FA0005C01298D3A8D4B8D5C8DCA01B9010F947E
:100FB0007C409B01AC01C501B4010F942C474B014F
:100FC0005C012D8D3E8D4F8D58A1CA01B9010F9442
:100FD0007C409B01AC01C501B4010F942C474B012F
:100FE0005C01A7019601C701B6010F947C409B01EB
:100FF000AC01C501B4010F942C470F94DA494B01A1
:101000005C012DEB37E346E855E30F94164087FF6C
:101010000FC020E030E0A901C701B6010F948C4950
:101020004601570187FF04C0B7FAB094B7F8B094EF
:101030002DEB37E346E855E3C501B4010F941640A4
:1010400087FD83CF20E030E040EA50E4C501B401E1
:101050000F9426480F949F481B01672B19F42224F4
:101060002394312CB10180E090E00F941B409B0150
:10107000AC0160E070E080E89FE30F9426482B010C
:101080003C019B01AC01C501B4010F947C404B01B4
:101090005C01A30192016D897E898F89988D0F94DF
:1010A0007C406D8B7E8B8F8B988FA3019201698D15
:1010B0007A8D8B8D9C8D0F947C40698F7A8F8B8F6E
:1010C0009C8FA30192016D8D7E8D8F8D98A10F94C1
:1010D0007C406D8F7E8F8F8F98A3A3019201C701F3
:1010E000B6010F947C4069A37AA38BA39CA380E1F3
:1010F000E1E5F1E18E010F5F1F4FD80101900D92E4
:101100008A95E1F70E947BFA2B013C0128EC420E04
:10111000511C611C711C0DA31EA381E0281A31080B
:1011200019F47501640104CF0E947BFA8B019C01C4
:10113000041915092609370937FD0BC02B013C019D
:1011400028EC420E511C611C711C80E00E94533936
:1011500002C00F949D2A2D893E894F89588D69813F
:101160007A818B819C810F942C4769837A838B834E
:101170009C83298D3A8D4B8D5C8D6D817E818F8115
:1011800098850F942C476D837E838F8398872D8D50
:101190003E8D4F8D58A169857A858B859C850F94EE
:1011A0002C4769877A878B879C8729A13AA14BA115
:1011B0005CA16D857E858F8598890F942C476D87FE
:1011C0007E878F87988B750164018E010F5E1F4F9C
:1011D0009E01235F3F4FAE01475F5F4FBE016B5FD4
:1011E0007F4F8DA19EA10E9468B9811196CF99CFA2
:1011F0008F929F92AF92BF92CF92DF92EF92FF9227
:10120000CF93DF938090560290905702A09058029F
:10121000B0905902FC01C080D180E280F38020E0D0
:1012200030E0A901C701B6010F941640882341F0B0
:10123000C0925602D0925702E0925802F0925902A0
:10124000C0911002D091110284E690E090931102B7
:1012500080931002C0902402D0902502E0902602D4
:10126000F090270280E090E0A0E8BFE380932402A2
:1012700090932502A0932602B09327020E943B86FA
:101280008092560290925702A0925802B092590250
:10129000D0931102C0931002C0922402D092250272
:1012A000E0922602F0922702DF91CF91FF90EF901B
:1012B000DF90CF90BF90AF909F908F900895CF9286
:1012C000DF92EF92FF920F931F93C12CD12C7601E6
:1012D0008C012DE531E149E551E165E571E181E5FB
:1012E00091E10E9468B91F910F91FF90EF90DF90FC
:1012F000CF9008954F925F926F927F928F929F92BC
:10130000AF92BF92CF92DF92EF92FF920F931F9313
:10131000CF93DF93CDB7DEB72C970FB6F894DEBF2F
:101320000FBECDBF2B013C0129873A874B875C87D5
:1013300047015801F601E080F1800281138120E02D
:1013400030E0A901B701C8010F94164081110BC00C
:10135000E1E8F8E285919591A591B491582F492F34
:101360003A2F2B2F04C05E2D4F2D302F212F852F8C
:10137000942FA32FB22F89839A83AB83BC8320E061
:1013800030E0A901B701C8010F941640811104C0D3
:10139000E12CF12C08E412E4C701D8018D839E836F
:1013A000AF83B887A50194016091591170915A11CA
:1013B00080915B1190915C110F94164087FF0CC0D7
:1013C0008092591190925A11A0925B11B0925C11C7
:1013D000CE0101960E945F894092511150925211A4
:1013E000609253117092541189859A85AB85BC85A2
:1013F0008093551190935611A0935711B0935811A3
:10140000CE0105960E945F892091591130915A11A1
:1014100040915B1150915C11C501B4010F941640CD
:1014200087FF0CC08092591190925A11A0925B11C3
:10143000B0925C11CE0101960E945F890E94B0ECCF
:101440002C960FB6F894DEBF0FBECDBFDF91CF91C3
:101450001F910F91FF90EF90DF90CF90BF90AF90D2
:101460009F908F907F906F905F904F900895CF9254
:10147000DF92EF92FF920F931F936B01FC01E080CC
:10148000F18002811381E1E5F1E12481358146811A
:10149000578160817181828193810E947A891F9135
:1014A0000F91FF90EF90DF90CF900895EF92FF9211
:1014B0000F931F93CF93DF937C018B010E9497EED4
:1014C000C1E5D1E12091240230912502409126020C
:1014D00050912702F70160817181828193810F947D
:1014E00026482C853D854E855F850F942C476C875B
:1014F0007D878E879F87C8010E945F89DF91CF918A
:101500001F910F91FF90EF900C94B0EC0D94540448
:10151000CF93DF93CDB7DEB72C970FB6F894DEBF2D
:101520000FBECDBF0F94AC0A0E94DA849CE0E6ECBB
:10153000F5E1DE01119601900D929A95E1F7811186
:101540000E94E784CE0101960F94012E2C960FB6CF
:10155000F894DEBF0FBECDBFDF91CF91089580918B
:10156000BB04659B02C0816001C08E7F8093BB0479
:10157000909103018091BB0491FF02C0826001C081
:101580008D7F8093BB048091BB044B9B02C0846021
:1015900001C08B7F8093BB048091630480FF10C0E7
:1015A0008091D90480FF0CC08091BB0480FF08C0EB
:1015B0008091A00681608093A00680E00F94352E74
:1015C00080916304869580FF11C08091D90486952F
:1015D00080FF0CC08091BB0481FF08C08091A006F1
:1015E00082608093A00681E00F94352E8091630481
:1015F0008695869580FF12C08091D9048695869540
:1016000080FF0CC08091BB0482FF08C08091A006BF
:1016100084608093A00682E00D94352E08958FE2B9
:1016200098E20E942CF48CB169E278E285FB88276D
:1016300080F90E942E818091030163E278E2869511
:1016400081700E942E8189B16DE178E283FB882749
:1016500080F90E942E8182B368E878E185FB8827B3
:1016600080F90C942E818091D804882331F062E0B7
:1016700070E080E090E00C9408F408950F931F93BD
:101680008091380E813019F40E947BFA08C0609175
:10169000800D7091810D8091820D9091830D00914C
:1016A000780D1091790D20917A0D30917B0D601B92
:1016B000710B820B930B28EE33E040E050E00F9467
:1016C0006C4680917C0D90917D0DA0917E0DB09126
:1016D0007F0DBC01CD01620F731F841F951F1F91E9
:1016E0000F9108951092380E1092780D1092790D86
:1016F00010927A0D10927B0D1092800D1092810D38
:101700001092820D1092830D10927C0D10927D0D1F
:1017100010927E0D10927F0D08958091380E8130C9
:1017200079F482E08093380E0E947BFA6093800DFA
:101730007093810D8093820D9093830D81E00895C5
:1017400080E00895CF92DF92EF92FF920F931F9364
:10175000CF93DF936C017A018B01C0E0D0E0CE150E
:10176000DF0581F0D8016D918D01D601ED91FC91DD
:101770000190F081E02DC6011995892B11F0219679
:10178000EECF7E01C701DF91CF911F910F91FF90A6
:10179000EF90DF90CF90089508950F943E4A1F92E6
:1017A0000F920FB60F9211242F933F938F939F9315
:1017B000AF93BF9380919A0D90919B0DA0919C0D3A
:1017C000B0919D0D3091A40623E0230F2D3720F416
:1017D0000196A11DB11D05C026E8230F0296A11D8B
:1017E000B11D2093A40680939A0D90939B0DA09316
:1017F0009C0DB0939D0D80919E0D90919F0DA09199
:10180000A00DB091A10D0196A11DB11D80939E0D5B
:1018100090939F0DA093A00DB093A10DBF91AF9198
:101820009F918F913F912F910F900FBE0F901F901E
:1018300018951F920F920FB60F9211240BB60F92AC
:101840002F933F934F935F936F937F938F939F93C8
:10185000AF93BF93EF93FF938091BF049091C00427
:10186000A091C104B091C204892B8A2B8B2B59F112
:101870009091BE04E091BC04F091BD048081892761
:1018800080838091BF049091C004A091C104B09165
:10189000C204181619061A061B060CF056C08091D1
:1018A000BF049091C004A091C104B091C2040197FB
:1018B000A109B1098093BF049093C004A093C1040F
:1018C000B093C20442C080911802E7E9F8E2E491C3
:1018D0009FEF90931802E230C9F050F4EE2399F094
:1018E000E13081F590916F009D7F90936F002AC049
:1018F000E43019F1E0F0E53029F5909173009D7F17
:10190000909373001FC010926E001CC090917000E5
:101910009D7F9093700091E09093B0009091B10002
:10192000987F94609093B1001092B3000BC0909197
:1019300071009D7F9093710005C0909172009D7F12
:101940009093720060E00E940DF9FF91EF91BF91BA
:10195000AF919F918F917F916F915F914F913F9147
:101960002F910F900BBE0F900FBE0F901F901895E8
:10197000FC0130819281930F92832181921760F450
:1019800094819F5F94838381830F821710F08FEF80
:10199000820F838381E0089580E00895FC01128224
:1019A00080818150838314820895FB014181DC0191
:1019B00012962C911297421768F013962C91139758
:1019C000241740F0608115962C91621718F4248139
:1019D0000C9497940895FC01A081B1811C92A2817E
:1019E000B3818C918F5F8C930280F381E02D908185
:1019F0008CE0899F800D1124E7EDF1E113AE84AFF7
:101A000008956091160270911702072E000C880B42
:101A1000990B0F941D402AE037ED43E25CE30F94ED
:101A20007C402091B7043091B8044091B9045091A2
:101A3000BA040F947C406093240270932502809333
:101A400026029093270208958091AC0D811104C065
:101A50008091B10D8093700708958091AC0D811134
:101A600004C08091B10D80937007089520E040E09C
:101A700060E070E08AE49DE80E948E4C81E08093F3
:101A80003A0D1092A6061092A50608950D94310EF7
:101A90000D94310E8F929F92AF92BF92CF92DF92B0
:101AA000EF92FF92CF938091A80D1092A80D8823FA
:101AB00059F0CF91FF90EF90DF90CF90BF90AF9013
:101AC0009F908F900C94244EC090BF0DD090C00D6D
:101AD000E090C10DF090C20DC114D104E104F104F5
:101AE00021F11092BF0D1092C00D1092C10D1092F5
:101AF000C20D81E080936E0284E00E94878581118F
:101B000019C08091A5069091A6068C0D9D1D9093FD
:101B1000A6068093A5068091D50C9091D60CC80E90
:101B2000D91ED092D60CC092D50C80916E0288231B
:101B300009F4B0C06091A5067091A606072E000CAE
:101B4000880B990B0F941D402091790730917A07EB
:101B500040917B0750917C070F947C406B017C0186
:101B600020E030E040E251E40F947C4020E030E09F
:101B70004AE754E40F947C404B015C0120E030E0E4
:101B8000A901C701B6010F94164087FD05C020E0EA
:101B900030E040EA50E404C020E030E040EA50EC9D
:101BA000C501B4010F942C4720E030E040E251E43D
:101BB0000F9426480F9498486B017C0197FF0AC048
:101BC000F094E094D094C094C11CD11CE11CF11C91
:101BD0008DE201C08BE280933B0DC701B60120E18D
:101BE00037E240E050E00F948E468AE0882E912C38
:101BF000A12CB12CCA01B901A50194010F948E4604
:101C0000605D60933C0DC701B60128EE33E040E013
